:020000040001F9
:109000000060002021C5010049C501004BC50100D9
:109010004DC501004FC5010051C501000000000011
:1090200000000000000000000000000053C5010027
:1090300055C501000000000057C5010059C50100D9
:10904000C9E201005BC501002DE301005BC5010021
:109050005BC50100000000005BC50100A9E3010041
:109060005BC501005BC501005BC501005BC501007C
:109070005BC501005BC501005BC501005BC501006C
:109080005BC501005D5002005BC501005BC50100CE
:10909000195102005BC50100FD4D02005BC50100D6
:1090A0005BC501005BC5010000000000000000007E
:1090B0005BC501005BC5010000000000000000006E
:1090C00000000000000000000000000000000000A0
:1090D0000000000000000000000000000000000090
:1090E0000000000000000000000000000000000080
:1090F0000000000000000000000000000000000070
:10910000000000000000000000000000000000005F
:10911000000000000000000000000000000000004F
:10912000000000000000000000000000000000003F
:10913000000000000000000000000000000000002F
:10914000000000000000000000000000000000001F
:10915000000000000000000000000000000000000F
:1091600000000000000000000000000000000000FF
:1091700000000000000000000000000000000000EF
:1091800000000000000000000000000000000000DF
:1091900000000000000000000000000000000000CF
:1091A00000000000000000000000000000000000BF
:1091B00000000000000000000000000000000000AF
:1091C000000000000000000000000000000000009F
:1091D000000000000000000000000000000000008F
:1091E000000000000000000000000000000000007F
:1091F000000000000000000000000000000000006F
:1092000010B5054C237833B9044B13B10448AFF3C0
:1092100000800123237010BDD41E00200000000038
:10922000FC58020008B5034B1BB103490348AFF3D8
:10923000008008BD00000000D81E0020FC5802007D
:10924000154B002B08BF134B9D46A3F5803A002118
:109250008B460F461348144A121A0CF0AFF90F4B05
:10926000002B00D098470E4B002B00D098470020D1
:10927000002104000D000D48002802D00C48AFF377
:1092800000800CF05DF92000290005F077FE0CF05D
:1092900043F900BF0000080000600020000000004B
:1092A00000000000D41E0020A433002000000000B5
:1092B00000000000074B1B781BB149F6FF1003F0BC
:1092C00089B8054B05481B78002B08BF6FF07F401D
:1092D000F5E700BFF21E0020F01E0020FFFF660031
:1092E000013838B5082811D8DFE800F034423E4E86
:1092F00005102E102200CCB2022C35D0032C06D043
:10930000012C03D103F072F8224B1C7038BD214BA5
:109310001B78002BFAD0204D142445F001054FF4A2
:109320007A40A847013CFAD1BDE8384003F0B6B80E
:10933000C9B2022903D00329E8D1012000E00020AE
:10934000BDE8384003F0DAB8C9B20229134B09D19D
:10935000012208E0C9B2012903D00229D6D1104B5D
:10936000F6E70F4B00221A70BDE83840FFF7A2BFA6
:1093700011F0FF0103D00229C8D10A4800E00A48D1
:10938000BDE8384003F026B84FF0FF10BDE8384084
:1093900003F091B8F11E0020B0560200F21E00202A
:1093A000F01E00208000FF0000FFFF00114870B594
:1093B00005234FF0A04140F20364012513F1FF3370
:1093C00008D20D490E234FF0A0400C2413F1FF33B7
:1093D0000AD270BD1A5C02F5E07605FA02F241F895
:1093E0002640C1F80825E9E75A5C02F5E07240F82A
:1093F0002240EBE7C4560200B65602002DE9F843BE
:109400002F4DDFF8C8C0DFF8C8E0DFF8B8800021D2
:1094100001274FF0A042284611F80C3007FA03F359
:10942000C2F80C35242300BF013BFCD11C4614F8C4
:109430000E90D2F8106526FA09F6F6075CBF07FA17
:1094400004F6334304F1010458BF9BB20E2CEED155
:1094500035F811409C421EBF25F81130052388F8CD
:1094600000304FF00073C2F808354FF08053C2F857
:1094700008354FF00053C2F8083501314FF08043F2
:10948000C2F8083505294FF08063C2F80835C3D10A
:109490000C4A13782BB1013BDBB2137023B100F0FF
:1094A00025F90120BDE8F883074B02881A8042881D
:1094B0005A8082889A80C288DA8002891A81F0E70D
:1094C000FE1E0020481B0020F41E0020C45602008F
:1094D000B6560200014B33F810007047F41E00200E
:1094E00010B50C4C00214FF0A0430222085D013161
:1094F00000F5E0700E2943F82020F7D1C3F8642767
:10950000C3F87027C3F87427C3F87827C3F868270F
:1095100010BD00BFB656020070B50F4E00224FF0CE
:10952000A04303250120915D013201F5E0740E2A6C
:1095300000FA01F143F82450C3F80815F3D1074AA3
:10954000C3F86427C3F87027C3F87427C3F87827D3
:10955000C3F8682770BD00BFB656020004000200C1
:1095600013B50949684604F057FC019C14B920461C
:1095700002B010BD2468E36898470028F7D1684618
:1095800004F053FCF1E700BFCC56020010B5FFF722
:10959000E7FF18B10368BDE81040184710BD70B56B
:1095A00004460D461646FFF7DBFF30B143683246EE
:1095B00029462046BDE87040184770BD064B1B7811
:1095C000024633B1054B1B781BB11C218020FFF7ED
:1095D000E6BF08210020FAE7081F0020BA1B002080
:1095E000024605210120FFF7DABF07B502AA0221D2
:1095F00022F8020D0846FFF7D2FF03B05DF804FB26
:1096000007B502AA022122F8020D0320FFF7C7FFC7
:1096100003B05DF804FB10B5FFF7A2FF18B1836833
:10962000BDE810401847012010BD0000014803F0BC
:1096300075B800BF1405EDFE10B504460A480BF0DE
:1096400049FF08B103F06AF8002C40F233314FF0C3
:10965000000208BF522104480BF0F8FE18B1BDE823
:10966000104003F05BB810BD2C1F002010B5064C55
:1096700000F0C8FE2268904202D80020FFF7DCFF0D
:109680000023236010BD00BF6C1F002010B505F043
:109690000DF90F4B0F4C1B7813B123680133236076
:1096A00000F0B0FE2368984208D10120FFF7C4FF04
:1096B00000210A20BDE8104000F048BE00F0B0FED6
:1096C00023689842F4D1012005F040FCF0E700BF88
:1096D000601B00206C1F002001F0ECBB82B002ABCD
:1096E00003E9030002B0FFF7C1BF000008B5002284
:1096F000082104480BF0AAFE18B1BDE8084003F0A9
:109700000DB808BD0C1F002008B5002252210948E1
:109710000BF09CFE08B103F001F800224FF4005159
:1097200005480BF093FE18B1BDE8084002F0F6BF03
:1097300008BD00BF2C1F00204C1F0020044B1A78CE
:10974000824203D0187008B9FFF790BF704700BF7E
:10975000601B002007B501F0A3FB00F0E7F801F063
:109760008FF801F09FFB1A4801F064FB194A1A4870
:1097700001210BF059FE08B102F0D0FF154A17483D
:1097800000210BF051FE08B102F0C8FF144A154841
:1097900001210BF049FE08B102F0C0FF01F038FAD8
:1097A000114A92E803006B4683E803000F4918460C
:1097B00005F056F808B102F0B1FF0D4805F08CF83D
:1097C00008B102F0ABFF05F065F803B05DF804FBEB
:1097D0004C1B0020D9960100E4560200E05602001E
:1097E0008D960100E8560200D85602002D96010021
:1097F00084320020704708B50BF088FEC00808BD11
:1098000008B5FFF7F8FF4FF6FF73B0FBF3F318440A
:1098100080B208BD3CDF704708B5B1210020FFF7DA
:10982000F9FF0220BDE8084004F0A4BA10B50446D0
:1098300000F064F821460B20BDE8104000F0E0BDC8
:109840002DE9F843837880460F46154613B179B168
:10985000012924D0184E194CA41BA4084FF000096C
:109860005FFA89F39C4209F101091DD8BDE8F8832C
:10987000012A0BD006D3022A0ED00F2AEAD1FFF715
:10988000CBFFE7E7022005F061FBE3E70C4A137822
:1098900083F001031370DDE706F0B8F8DAE7002A79
:1098A000D8D101F025F8D5E756F823302A463946B5
:1098B00040469847D4E700BFCC1E0020CC1E0020B5
:1098C000BA1B0020092816D1022902D0032907D08B
:1098D00070474FF0A0434FF40022C3F80C257047A7
:1098E000054B1B7813F0020F4FF400224FF0A043FA
:1098F000F3D0C3F808257047701F0020074B18707D
:109900004FF0A04310F0020F4FF400220CBFC3F839
:109910000C25C3F8082501F09FB900BF701F002077
:109920004FF0A0430222C3F84C2770474FF0A043EA
:109930000322C3F84C27704770B51C4C2278052AC7
:1099400023D80D466B1ADBB2984210D915F8013BAB
:10995000A3F11E06092E19D8511C21701D3B0A20A7
:1099600093FBF0F100FB1133114930338B5401218B
:10997000022000F045FD2378062B06D10C48002379
:10998000837105F0F3FCFF23237070BDA3F159062A
:10999000092E03D8511C2170583BE0E72A2BD1D166
:1099A000002ACFD0013A2270E1E700BF611B0020FE
:1099B00085320020014B00221A707047611B002085
:1099C00041DF704728DF704706490022535C33B9F6
:1099D0000132B2F50C7FF9D1034A137070470123AD
:1099E000FAE700BFE81F0020881B002082B045284E
:1099F000ADF804101ED89DF804200D2A1AD89DF841
:109A00000530042B16D80C49097851B1C3EBC303B8
:109A10005B00462111FB0030084B1A44105C02B079
:109A20007047462148430E2101FB030304480344C9
:109A3000985CF4E70020F2E7881B0020E81F002074
:109A400018560200094B1B7853B100F14003084A35
:109A50005B00DBB2D118D05C497800EB0120704785
:109A6000044BC03833F81000704700BF881B00203B
:109A7000901F00200856020030B5807858B10D487C
:109A800049B10023C25C5C1CA4B22AB9013911F0AF
:109A9000FF0101D1204430BD551E012D02D9743A79
:109AA000012A05D802339BB2FF2BEBD90020F2E745
:109AB0002346F9E72422002010B5094A0949107805
:109AC0000B6818B9084C24689C4207D00133052B59
:109AD000A8BF00230B6008B10023137010BD00BFA6
:109AE000E01F0020E41F0020DC1F00207FB501AC38
:109AF00084E807000F4E104A33680C2505FB032548
:109B000094E80700013385E80700052293FBF2F291
:109B100002EB82029B1A094A33601078084910B19F
:109B20000B6004B070BD09688B4204BF0123137041
:109B3000F7E700BFDC1F00208C320020E01F002070
:109B4000E41F002030B50C4685B00146054620468E
:109B500003F00EFD07280ED103F05CFDCDE90154A2
:109B600000238DF80C3004AB13E9070005B0BDE805
:109B70003040FFF7BBBF05B030BD30B5002389B022
:109B800004460D46CDE90133CDE903330A4601AB66
:109B90004188008803F062FDD0B903A9284603F08C
:109BA0009DFC039B5A88A3689A4209D192000499AC
:109BB00060680BF0F8FC284603F0B4FC09B030BD37
:109BC000284603F0AFFC29462046FFF7BBFFF5E728
:109BD0002146284603F0C8FC07280BD103F01AFDE4
:109BE000CDE9054501238DF81C3008AB13E90700CA
:109BF000FFF77CFFA2686068920000210BF0DEFC9A
:109C0000DCE70000064B1B783BB9064B1868064B97
:109C10001B68C31A5842584170470020704700BF64
:109C2000E01F0020DC1F0020E41F002008B5FFF724
:109C3000E9FF30B9044B1868044B0C2202FB0030DA
:109C400008BD0020FCE700BFE41F00208C3200208C
:109C500010B50446E00705D50D490E48FFF78DFF06
:109C6000FFF7B2FEA10703D50B490C48FFF785FFAC
:109C7000620703D50A490B48FFF77FFF230705D585
:109C800009490A48BDE81040FFF777BF10BD00BF83
:109C9000182200207C1B0020D01F0020701B0020F9
:109CA000242300208C1B0020841F0020641B002024
:109CB00010B50446E00702D50A4803F061FCA1078D
:109CC00002D5094803F05CFC620702D5074803F09F
:109CD00057FC230704D50648BDE8104003F050BCEC
:109CE00010BD00BF18220020D01F00202423002018
:109CF000841F0020F8B5154803F0D8FA03F0ECFAF9
:109D000008B102F00BFD124A137873B11148124AE0
:109D1000124F0023121AD20819461E469A4207D142
:109D2000FF20BDE8F840FFF793BFFFF749FEEBE7E0
:109D300010F833400C44102C00EBC305DBBFC919ED
:109D400069606E60E1B20133E8E700BFAD9E0100DB
:109D5000302300209C1E0020B41E0020741F002011
:109D600010B50446E00703D50B490C48FFF7EAFE9F
:109D7000A10703D50A490B48FFF7E4FE620703D5A4
:109D800009490A48FFF7DEFE230703D508490948B9
:109D9000FFF7D8FE012010BD182200207C1B0020F8
:109DA000D01F0020701B0020242300208C1B0020CB
:109DB000841F0020641B002038B51446032819D8DE
:109DC000DFE800F0141A02110D484FF48072651894
:109DD000AA42BCBF521A94B20144224618460BF064
:109DE000E2FB204638BD07481022F0E706484FF452
:109DF0000C72ECE70024F4E704484022E7E700BFD8
:109E000024220020741F0020E81F0020901F002043
:109E100070B505460E461446032818D8DFE800F052
:109E20001C1902140E484FF48072A1198A4201DAFB
:109E3000921B94B22246194630440BF0B4FB0DB984
:109E4000FFF7C2FD204670BD06481022EDE7002452
:109E5000F8E705484022E8E704484FF40C72E4E7CD
:109E600024220020741F0020901F0020E81F0020E3
:109E700008B540F6F8731B685A1C08BF0A4B4FF030
:109E8000805208BF1B6811691269581C04BF302337
:109E90004B43B3FBF2F3581EFFF794FD981EBDE849
:109EA0000840FFF78FBD00BF1410001008B50378FD
:109EB00013B1052B0CD008BD43681BB9164B01220A
:109EC0001A70F8E70B2BF6D1BDE80840FFF7D0BFBA
:109ED0004368002BEFD1FFF795FE0028EBD1FFF789
:109EE000A5FE037A23B1012B0ED0FFF7E5FDF2E7C3
:109EF000D0E9001003F03CFB0028F6D0072808D179
:109F0000BDE8084003F086BBD0E9001003F02CFB4D
:109F1000F2E70828DFD1CEE73023002010B590B05B
:109F20000023024604468DF801000DF102008DF871
:109F300000300BF038FBA01C6946C0B200F07CFC7E
:109F400010B010BD00B58FB06B463822FFF734FF5C
:109F50006946C0B2FFF7E2FF0FB05DF804FB07B53A
:109F600002A901F8010D012000F066FC03B05DF8C4
:109F700004FB10B51C4613462246FFF749FFA042DA
:109F800034BF04200020BDE81040FFF7E8BF000008
:109F9000F0B5203887B00C4615461F2800F2128114
:109FA000DFE810F0200039004D005B0067006C0016
:109FB00010018300100110011001100110011001A7
:109FC0001001100110018B00AA00BD00C600CF00D7
:109FD0001001EF0010011001100110011001F90033
:109FE0000001070119B10220FFF7B9FF3FE0764BEE
:109FF00001AA03F11006154618685968144603C4EF
:10A000000833B3422246F7D11B8823802946122009
:10A01000FFF784FF2BE00329E5D15378107892787D
:10A020008DF801308DF800200099FFF7DFFC002348
:10A030008DF804008DF8053001A90220E8E7012918
:10A04000D1D1117801AB022249002046FFF7B4FEBE
:10A05000C0B20228C7D101A9DAE70229C3D15378D7
:10A06000117801EB032189B20020FFF76BFF07B0E5
:10A07000F0BD0129B7D111782046F6E70129B2D108
:10A080001578524B524A9B1ADB080020C1B28B4212
:10A09000A9D902EBC10412F83110A94200F1010064
:10A0A000F4D1636859681878B2E702299BD15378D4
:10A0B000117801EB032189B2DEE7052993D11279EA
:10A0C000EB78297803EB02236A7801EB8101C2EB7C
:10A0D000C202C1EBC1011144AA789BB202EB41015B
:10A0E0008DF804301B0A8DF8053001AA012389B2CE
:10A0F0000020FFF73EFFBAE703297FF474AF117821
:10A100006B78927803EB02239BB28DF804301B0A24
:10A110008DF8053001AA022349000120E9E74B1E12
:10A120001178C1EBC101C90089B2DBB20132DFE7AE
:10A130004B1E1178C1EBC101C90089B2DBB20132FB
:10A14000EBE71778214B4A1E21495B1AD2B2DB0894
:10A150000024E0B29842BFF446AF01EBC00611F80C
:10A160003000B84204F10104F3D1736819789142C8
:10A1700005D1691C58680BF016FA002034E704205A
:10A1800032E74B1E1178C1EBC101C90089B2DBB2C5
:10A1900001320220ADE701297FF425AF1078FFF7E7
:10A1A00057FDEAE701297FF41EAF1078FFF7D8FDCD
:10A1B000E3E701297FF417AF14782046FFF778FD15
:10A1C0002046ECE701200FE7EC560200CC1E0020F1
:10A1D000B41E00203CDF70473DDF70473EDF704714
:10A1E00007B5002001A9FFF7F9FF0198C0F340006F
:10A1F00003B05DF804FB07B5024601A90020FFF794
:10A20000EDFF019B72B143F002034FF0FF310020DC
:10A210000193FFF7E1FF01990020FFF7DBFF03B097
:10A220005DF804FB23F00203EFE700002DE9F041A5
:10A23000084E094CA41B07468846A4080025A542E1
:10A2400001DBBDE8F08156F8253041463846984795
:10A250000135F4E78C1E0020981E002010B5094A35
:10A26000094910780B6818B9084C24689C4207D03B
:10A270000133142BA8BF00230B6008B10023137017
:10A2800010BD00BF382300203C23002034230020D1
:10A2900037B56C4684E803000E4D0F4A2B6894E8EE
:10A2A000030002EBC30282E803005A1C142192FB54
:10A2B000F1F301FB1323094A2B601078084910B110
:10A2C0000B6003B030BD09688B4204BF01231370DB
:10A2D000F7E700BF34230020CC32002038230020D1
:10A2E0003C230020064B1B783BB9064B1868064BF5
:10A2F0001B68C31A5842584170470020704700BF7E
:10A3000038230020342300203C23002008B5FFF729
:10A31000E9FF28B9034B04481B6800EBC30008BDE4
:10A320000020FCE73C230020CC32002010B5FFF7D2
:10A33000D9FF00B110BDFFF7E9FF0446FFF78EFF1C
:10A3400061682078FFF772FFF1E7000073B50446FB
:10A35000631E0D46C8B2072B0AD8DFE803F02E397A
:10A36000090409091E3E431E58425841FFF743FFA6
:10A370002946204605F078FA002C3AD0052C2FD13A
:10A38000022D2FD18DF80040019502AB13E9030097
:10A3900002B0BDE87040FFF77BBF0028164E13BF28
:10A3A0000123002301200020337000F069FC307885
:10A3B00080F00100FFF7C2F9DAE70028D8D10E4B90
:10A3C0001B7813B104F0AAFFD2E704F0BFFDCFE77A
:10A3D0000028CDD1FFF7EEFACAE7084B1870C7E79F
:10A3E000042CCFD12946204602B0BDE87040FFF7CB
:10A3F0001DBF02B070BD00BFC8320020081F002082
:10A40000FFF7A4BF054B5B685A78187800EB022071
:10A4100080B2002808BF0F20704700BF9C1E00209C
:10A42000054BDB685A78187800EB022080B20028D0
:10A4300008BF4FF4167070479C1E0020054B5B69E7
:10A440005A78187800EB022080B2002808BF052057
:10A45000704700BF9C1E0020034B1888034B1B88CD
:10A46000C31A5842584170472A2500202825002049
:10A47000064B5A79022A07D1587810B1987880F0A3
:10A48000010000F0010070470020FAE7C22300201D
:10A49000014B1878704700BF6C33002000B58BB0BB
:10A4A00000231122CDE9063308931223CDE90423BA
:10A4B0000B4B0C4A09930C4B00934023CDE902232C
:10A4C00001930A4A0623694604A803F0D1FD08B1A6
:10A4D00002F024F9064B01225A710BB05DF804FB1F
:10A4E00000E0D701C82300208223002085A50100B9
:10A4F000C223002010B5022808BF074B044614BF32
:10A50000002119790820FFF77BFF21460720BDE8CD
:10A510001040FFF775BF00BFC223002008B5FFF74A
:10A520009BFF38B9044A054B11885B5C0B4401332F
:10A53000DBB2138008BD00BF28250020282400209E
:10A54000F8B50E4B0E491B88CD5CEA18FF2A07466A
:10A5500010DDDC43E4B22E1BF6B224B101332246F7
:10A5600019440BF020F80649324638190BF01BF855
:10A570002846F8BD01332A461944F7E7282500206C
:10A58000282400202DE9F043037893B0042B0BD846
:10A59000DFE803F003A09B0A0300504E504F0DF17B
:10A5A000070003F0D3FD10B113B0BDE8F08332789B
:10A5B0009DF80730BB54002A63D11A0608D57E3BAC
:10A5C000DBB2484A022B1370E9D001233370E6E76F
:10A5D0001F2B04D9444A03F01F031370DFE70F2B2E
:10A5E000DDD9424D03F0010903F00401C3F38002F9
:10A5F00003F00808C3F3C0046B79012B02D06B7819
:10A60000934209D06A70002937D0AB78002B14BF71
:10A6100003200220FFF76EFF6B79012B02D02B790C
:10A62000A34209D02C71B8F1000F28D0FFF720FF0A
:10A63000C1B20820FFF7E4FE6B79012B04BF0223AF
:10A640006B71B9F1000F01D0FFF768FFFFF704FF4E
:10A65000044678B90DF108084046FFF771FF8146BE
:10A66000E3B2994506D918F8040003F08DFD0134D2
:10A670000028F5D00123EB7091E70120CAE740469E
:10A68000D6E7184C01322178D2B28A42327086D392
:10A690004A1E3070D2B2034690420DDB7A1812F88F
:10A6A000012C9A420DD10439114A7878C9B2FFF7CA
:10A6B0006FFC0023237072E73D5C2B44DBB201305A
:10A6C000EAE70520FFF74BFCF3E703F07DFDFFF71A
:10A6D000E5FE69E703F02AFD66E700BF802300205E
:10A6E00040230020812300206C330020C22300205F
:10A6F000432300202DE9F84F1C4FDFF878B03C8849
:10A7000004F1010A0AEB0006B6B2054688465FFA74
:10A7100086F9BBF800309C4201D2B3421ED99C425C
:10A7200003D9FF2E01D94B4518D91148B6F5807FC2
:10A73000055516D9E443E4B22D1BEDB224B12246EF
:10A74000414650440AF02FFF09482A4608EB04010D
:10A750000AF029FFA7F80090BDE8F88FFFF7DEFEAA
:10A76000D7E72A4641465044F2E700BF2A25002099
:10A77000282400202825002010B50C463D2C90B040
:10A7800011461DD804F140038DF8010022460DF159
:10A7900002008DF800300AF006FF0020A31C0146DD
:10A7A0001DF80120013102448B42D0B2F8DC10A91F
:10A7B0000B44E01C6946C0B203F8402CFFF79AFF37
:10A7C00010B010BD024A00231380024A1380704764
:10A7D0002A2500202825002010B5FFF7F3FF03F0FD
:10A7E000F3FC4FF0A04304220024C3F84427064B97
:10A7F00020465C719C705C70FFF77CFE214608204F
:10A80000BDE81040FFF7FCBDC2230020094B5A7978
:10A8100032B1DA780AB9FFF7DFBF0022DA70704789
:10A820004FF0A043D3F810359B0301D5FFF736BE98
:10A83000704700BFC223002010B53E2890B00446E8
:10A840001BD8A0F1800302460DF101008DF8003005
:10A850000AF0A9FE0020631C01461DF80120013109
:10A8600002448B42D0B2F8DC10A90B44A01C69460C
:10A87000C0B203F8402CFFF73DFF10B010BD000040
:10A8800008B50B4A0B4801210AF0CEFD08B101F0D2
:10A8900045FF4FF0A0430422C3F84427D3F81035F6
:10A8A0009B0303D5BDE80840FFF7F8BD08BD00BF16
:10A8B0000DA801000057020008B500224FF4006106
:10A8C00004480AF0C3FD18B1BDE8084001F026BFF6
:10A8D00008BD00BF0824002008B5FFF77DFF4FF03A
:10A8E000A043024AC3F8442708BD00BF0400020089
:10A8F000084A5379022B0BD153784BB1937883F0EC
:10A900000103002B14BF032002209370FFF7F2BD58
:10A91000704700BFC2230020014B1878704700BF6A
:10A9200090330020034B18884FF6FF73C01A18BFEE
:10A9300001207047D41B0020030670B504460E4664
:10A9400015460BD418B9911C1A20FEF7F5FF2A46BC
:10A9500031462046BDE8704004F0BEBE70BD000028
:10A9600010B5094A094910780B6818B9084C2468D1
:10A970009C4207D00133052BA8BF00230B6008B110
:10A980000023137010BD00BF582500205C25002057
:10A99000542500200C490D4A0B6842F8230001336E
:10A9A000052293FBF2F202EB82029B1A084A0B602B
:10A9B0001078084908B10B60704709688B4204BFE2
:10A9C00001231370704700BF54250020703300200E
:10A9D000582500205C250020064B1B783BB9064B10
:10A9E0001868064B1B68C31A58425841704700202C
:10A9F000704700BF58250020542500205C2500200A
:10AA000008B5FFF7E9FF28B9034B04481B6800EBC2
:10AA1000830008BD0020FCE75C2500207033002087
:10AA2000F8B54F4A1378174613B1013B1370F8BDC0
:10AA30004C4A13781646002BF7D14B4C23689BB930
:10AA4000FFF7CAFF60B1494C2278002AEFD048488E
:10AA50000AF040FD08B101F061FE00232370E6E733
:10AA6000FFF7CEFF03682360FEF7D5FD0028DED098
:10AA700023681D78752D54D020D8022D38D015D8D4
:10AA8000002D62D0012DD2D158785A1C00F120033C
:10AA9000DBB2072B22600ED800F0070005FA00F0A9
:10AAA000C0B201F0B7FA01F0E7FA1EE0042DBED300
:10AAB000732D2ED8284600F0A4FA16E0782D39D050
:10AAC00008D8762D31D0772DB1D12A4B187801F0E6
:10AAD00095FAE8E7802D30D0A9D3A5F184036F2B38
:10AAE000A5D805F07F0000F05EFB2368013313E07A
:10AAF00058785A1C00F12003DBB2072B2260F2D8F1
:10AB0000012300F0070003FA00F0C0B201F08AFA56
:10AB1000C9E75A783A7002332360174B1B783370B9
:10AB200085E7154A59781170F5E701F051FA114B94
:10AB30001870DAE701F068FAB5E7FFF761FF03681C
:10AB400023600E4B01221A70E7E7FFF709FF0B4B5A
:10AB500025601D70084B05221A70064B1D70DCE73E
:10AB600050250020512500202C25002062250020A2
:10AB70003025002061250020B81B00206025002022
:10AB8000034A00231360034A1360034A137070479B
:10AB9000542500205C2500205825002008B5FFF72B
:10ABA000EFFF054A00231360044A1370044A137030
:10ABB000044B05221A7008BD2C25002060250020BA
:10ABC00050250020B81B002010B50E4B1B78024604
:10ABD00043B1FFF715FF0368934211D1BDE8104060
:10ABE000FFF7DCBF084CFFF7D5FE227842B90821F9
:10ABF00006480AF02BFC08B101F090FD01232370F8
:10AC000010BD00BF602500206225002030250020F7
:10AC100008B5054A054801210AF006FC18B1BDE84F
:10AC2000084001F07BBD08BD21AA010004570200C5
:10AC30000A280CD1064B1B784BB1064A136833B176
:10AC4000013B13601BB902210920FFF7D9BB7047F4
:10AC5000B91B00206425002010B5074B1B784BB1B1
:10AC6000064C22681AB903210920FFF7C9FBFFF738
:10AC7000E5FB206010BD00BFB91B0020642500204B
:10AC800010B50B4B1A6804460AB100221A60094B32
:10AC90001C7044B1FFF7E0FF84F001010920BDE81A
:10ACA0001040FFF7ADBB03210920FFF7A9FBF3E735
:10ACB00064250020B91B0020F0B5054685B01022A0
:10ACC000002168460AF07AFC2B7843BB1C4E1D4CD1
:10ACD0006868A41BA408A1B203F0BEFC08B101F08F
:10ACE0001DFD0022D3B2A34211DA04A901EB4300F7
:10ACF00009E0696830F8107C31F8131023443944B6
:10AD000020F8101CDBB29C42F3D80132EAE70025A0
:10AD1000A54206DB03F072FD0B4B00221A7005B052
:10AD2000F0BD56F82570BB683BB1FA890A2A04D8F1
:10AD30003DF915009847BB89FB810135E8E700BF65
:10AD4000981E00209C1E0020C8250020F8B5234E28
:10AD5000234C0025A41BA4082A46A54223DB002A75
:10AD60003AD0204F3A78D2B91F49204803F0CEFBA1
:10AD700008B101F0D3FC0025AC4222DCA4B221468C
:10AD80001B4803F069FC08B101F0C8FC21461948D2
:10AD900003F062FC08B101F0C1FC01233B70BDE887
:10ADA000F84003F0ADBC56F82510CB890A2B04D827
:10ADB0004B6803B19847012201E00A3BCB81013582
:10ADC000CBE756F82530E8B2196803F0E7FB08B185
:10ADD00001F0A4FC0135CFE7F8BD00BF981E0020AC
:10ADE0009C1E0020C8250020B9AC01000C570200B1
:10ADF00088250020A825002008B5002252210448FB
:10AE00000AF024FB18B1BDE8084001F087BC08BD7A
:10AE10006825002008B5054A054801210AF004FB11
:10AE200018B1BDE8084001F079BC08BD4DAD010086
:10AE300008570200014B1860704700BFCC25002066
:10AE4000024B186808B1036818477047CC250020EA
:10AE5000024B1B680BB15B6818477047CC2500207C
:10AE6000054B1988814205D01880044B1B680BB133
:10AE7000DB681847704700BFD2250020CC25002092
:10AE8000054B1988814205D01880044B1B680BB113
:10AE90001B691847704700BFD0250020CC25002033
:10AEA00000F07AB808B5FEF7A5FCBDE80840FEF74B
:10AEB0007DBA00002DE9F74FFEF7A0FA314F0026CA
:10AEC000E8465FFA86FA5046FEF704FB37F8029F21
:10AED000814583462ED02C4B1A78930701D500F07C
:10AEE0005CF80025012489EA0B0914EA090F1BD03C
:10AEF0001BEA040F14BF012200228DF802208DF8F6
:10AF000000508DF801A0FEF77BFC40F00100ADF889
:10AF1000040098E8030000F04FF898E80300FEF7FB
:10AF2000DDFB3A8862403A800135EDB264000E2DB7
:10AF3000A4B2DAD10136052EC3D14FF6FF73ADF8B6
:10AF4000003000238DF80230FEF75AFC40F001007B
:10AF500002ABADF8040013E903000C4C00F02CF830
:10AF600001F0B0F8FFF76CFF2378834207D0FFF7BA
:10AF700067FF207003B0BDE8F04F01F0A6B803B042
:10AF8000BDE8F08FD42500209E260020D425002087
:10AF900008B5FEF74BFC08BD7047704738B5054D46
:10AFA000044645F001054FF47A40A847013CFAD128
:10AFB00038BD00BF1057020010B586B06C4684E85B
:10AFC0000300BDF80430BDF80020ADF80C2043B1FB
:10AFD00092B24FF6FF739A4203D094E80300FEF753
:10AFE0007DFB0023ADF8163094E8030006AB049017
:10AFF000ADF8141013E9030006B0BDE8104000F0EE
:10B00000A5BD08B5002800F0CD80822813D1FFF738
:10B0100017FF810700F1C680392000F0BDFE01F066
:10B020002BF86420FFF7BAFF392000F05BFFBDE882
:10B03000084001F021B883280ED1FFF701FFC207B5
:10B0400000F1B080532000F0A7FE01F015F8642055
:10B05000FFF7A4FF5320E8E784280ED1FFF7F0FEA6
:10B06000430700F19F80472000F096FE01F004F8AE
:10B070006420FFF793FF4720D7E7021FD2B2A02A30
:10B0800002D800F089FED2E700F12002D2B2072AEE
:10B0900007D800F0070301209840C0B200F09EFFDF
:10B0A000C5E700F15B02D2B2022A0BD8A52807D06F
:10B0B000A6280CBF82208320BDE80840FFF7D0BE41
:10B0C0008120F9E700F15802D2B2162A6AD8A828DE
:10B0D00031D0A92831D0AA2831D0AB2831D0AC2822
:10B0E00031D0AD2831D0AE2831D0AF2831D0B12801
:10B0F00031D0B02831D0B22831D0B32832D0B428E2
:10B1000033D0B52834D0B62835D0B72836D0B828B3
:10B1100037D0B92838D0BA2839D0BB283AD0BC2883
:10B120003BD0BD283CD0BE280CBF70200020BDE81D
:10B130000840FFF7A5BEE220F9E7E920F7E7EA209B
:10B14000F5E7B520F3E7B620F1E7B320EFE7B42049
:10B15000EDE7B720EBE7CC20E9E7CD20E7E740F2C9
:10B160008310E4E74FF4C570E1E74FF4C970DEE700
:10B170004FF4CA70DBE740F22120D8E740F22320E9
:10B18000D5E74FF40970D2E740F22520CFE740F22F
:10B190002620CCE740F22720C9E740F22A20C6E764
:10B1A0006F20C4E708BD08B50346002858D08228A0
:10B1B00012D1FFF745FE810752D5392000F0ECFD92
:10B1C00000F05AFF6420FFF7E9FE392000F08AFE04
:10B1D000BDE8084000F050BF83280DD1FFF730FED6
:10B1E000C2073DD5532000F0D7FD00F045FF642095
:10B1F000FFF7D4FE5320E9E784280DD1FFF720FEA6
:10B2000043072DD5472000F0C7FD00F035FF64202F
:10B21000FFF7C4FE4720D9E7021FD2B2A02AD5D932
:10B2200000F12002D2B2072A07D800F0070301205C
:10B230009840C0B200F0DAFECAE700F15B02D2B279
:10B24000022A04D80020BDE80840FFF709BE5833A1
:10B25000DBB2162B04D80020BDE80840FFF710BE73
:10B2600008BD08B528B100F0B9FEBDE8084000F0FF
:10B2700003BF08BD08B528B100F0B8FEBDE808401E
:10B2800000F0FABE08BD08B500F0D4FE00F094FE50
:10B2900000F0F2FE0020FFF7E3FD0020BDE80840CB
:10B2A000FFF7EEBD08B500F0AFFEBDE80840FFF7C0
:10B2B000EABF2DE9FF41804600F009FF002840F079
:10B2C000888098F80670B8F80420D8F8000002903A
:10B2D00002AB98F80250ADF804003F09002A78D07C
:10B2E00080B24FF6FF71884273D0ADF80C208DF814
:10B2F0000A5093E8030000F0F7FC044600F0F2FC6B
:10B3000000F096FCC4F303330F2B62D8DFE813F090
:10B3100010001000320032007B006100610061000B
:10B3200094006100F800F8005701610062017301A8
:10B33000C4F30723C4F3032613F0F00F18BF36013C
:10B34000E4B25DB126B1304600F064FE00F094FE38
:10B35000204604B0BDE8F041FFF753BE2046FFF79A
:10B3600022FFB6B3304600F05DFE04B0BDE8F04108
:10B3700000F082BEC4F3072303F0F003C4F30326F6
:10B38000202BE0B218BF360168B1012824D09DB34C
:10B390003FB198F80630D907DBD56FF3071388F86B
:10B3A0000630304602E06DB1304627B904B0BDE842
:10B3B000F041FFF756BF012FF8D104B0BDE8F041CE
:10B3C00000F03EBE1FB900F041FE30460CE0012FF8
:10B3D000F9D104B0BDE8F0815DB1052FF9D800F0D6
:10B3E000F7FD30423046E1D004B0BDE8F041FFF750
:10B3F00041BF042FEDD8E8E7002FE6D004B0BDE848
:10B40000F041FFF7D0BEC4F381234BB1012BE0D153
:10B4100085B1C4F3090004B0BDE8F041FFF730BDC9
:10B4200035B1C4F3090004B0BDE8F041FFF718BD21
:10B430002846F8E72846EEE714F4407F2CD1002D8B
:10B44000C7D1C4F34210E2064FEA800304F00F00B4
:10B4500000FA03F644BF0F209840C4F381244CBF88
:10B46000C0432846022C09D00ED8012C40EA060021
:10B470000DD004B0BDE8F04100F0E4BB304304B0AF
:10B48000BDE8F04100F0E6BB00F0DCFB304604B064
:10B49000BDE8F04100F0CEBBC4F30122D3B2FDB150
:10B4A00002F00103002B94D0C4F34210830004F097
:10B4B0000F0000FA03F514F010001CBF0F20984095
:10B4C000C4F3812418BFC043022C0BD010D8012C28
:10B4D00040EA05000FD004B0BDE8F04100F0F2BB37
:10B4E0005B08DFE7284304B0BDE8F04100F0F2BBA1
:10B4F00000F0E8FB284604B0BDE8F04100F0DABBFC
:10B50000E6B2F02E2FD009D8A6F1C0031F2B13D915
:10B51000002D4ED0002F49D030461AE7F22E37D0FA
:10B520002ED3F32EF4D1002D3BD0C4F3042004B06D
:10B53000BDE8F04100F099BBC4F3042006F0100709
:10B5400045B100F097FB17B13601F0B22EE706F0D7
:10B550000F002BE700F098FB17B13601F0B243E77C
:10B5600006F00F0040E74DB1042F3FF632AFC4F3B1
:10B57000042004B0BDE8F04100F092BB052FF4E7D1
:10B58000C4F3042045B104B0BDE8F04100F072BB43
:10B59000C4F30420002DF6D004B0BDE8F04100F063
:10B5A00073BB04B0BDE8F04100F05CBBC4F3042001
:10B5B000E9E70FB1304621E7C4F30420ECE7C4F318
:10B5C0000322E1B24046FEF757FA04B0BDE8F0416D
:10B5D000FFF7FABA14F0FF0F7FF4FBAE002D3FF433
:10B5E000F8AEFFF75FFE3220FFF7D8FC04B0BDE8ED
:10B5F000F041FEF711B9C4F30322E1B2404604B0B2
:10B60000BDE8F041FEF71CB91FB56B4683E80300A7
:10B61000BDF80420BDF80010ADF80C101AB90020D8
:10B6200005B05DF804FBBDF80C104FF6FF729142B7
:10B63000F5D093E8030000F057FB0123C0F3033279
:10B64000934013F4104F1CD113F4406FC0B208D1D3
:10B6500013F00C0FE3D0A4280CD8042808D201283A
:10B6600006D9E7280AD8E02802D20438A028D6D87C
:10B670000120D5E7A0F1E003072BF1E7F028CED1B8
:10B68000F6E7C0F3C020CBE782B002AB03E90300CA
:10B6900002B0704782B002AB03E9030002B070470A
:10B6A00070B5094B094E1C78094D3378A34200D17F
:10B6B00070BD05EBC40355F8340059680134FFF739
:10B6C000E9FF04F00704F0E72926002028260020DF
:10B6D000E8250020024B18685968FFF7DBBF00BF60
:10B6E000E0250020F7B5224B9A7912F0F00F0AD12D
:10B6F0009A7842B11F4A204F1278204E4FF6FF7CB5
:10B700003978914201D103B0F0BD988858B31978C7
:10B710005C788DF804108DF80540BDF8045065453F
:10B7200021D006EBC20595F801E0A6451BD116F81D
:10B7300032408C4217D1A978A9B9A988091A89B2CF
:10B74000C72910D899790A48012262F30711997123
:10B75000AB7962F30713AB71FFF7ABFD03B0BDE844
:10B76000F040FFF79DBF013202F00702C8E700BFBB
:10B77000E02500202926002028260020E82500209A
:10B780002DE9F04FA74E91B0044600680A90B088AA
:10B79000358821786278A778B4F80490ADF80C5019
:10B7A0000AAB96F800E096F801C0B046002800F019
:10B7B0004181ADB24FF6FF7A554500F03B81B57837
:10B7C0000195002D00F03681A9EB000096F806B037
:10B7D00080B2C7280BF0F00500F2D280002D40F0B7
:10B7E00081808DF810E08DF811C0BDF81000504533
:10B7F0003D4619D08DF828108DF829203088BDF8E5
:10B8000028C0844510D17FB9012363F3071B86F854
:10B8100006B0FFF75FFF3046FFF74BFDB379A3712A
:10B82000284611B0BDE8F08FB9F1000F09D1002F03
:10B83000F6D098F8063043F0010388F8063000256A
:10B84000EEE78DF824108DF82520BDF824604FF622
:10B85000FF708642EBD0002FEBD17348734E007817
:10B8600096F800E0DFF8C8C1704514D18DF82920A2
:10B870008DF82A70ADF82C908DF8281093E803000D
:10B8800000F032FAC0F30332C3B2032A1DD8DFE856
:10B8900002F0131321210CEBC00696F801809045AD
:10B8A00006D11CF83080884502D1B678002EB7D179
:10B8B000013000F00700D7E710F4706F01D0002BC3
:10B8C000AED02033DBB2072BAAD92046FFF7F1FC1C
:10B8D000019DA5E710F4706FF3D0A27912F0F00F7C
:10B8E000EFD19DE78DF814E08DF815C0BDF8140078
:10B8F000504515D08DF828108DF829203088BDF8D6
:10B90000285085420CD15FB984F806B02046FFF775
:10B91000D0FC2368336063687360FFF7DBFED7E712
:10B920008DF82A70ADF82C908DF828108DF829200C
:10B9300093E80300FFF768FE002800F00381002F62
:10B9400000F0008198F806301F2B0DD9B8F80020C0
:10B95000ADF8302000228DF83220ADF834908DF80B
:10B9600036300CA8FFF7A5FC2368C8F800306368E0
:10B97000C8F80430FFF7B6FEFFF7ACFE01254FE72D
:10B980009DB98DF829208DF82A70ADF82C908DF88E
:10B99000281093E80300FFF777FE3046FFF789FC95
:10B9A00035607560FFF796FE3AE78DF818E08DF880
:10B9B00019C0BDF81800504511D08DF828108DF829
:10B9C00029203088BDF82850854208D13FB984F835
:10B9D00006B02046FFF76DFC3760776078E78DF89A
:10B9E0002A70ADF82C908DF828108DF8292093E856
:10B9F0000300FFF709FE002800F0A480002F00F0EC
:10BA0000A18098F806301F2BAED9B8F80020ADF809
:10BA1000382000228DF83A20ADF83C908DF83E3069
:10BA20000EA89FE7E02500202926002028260020D8
:10BA3000E8250020002875D08DF81CE08DF81DC089
:10BA4000BDF81C504FF6FF76B5426BD098F8025007
:10BA5000002D67D1A9EB000080B2C72851D83D4620
:10BA6000002F6FD08DF820E08DF821C0BDF82000A8
:10BA7000B0422DD08DF828108DF82920B8F800009C
:10BA8000BDF82860864223D198F80630DA0718D42A
:10BA900013F0F00F15D003F0F002F02A1CBFC3F32F
:10BAA00003120132A3711CBF62F30713A371204676
:10BAB000FFF7FFFB2368C8F800306368C8F804305C
:10BAC00070E72368C8F800306368C8F80430A7E658
:10BAD0008DF82A70ADF82C908DF828108DF829205B
:10BAE00093E80300FFF790FD00287FF43DAF98F83E
:10BAF0000630204643F0010388F80630FFF7D9FBF3
:10BB00008EE68DF82A70ADF82C908DF828108DF8FF
:10BB1000292093E80300FFF7B7FDC8F80050C8F8E4
:10BB200004503FE777B18DF82A70ADF82C908DF86E
:10BB300028108DF8292093E80300FFF765FD002801
:10BB40007FF412AF2046FFF7B4FB17E7F0B587B0DC
:10BB50006C4684E803002046FFF712FE2D4E2E4D62
:10BB6000074688B1BDF80430BDF80020ADF80820C4
:10BB700043B192B24FF6FF739A4203D094E80300A8
:10BB8000FFF788FD254C40E094E8030004AB83E810
:10BB90000300BDF80420BDF81010ADF80C10002A09
:10BBA000F0D089B24FF6FF729142EBD03478297809
:10BBB000621C02F007028A420BD0184F327003CB8E
:10BBC00007EBC40C47F83400CCF80410FFF768FD0D
:10BBD000D8E7FFF767FB124B37702F701F605F606D
:10BBE00007B0F0BD04EBC000FFF7CAFD0028F7D096
:10BBF0002B7804EBC30254F833005168FFF74AFD79
:10BC00002B78013303F007032B70287833788342B5
:10BC1000E8D1E5E72826002029260020E825002095
:10BC2000E0250020014B186000F04EBA7826002075
:10BC300070470000024A13681843106000F043BACE
:10BC40002C260020024A13681840106000F03BBA0E
:10BC50002C260020024A13685840106000F033BAC6
:10BC60002C2600200020FFF7DDBF012303FA00F09F
:10BC7000FFF7D8BF012303FA00F0024B1B681843FB
:10BC8000FFF7D0BF78260020012303FA00F0034B12
:10BC90001B6823EA0000FFF7C5BF00BF782600201D
:10BCA000012303FA00F0024B1B685840FFF7BABFAC
:10BCB00078260020024B1B681843FFF7B3BF00BF74
:10BCC00078260020024B1B681840FFF7ABBF00BF6F
:10BCD00078260020024B1B685840FFF7A3BF00BF27
:10BCE00078260020704700002DE9FF416B4683E86D
:10BCF0000300BDF80430002B42D09DF800609DF891
:10BD000001508DF808608DF80950BDF808204FF6F5
:10BD1000FF739A4234D09DF802305BB31B4B1C4A30
:10BD20001B6812688DF80C608DF80D5043EA02080C
:10BD30001F2728FA07F3DB07FCB213D417F1FF37EC
:10BD4000F7D20024134A0E2303FB05239C558DF8DC
:10BD500000608DF801500099204604B0BDE8F04124
:10BD600000F0B7B90399204600F0B3F980B201287A
:10BD7000E4D0E7E7074A0E2303FB05239C5DE6E7D3
:10BD80004FF0000004B0BDE8F08100BF782600202D
:10BD90002C260020302600202DE9F0474B4B1B7845
:10BDA0008BB14B4B1B7873B1C2081A2A09D8494B87
:10BDB0001B68134400F00702012090405A7810439A
:10BDC0005870BDE8F087444DDFF8088195F90070A0
:10BDD000DFF80CC177B3414ED8F8009096F90030E7
:10BDE0009CF90020B6461C464FF0FF31062609EBB1
:10BDF000040A9AF802A05045E3D0B1F1FF3F03D105
:10BE0000BAF1000F08BF214604F1010A9AFBF6F4CB
:10BE100006FB14A464B29442E9D1A3420AD14A1C9D
:10BE20001AD10133013F93FBF6F206FB12368EF86E
:10BE300000602F709CF90030D8F800201A440621C9
:10BE40000133907093FBF1F201FB12338CF8003058
:10BE50002B7801332B70B4E74F1C97FBF6F206FBEF
:10BE6000127252B24FF0010E4FF000090626D8F8B8
:10BE7000007007EB020A9AF802A0BAF1000F1FD077
:10BE80000F4487F802A0D8F80070174487F8029092
:10BE90004F1C97FBF6F106FB117149B2571C97FB3B
:10BEA000F6F206FB127252B29442E0D1A3EB0E03FB
:10BEB000063393FBF6F206FB12338CF80030B9E739
:10BEC0000EF1010E5FFA8EFEE8E700BF081F0020AA
:10BED000BA1B0020BC1B00209826002099260020B9
:10BEE0009A2600202DE9F0432D4B1B7893B12D4B62
:10BEF0001B787BB1C2081A2A0AD82B4B1B68134443
:10BF000000F0070001228240587820EA02005870B1
:10BF1000BDE8F083254E96F90030002BF8D0244D73
:10BF2000214F244C2978D7F8008094F900E04FF095
:10BF3000060C08EB010292F80290814527D1013BE3
:10BF400000205BB2907033700BB92B70237094F9A2
:10BF5000003006225E1D96FBF2F002FB106081426B
:10BF6000D6D13E6895F90050053393FBF2F102FB00
:10BF700011314BB2053191FBF2F002FB101131444B
:10BF8000897809B12370C3E7AB42EDD1FAE70131FB
:10BF900091FBFCF20CFB12127245D1B2C9D1B7E78A
:10BFA000081F0020BA1B0020BC1B00209826002080
:10BFB000992600209A2600200448012300210268C7
:10BFC000D15401331C2BFAD1704700BFBC1B002099
:10BFD000014B1878704700BF9C260020024A137856
:10BFE00018431070704700BF9C260020024A137847
:10BFF00023EA0000107070479C260020014B187047
:10C00000704700BF9C260020014B00221A70704729
:10C010009C260020024A137818431070704700BF16
:10C020009D260020024A137823EA00001070704712
:10C030009D260020014B00221A7070479D2600208B
:10C04000014B1870704700BF9B260020014B002257
:10C050001A7070479B260020064B1B6800205A1C54
:10C060001C3312F8011B09B10130C0B29A42F8D159
:10C07000704700BFBC1B002038B50E4C0E4922682B
:10C080000978117021680D480A7800780C4D024338
:10C090000A7095F9002042B1236819780A431A7092
:10C0A000FFF7DAFF08B100232B702068BDE83840A5
:10C0B000FEF7CEBEBC1B00209C2600209D26002043
:10C0C0009B260020704770477047FEF761BF002035
:10C0D000704707B5ADF804100199FDF787FCA0F192
:10C0E000C0021F2A034604D8FDF7ACFC03B05DF87C
:10C0F00004FBBE2809D8A82825D2A42815D80428CE
:10C1000011D2012809D0002307E0E72807D8E0284A
:10C1100009D2BF28F7D14FF460431846E6E7F0286C
:10C12000F1D340F4A0439BB2F7E7A52808D044F22E
:10C13000820244F28300A62B0CBF13460346ECE7B1
:10C1400044F28103E9E730D0A92831D0AA2832D0BF
:10C15000AB2833D0AC2834D0AD2835D0AE2836D07B
:10C16000AF2837D0B12838D0B02839D0B2283AD04B
:10C17000B3283BD0B4283CD0B5283DD0B6283ED01B
:10C18000B7283FD0B82840D0B92841D0BA2842D0EB
:10C19000BB2843D0BC2844D0BD2845D0BE2844F29B
:10C1A000704318BF4FF48843B7E744F2E243B4E763
:10C1B00044F2E943B1E744F2EA43AEE744F2B5435F
:10C1C000ABE744F2B643A8E744F2B343A5E744F231
:10C1D000B443A2E744F2B7439FE744F2CC439CE761
:10C1E00044F2CD4399E744F2835396E744F28A53ED
:10C1F00093E744F2925390E744F294538DE744F26C
:10C2000021638AE744F2236387E744F2246384E7E7
:10C2100044F2256381E744F226637EE744F2276314
:10C220007BE744F22A6378E744F26F4375E72DE930
:10C23000F34106460025EFB23846FDF74BF90024DE
:10C24000804648FA04F2D207E3B21AD58DF80430DA
:10C250008DF8057001990020FFF73BFF83B2B342D0
:10C260000BD0C0F3072313F0C00F03F0E00201D09E
:10C27000A02A06D1C0B2B04203D1012002B0BDE86D
:10C28000F08101340E2CDCD10135052DD3D10020F5
:10C29000F4E710B504462C20FFF7C9FF20B1204673
:10C2A000BDE81040FFF7C3BF10BD000038B5FDF773
:10C2B00097FF60BB164DC92445F0010504E0FDF76A
:10C2C0009DF84FF47A40A847013C14F0FF04F6D1E2
:10C2D0000820FFF7DEFF0F4B18701820FFF7D9FF7B
:10C2E00048B90024FEF7C4F888B984B90420BDE831
:10C2F000384002F02BBE0D20FFF7CBFF0028F0D115
:10C300000B20FFF7C6FF80F00100C4B2EAE738BD9A
:10C3100020570200482B00207047000008B50C4849
:10C32000816801F019FE08B100F0F8F90948816848
:10C3300001F012FE08B100F0F1F90748816801F040
:10C340000BFE18B1BDE8084000F0E8B908BD00BF19
:10C35000E8260020C4260020A026002008B50A48B0
:10C3600001F00EFE08B100F0D9F9084801F008FE0E
:10C3700008B100F0D3F9054801F002FE18B1BDE89C
:10C38000084000F0CBB908BDE8260020C4260020F4
:10C3900038B5C0F346420B4BC0F34621C0F346000C
:10C3A0005D5C995C1C5C084801F07F0101F0F7FDC1
:10C3B0006908064801F0F3FD61080548BDE838400A
:10C3C00001F0EDBD26570200E8260020C42600201B
:10C3D000A026002008B5044B1860FFF7D9FFBDE880
:10C3E0000840FEF739BC00BF6C2700201FB50023B2
:10C3F00000937F234FF0A0428DF801304FF08073FF
:10C40000CDE9012369461E4B1E4A1F48039301F0E4
:10C4100073FD08B100F082F900211B4801F0BFFD57
:10C4200008B100F07BF94FF400030293154A174B53
:10C4300017480393694601F05FFD08B100F06EF9FB
:10C440000021134801F0ABFD08B100F067F94FF48B
:10C45000800302930B4A0F4B0F480393694601F088
:10C460004BFD08B100F05AF900210B4801F097FD8F
:10C4700008B100F053F9FFF751FF05B05DF804FB78
:10C48000A857020019C30100E8260020AC5702009B
:10C49000C4260020B0570200A026002008B5FFF7F0
:10C4A0005DFF4FF0A0430222C3F86027C3F85C276A
:10C4B000C3F8582708BD4FF0A04310F4000F4FF009
:10C4C000807214BFC3F80C25C3F808254FF0A043B1
:10C4D00010F4004F4FF4000214BFC3F80C25C3F84A
:10C4E00008254FF0A04310F0800F4FF4800214BFD6
:10C4F000C3F80C25C3F808257047000010B50446A2
:10C5000008B1064B1868FFF743FF1CB1BDE81040A7
:10C51000FFF704BFBDE81040FFF720BF6C270020E5
:10C520000649074A074B9B1A03DD043BC858D05005
:10C53000FBDC00F013F8FCF783FE00009C590200BE
:10C54000481B0020D41E0020FEE7FEE7FEE7FEE7C2
:10C55000FEE7FEE7FEE7FEE7FEE7FEE7604B614A27
:10C560001B68C3F3423313604FF080430022C3F8CB
:10C570000C21C3F81021C3F838254FF0805203F581
:10C580004043D2F80414C3F82015D2F80814C3F8B5
:10C590002415D2F80C14C3F82815D2F81014C3F8D7
:10C5A0002C15D2F81414C3F83015D2F81814C3F8A7
:10C5B0003415D2F81C14C3F84015D2F82014C3F86F
:10C5C0004415D2F82414C3F84815D2F82814C3F837
:10C5D0004C15D2F82C14C3F85015D2F83014C3F807
:10C5E0005415D2F83414C3F86015D2F83814C3F8CF
:10C5F0006415D2F83C14C3F86815D2F84014C3F897
:10C600006C15D2F84424C3F87025374B1B680A2BED
:10C6100006D1364B1B681BB9354BFB22C3F81825D6
:10C62000344B1B78062B13D1334B1B6819070FD1E2
:10C63000324B1B6803F0F002302A03D003F0E00312
:10C64000402B05D12E4B2F4A1B6803F04F0313607C
:10C650004FF08043D3F80024D20744BF6FF00102AB
:10C66000C3F800244FF01023D3F80022002A03DB84
:10C67000D3F80432002B2FDA234B0122C3F8042510
:10C68000D3F80024002AFBD04FF010221521C2F865
:10C690000012D3F80024002AFBD04FF010231522FB
:10C6A000C3F80422184B1A46D3F800140029FBD013
:10C6B0000021C3F80415D2F80034002BFBD0BFF3DF
:10C6C0004F8F1249124BCA6802F4E0621343CB60E9
:10C6D000BFF34F8F00BFFDE70E4B0F4A1A60704744
:10C6E000440200103C0500403001001034010010ED
:10C6F00000F00040E00F00F0E40F00F0E80F00F061
:10C7000058020010E40E004000E0014000ED00E09F
:10C710000400FA05C01B00200090D0031FB50021C3
:10C72000039001AA44F20100CDE9011100F004F8E0
:10C7300005B05DF804FB000072B6094B1B68DB070F
:10C7400000D500BEBFF34F8F0649074BCA6802F4FD
:10C75000E0621343CB60BFF34F8F00BFFDE700BF24
:10C76000F0ED00E000ED00E00400FA0512F0030334
:10C7700010B511D1094C22604C1CE400A4B2224433
:10C78000074C2260074A1370074A1370074A10804B
:10C79000074A1846118010BD0720FCE778270020C3
:10C7A0007427002070270020802700207C2700208D
:10C7B0007E2700202DE9F3472B4D2B888B42064620
:10C7C0000C4617464BD302A84FF0000800F8018D25
:10C7D00000F088F8254B264A18781178CBB2254905
:10C7E00009888B4238BF0133C0B238BF5FFA83F883
:10C7F00040452ED092F800801378DBB2994286BF74
:10C800000133DBB2002313709DF8070000F08EF8AF
:10C810004FF6FF73984524D0DFF860A0DAF80030B7
:10C820004FEAC80903EB090243F83870A6B19CB17E
:10C83000114B28881B68224608FB0030314608F05F
:10C84000B2FEDAF800304B4400209C8002B0BDE814
:10C85000F0874FF6FF78D7E700209080F6E70920B1
:10C86000F4E70420F2E700BF7C27002080270020A7
:10C87000702700207E2700207427002078270020C2
:10C88000F8B5124C124D264622782B789A4200D1E8
:10C89000F8BD23780F48104A078812680F48DBB2AA
:10C8A00019B202EBC10C006852F83120BCF8041038
:10C8B00003FB070090470A4A23781288DBB29A42AA
:10C8C00086BF0133DBB200233370DDE78027002011
:10C8D000702700207C270020782700207427002064
:10C8E0007E27002070B5EFF3108672B60C4A94686C
:10C8F00001239CB993600B4B0B4DD3F8801029405A
:10C900001160C3F88050D3F8841051604FF0FF32AB
:10C91000C3F88420047006B962B670BD0370FAE7EC
:10C920008433002000E100E0FC06FFBD10B5084B99
:10C930009A685AB150B9EFF3108172B6054A1C6873
:10C9400014605C685460986001B962B610BD00BFA5
:10C950008433002000E100E070B5064E0546002457
:10C9600056F824300BB1284698470134042CF7D1EF
:10C9700070BD00BF902700200B4A0C4B518814203B
:10C9800000FB0131CB6833B90420496810700122E3
:10C99000074801F018B805230649137002238B805D
:10C9A000012200230968F3E7A8270020C027002000
:10C9B000781E00207428002007B500230549009345
:10C9C000054A09680548082300F0CFFF03B05DF869
:10C9D00004FB00BF74280020C0570200781E00200E
:10C9E00007B50023009301460823034A034800F0DB
:10C9F000BCFF03B05DF804FBB8570200781E0020AE
:10CA000013B500230C46009301460423074A084847
:10CA100000F0ABFF38B9074B142202FB04340123AA
:10CA2000237402B010BD0E20FBE700BFB457020014
:10CA3000781E0020C027002037B50A480A4B4268FC
:10CA40009C88196853880325033305709BB2002026
:10CA500000909B0001EB8401044800F086FF03B0C6
:10CA600030BD00BFA827002074280020781E0020B9
:10CA700010B50146044800F054FE1C220446002173
:10CA800008F09CFD204610BD6028002078B10268A7
:10CA9000084B9A420BD14068074B984205D00133AE
:10CAA00098420CBF012003207047002070470320EC
:10CAB000704700BFDEC0ADDEFE011EF1033083B261
:10CAC00040F2FD32934230B50ED909200BE02289A5
:10CAD00065892A441A4492B2B2F5806F08D2088060
:10CAE00062891344638130BD024C20780028EED067
:10CAF0000720F8E7C02700204388033300EB8303B7
:10CB0000994209D382884FF6FF739A4206D0008873
:10CB1000B0FA80F04009704702207047012070474A
:10CB20002DE9F8430223DFF860800B800D4617469D
:10CB300000F5805600F108044FF00109B4420FD20D
:10CB4000236801330CD031462046FFF7D5FF48B1AA
:10CB50000FB187F8009002280BD14FF480632B802F
:10CB6000BDE8F883A368D8F80020934201D9C8F83B
:10CB700000302B886288033313442B80638803338F
:10CB800004EB8304DAE700BFB827002070B5144A2D
:10CB9000142303FB00200B6844680D4604F58056FF
:10CBA0009BB15C88033403EB8404B4420BD223684A
:10CBB000013308D031462046FFF79EFF012809D0F7
:10CBC00005D30228F1D1002003E00834EDE72C6002
:10CBD000012070BD6388033304EB8304E5E700BFE5
:10CBE000C027002037B5436805460C4613B31E4ADC
:10CBF000D1688B421ED3126993421BD813F00300F5
:10CC000018D11A4A29891289914213D129689A6840
:10CC100091420FD1164A5268934201D80A2004E08B
:10CC200002F580529342F9D22080B0FA80F0400998
:10CC300003B030BD0023238023880BB10020F7E729
:10CC4000019301A92088FFF7A1FF10B923880133C0
:10CC5000F1E7019B2A6899689142F2D16B60034B1E
:10CC60001B892B81E4E700BF781E0020A827002045
:10CC7000C02700202DE9F0411C461B4B1B780646BF
:10CC80000F4615465BB362B35CB3DFF86480A388DC
:10CC90000BB10A2019E098F80030C3B1A388013322
:10CCA000A380F4E723681EB19988328891420ED19F
:10CCB0001FB119883A88914209D19B682B6023687B
:10CCC0006B600A4B1B892B810020BDE8F081214657
:10CCD000A088FFF75BFF0028E4D12060DEE7022098
:10CCE000F3E70520F1E700BFA0270020A8270020D8
:10CCF000C027002008B5074B191D5888FFF746FFCD
:10CD000018B1BDE80840FFF797BEBDE80840FFF73F
:10CD100033BE00BFA82700202DE9F04FA74FDFF852
:10CD2000C09289B00646B8463B6823B94946A44834
:10CD300000F031FD3860D8F8005029784B1E052BE3
:10CD400000F20281DFE813F0060066006600F700DB
:10CD5000F700500126B19B4B00225A60012411E0DC
:10CD60002B79032B0AD8DFE803F00226323D01239A
:10CD70002B71FFF721FE002800F0D780914B002295
:10CD80005A600E241422002103A808F017FC41F673
:10CD90001D539C4208BF0024D8F8003004941A7830
:10CDA000023A042A00F2C381DFE812F0A401B001C4
:10CDB000D301DB01E201844B1A78022A4FF0000212
:10CDC00040F0DA811A705868FFF70AFED3E77F490E
:10CDD0007F48002302222B718A800122096800F01B
:10CDE000F2FDC8E7794C00262E712068764DFFF7DA
:10CDF000F7FD784BD4F800C05A8814235343EA183F
:10CE0000EE5451682160A188C2F804C01181022249
:10CE1000A280B0E7B5F814A0AA7DDFF8ACB1142366
:10CE2000AEB1022A06D903FB0AB3EA881989033294
:10CE30000A441A81142303FB0ABAEB88BAF80A20C1
:10CE4000C3F57F43FD331344AAF80A3086E703FB9A
:10CE50000AB318895C6804EB8004062A05D8DFE869
:10CE600002F0274D35431D5967000F24AB7D022B7F
:10CE700007D9142202FB0AB2EB88118903330B4451
:10CE80001381142303FB0ABAEB88BAF80A20C3F50E
:10CE90007F43FD331344AAF80A3073E74E484F49E5
:10CEA00000234360AB690360FFF79CFE002859D064
:10CEB0000223AB75002300930423EA18214644485B
:10CEC00000F053FD002830D00E24CFE72B69002B53
:10CED0000CBF01230323AB750023009305F10C0263
:10CEE000042304F10801EAE70123AB750022EB8873
:10CEF00000929B002A6904F10C01E0E7032914BFAA
:10CF000006230523AB7500230093042305F10802D3
:10CF1000E118D4E70623AB75304B19882E4B5868BF
:10CF2000FFF76EFD04460028A0D109B0BDE8F08FE0
:10CF300041F61D549AE7002E7FF410AF2B79012B98
:10CF400020D003D3022B2FD00F241BE702232B71F9
:10CF5000CDE904660DF10A01EB68039303A8FFF71E
:10CF600041FE08B90A240DE70498BDF80A10838829
:10CF7000EB8003882B81FFF743FD0446002C7FF4F0
:10CF800001AFD2E7DFF85CA003AA53463146A81DE3
:10CF9000FFF770FE044650B9BAF804100498FFF782
:10CFA0002FFD04460A2CE9D141F61D54EAE6082279
:10CFB0003146504608F002FBF4E700BFBC270020D2
:10CFC00060280020A0270020C0270020742800200F
:10CFD000781E0020A8270020842700208028002019
:10CFE000B427002084280020002E7FF4B7AE654BC4
:10CFF000DA7AAAB1DE721A78013A062AA4D801A117
:10D0000051F822F0B7D00100B1D00100C5D0010025
:10D01000CBD0010049CF0100D1D00100E7D0010001
:10D020001A78072AE7D801A151F822F04DD0010063
:10D03000F7CF0100F7CF010069D001007DD00100DA
:10D040009DD001009DD0010065D001001A890132F8
:10D050001A8100225A80DA724B4A1278B2FA82F2AE
:10D0600052099A72012207E0484958688A88408824
:10D07000033202448A8002221A70BCE7424C5A886A
:10D080004249142505FB02420868546850608888AC
:10D09000108102228A800C600622EDE70722EBE76E
:10D0A000394900229A72CA6842B9097C31B15A8062
:10D0B000FFF720FE61E79A7A002AF1D100221A7068
:10D0C0005A805CE0FFF7B8FC57E7FFF755FC54E7E0
:10D0D00006221A702C4A5B88142101FB032358682E
:10D0E000FFF77EFC49E707221A7000225A60FFF71B
:10D0F00063FC42E701228DF80C201A89ADF8182054
:10D100009A88ADF81A20DB68059310E002228DF8AA
:10D110000C201A89ADF818209A88ADF81A20DA6820
:10D1200005929B7D9A1F534253418DF81C3003A8F2
:10D13000FFF712FC002649461548C8F8006000F0C9
:10D1400055FB0121134800F0F9FB00287FF4ECADFA
:10D15000EBE603228DF80C20DA88ADF818201A8946
:10D16000CFE704228DF80C20DB88ADF81830DEE71D
:10D1700005238DF80C30DAE7074B012119705A604E
:10D1800012E700BFA8270020C02700207428002035
:10D190006028002070280020A02700204068FFF7AA
:10D1A000BBBD000008B50121044800F0B1FB18B96F
:10D1B000BDE80840FFF7B0BD08BD00BF70280020E3
:10D1C0002DE9F3419846344B1B7806460D46002B5B
:10D1D00059D0002959D009884FF6FF73994256D08B
:10D1E0006B88002B53D06B689B0752D14AB92F89AB
:10D1F0000DF102013846FFF761FC30B102B0BDE825
:10D20000F08113885788ADF8023001A8FFF730FC91
:10D21000044658B9BDF80230204A142101FB03230B
:10D2200058890338C01B58810820E7E780F8008040
:10D2300000238375BDF8023083826B68036101218E
:10D24000174800F070FBE0602B8823816B88A38077
:10D25000B8F1030F04BF0423A375E78004BF33684C
:10D26000A3610025658101A90E4800F084FA36B15A
:10D270007560E36833600C4BB5721B893381FFF72F
:10D2800091FF0020BAE70220B8E70520B6E70420A6
:10D29000B4E70320B2E700BFA0270020C02700208A
:10D2A000B827002060280020A827002008B5084BD8
:10D2B0001A68042A09D01968064A42F82100012197
:10D2C000184600F030FB002008BD0C20FCE700BF32
:10D2D0007C280020902700202DE9F04F14228BB0ED
:10D2E00000210DEB020008F069F9724A137803F08F
:10D2F000FF01CDE9011243B105A8FFF72DFB4FF067
:10D30000000840460BB0BDE8F08F029B181D00F0EE
:10D3100020FB05460028F2D140F6F8734FF080520A
:10D320001B68654C581C04BF644B1B681269591C70
:10D3300004BF3023534323610022A3F50053604907
:10D34000E360204600F008FB039480460028D8D113
:10D350001C238C225B495C48DFF87C915B4F00F01A
:10D36000ABF9C2464FF0020B4446039BDE685644BD
:10D3700030463146FFF78AFB012849D035D30328D0
:10D3800020D106F580520868013040F087800431D2
:10D390008A42F8D1D9F800203AB902220123C9F80B
:10D3A0000060A9F8042001930AE0142262430220DD
:10D3B000B918B854464A4E60548001340881A4B26A
:10D3C00045F001050AF5805ABAF5005FCDD1BBF1F1
:10D3D000010F98BF0025EDB2022D03D0062D33D0EA
:10D3E000002D3AD14FF00B088BE7142161437A18D6
:10D3F00000207854566001F1100208313A44394453
:10D400003046FFF78DFB45F002050134A4B2D9E7A1
:10D41000019B53B114226243B9180220B85401345D
:10D42000D9F800204A600881A4B200222949C9F82D
:10D4300000603046FFF774FBB9F80420022A14BFDD
:10D44000082204221543BDE7029A0123137005A8A0
:10D4500000235360FFF780FA53E704A8FFF708FBA7
:10D46000C8B10123013D03700A2D09D8DFE805F09A
:10D4700006080608070807080F110F0000230371AC
:10D4800004A9114800F077F9FFF78CFE39E7032370
:10D49000F5E70223F3E74FF0080832E70BF1FF321C
:10D4A0001FFA82FB14226243B9184E600321B9545B
:10D4B000ABE700BFA0270020781E0020141000104A
:10D4C000D4570200D427002060280020C027002065
:10D4D000A8270020782800207428002073B50D4666
:10D4E0000446C8B1C1B10DF10601FFF77BFBA8B13D
:10D4F0000B4BBDF806006668142202FB00300121C8
:10D500000C3000F010FA2E6063680C336B6001235E
:10D51000A372002002B070BD0520FBE70A20F9E7E6
:10D52000C027002013B50446A8B10DF10601FFF78E
:10D5300059FB90B10B4ABDF80630142101FB0323BF
:10D54000DA6862B1A27A52B1DA680020013ADA6090
:10D55000A07202B010BD0520FBE70A20F9E7062003
:10D56000F7E700BFC027002002230022FFF728BEF4
:10D5700018B103230022FFF723BE052070470000E7
:10D5800037B50F4B1B7805469BB1A0B101A8FFF73B
:10D590006FFA90B104230024037004712B68C360F8
:10D5A00001A9084800F0E7F8FFF7FCFD204603B0AA
:10D5B00030BD0220FBE70520F9E70820F7E700BFB0
:10D5C000A02700206028002013B5104B1B780446CC
:10D5D000ABB14FF6FF73984213D001A8FFF748FA9A
:10D5E00088B10523037001230371C48001A9084891
:10D5F00000F0C1F8FFF7D6FD002002B010BD0220F8
:10D60000FBE70420F9E70820F7E700BFA027002088
:10D610006028002007B50E4B1B78A3B101A8FFF7C7
:10D6200027FA90B10623037001A90A4800F0A3F875
:10D63000094B1A780AB10122DA72FFF7B3FD002014
:10D6400003B05DF804FB0220FAE70820F8E700BF0A
:10D65000A027002060280020A827002007B5ADF8EB
:10D66000060002A820F8041D01460DF10600FFF790
:10D6700001FB03B05DF804FB13B502AC134624F8BC
:10D68000020D0A4600202146FFF7F4FA02B010BD51
:10D6900013B502AC134624F8020D0A4620460021B9
:10D6A000FFF7E8FA02B010BD20B119B103680B60B2
:10D6B000002070470520704710B561B1B2FBF3F44C
:10D6C00003FB1424A4B244B9C0E90014846082812D
:10D6D000C381204610BD0E20FCE70920FAE782B086
:10D6E00050E8022FC188B2EB324F4FF0000317BF52
:10D6F00092B241EA014142EA014104E04268B2EBE0
:10D70000324F08BF012340E80212002AE8D18DF809
:10D7100007309DF80730002B0CBF1120002002B00D
:10D72000704737B550E8013F9DB2C48925448489CC
:10D73000A54228BF2D1B0489A54202BFBFF32F8F2E
:10D74000002207E0C5EA030540E80154002CE9D1B6
:10D750004FF001028DF803200193019B9DF80320F7
:10D760000B6002F0FF0322B10B880068184403B07D
:10D7700030BD1846FBE70A884B889A4209D150E829
:10D78000012FC2EA024240E80123002BF7D1012019
:10D7900070470020704737B550E8023F1FFAA3F5E5
:10D7A000C488A54202BFBFF32F8F00220DE0C489B9
:10D7B00025448489A54228BF2D1BC3EA054540E8BE
:10D7C0000254002CE8D14FF001028DF803200193A0
:10D7D000019B9DF803200B6002F0FF0322B14B88F0
:10D7E0000068184403B030BD1846FBE70A884B8830
:10D7F0009A4209D150E8022FC2EA224240E80223AD
:10D80000002BF7D1012070470020704701F01F0264
:10D810004B090121914000EB830000F063B84B09F4
:10D8200010B501F01F040121A14000EB830000F0BE
:10D830004EF8E04000F0010010BD01F01F0301228E
:10D840009A404B0900EB8300D14300F056B84B09D6
:10D8500001F01F0150F82300C84000F0010070479C
:10D860002DE9F0474E1E760980460F460136002509
:10D8700058F8254008EB850AE44394FAA4F4B4FA76
:10D8800084F44FEA4519202C06D10135AE42EFD879
:10D890003C462046BDE8F0874C44A742F5D92146D6
:10D8A0004046FFF7BCFF0028F3D0DAF80040E4431D
:10D8B00094FAA4F4B4FA84F4E5E750E8002F0B4698
:10D8C00040E8003C9CF0000FF7D11046704750E84C
:10D8D000002F42EA010340E8003C9CF0000FF6D123
:10D8E0001046704750E8003F43EA010240E8002C30
:10D8F0009CF0000FF6D11046704750E8003F03EA55
:10D90000010240E8002C9CF0000FF6D11046704751
:10D9100050E8002F02EB010340E8003C9CF0000FB0
:10D92000F6D11046704750E8003F03EB010240E893
:10D93000002C9CF0000FF6D11046704750E8003FD5
:10D94000A3EB010240E8002C9CF0000FF6D110463A
:10D9500070470121FFF7BBBF0B4620B11BB103602D
:10D960001B68114618470E2070472DE9F04108B397
:10D9700002B3D0F800E0BEF1000F1ED0FBB1476843
:10D98000D7F80480B3FBF8F708FB1737BFB942EAB2
:10D99000010C1CF0030F14D1C768B94211D34C1EFF
:10D9A00005691C44AC420CD8DEF80C40A446BDE826
:10D9B000F04160470E20BDE8F0810820FBE7092018
:10D9C000F9E71020F7E7F0B5D8B1D0F800C0BCF106
:10D9D000000F18D0CAB14768D7F800E00EF1FF3742
:10D9E0000F4214D1C768B94211D34C1E05690EFB12
:10D9F0000244AC420BD8DCF81040A446BDE8F0402D
:10DA000060470E20F0BD0820FCE70920FAE710204F
:10DA1000F8E729DF704728DF704770B50568AB6805
:10DA200086B004460E4673B114220021684607F002
:10DA3000C5FDA36805932379019633B1012B0ED060
:10DA4000AB686846984706B070BD01238DF800307A
:10DA500023690293E368039363690493F0E7022365
:10DA60008DF80030E3681B030293F5E70846704722
:10DA700000207047024B187A003018BF0120704711
:10DA800028290020034B187A0122B0FA80F05A743A
:10DA9000400970472829002008B510461A4607F0AB
:10DAA00082FD002008BD000008B5142200210448B2
:10DAB00007F084FD0348FFF712FE002008BD00BFF9
:10DAC000282900201829002010B5094C094B436073
:10DAD0002046FFF73EFF40B907F074F91C2320747D
:10DAE0008C2205490548FFF7E7FD002010BD00BF67
:10DAF00028290020C85702008C280020182900205F
:10DB000070B5244D244E2B7A2C463BB9234924482A
:10DB1000FFF741FE306008B9686070BD02232372D0
:10DB200033681A7972B1012A24D018460321FFF70D
:10DB300074FF00232372636018491948BDE87040E0
:10DB4000FFF754BED3E90520121AB2F5805F28BF53
:10DB50004FF48052D3E903159208012A014438BFDB
:10DB600001222844FFF755FF50B11128DDD10123D0
:10DB70002372D2E7D3E903021044FFF74CFFF3E727
:10DB8000237C002BC9D10146BDE87040022000F083
:10DB900009B800BF28290020402900203C29002086
:10DBA0001829002038B5831E012B45D8234C237A31
:10DBB000002B41D0022B09D1032830D0204B00226A
:10DBC0001B68E2601A793AB1012A22D0637C7BBBE0
:10DBD000BDE83840FFF794BFD3E905128D1AB5F5BB
:10DBE000805F94BF521902F580529A619142EDD143
:10DBF00002284FF0000308BF19462372104B18BFCC
:10DC00000D211868FFF709FF0E490F48FFF7EEFDD9
:10DC1000DCE71A6901321A615B699A42E7E7E36857
:10DC20000133082B01D8E360D0E70023E360DFE78E
:10DC3000BDE8384007F0B6B838BD00BF282900203D
:10DC4000402900203C2900201829002000F0FD0375
:10DC5000012B08D1044B00225A74421E50425041FD
:10DC60001874FFF74DBF70472829002010B5064CE7
:10DC7000201DFFF76EFE28B9637C1BB9BDE810407C
:10DC8000FFF73EBF10BD00BF282900202DE9F3415A
:10DC900080460D460F4801A916461F46FFF741FD75
:10DCA0000446A8B11C22002107F088FC2D0B01239B
:10DCB000237101A9C4F80080A760E560666105488A
:10DCC000FFF759FDFFF7D2FF002002B0BDE8F08159
:10DCD0000420FAE7182900202DE9F74381468846F9
:10DCE000104801A917461E46FFF71BFD0446B0B1B8
:10DCF0001C22002107F062FC00250A9BA36001A9F9
:10DD00002571C4F80090C4E9037866610548FFF7FF
:10DD100032FDFFF7ABFF284603B0BDE8F0830420D7
:10DD2000FAE700BF1829002033DF704741DF704752
:10DD3000064B10B500241C70054B1C60BFF35F8FB1
:10DD40000449054800F068F8204610BD4D29002020
:10DD500050290020F45702004429002008B507F09C
:10DD600031F818B1BDE80840FFF7E0BF20BF40BF61
:10DD700020BF08BD70B5224C054601212046FFF7A3
:10DD80009CFDBFF35F8F264638B9042D0AD01D4B8A
:10DD90001A781AB1BFF35F8F206070BD1A4A1570F0
:10DDA00001221A70194C184D636828787BB9023823
:10DDB000012813D8BFF34F8F1549164BCA6802F4D8
:10DDC000E0621343CB60BFF34F8F00BFFDE71B68DA
:10DDD000984788B1204600F028F8E5E706F0F2FF02
:10DDE00008B1FFF7A1FF4FF080430122C3F80025DF
:10DDF000BFF34F8F20BFFDE7BFF35F8F3060CCE7ED
:10DE0000502900204D2900204C29002044290020C1
:10DE100000ED00E00400FA0501600B6843604A6809
:10DE2000934204BF002343607047436843B10268D4
:10DE300091680B4443605268934204BF00234360DF
:10DE400070470178036AC26821B1C3F80C2500232A
:10DE500043707047C3F80825F9E710B5037D044601
:10DE6000002B3FD183697BB9E278A378934213D129
:10DE70002178236AE26861B1C3F808250123637041
:10DE8000A378053323611BE098472379022BEBD05D
:10DE900010BDC3F80C25F1E71AB92046FFF7D1FFF2
:10DEA000EEE72078236AE168C8B1C3F80815A378C3
:10DEB00013FB02F31B1201210533617023612175ED
:10DEC0002379022BE4D1E36921691868224607F01F
:10DED000BDFA0028DCD0BDE81040FEF71FBCC3F837
:10DEE0000C15E4E7FFF7ADFF00230375C2788378D4
:10DEF0009A1A53431B12C4E770B582610B788D6880
:10DF000003708B6883608B68C3604B6803624B78D7
:10DF100083700446C868E0610E4A002107F084FA65
:10DF2000064648B903464FF0A042032135B92046C2
:10DF3000FFF787FF01232371304670BDE80748BF14
:10DF400003F5E0704FEA550548BF42F82010013351
:10DF5000ECE700BF5BDE010070B5044602230371ED
:10DF6000E1600D46FFF76DFF836886692B4300254E
:10DF7000836005758561FFF770FFA661284670BD57
:10DF800038B5C3690446186807F0A4FA0546204668
:10DF9000FFF757FF0DB901232371284638BD837859
:10DFA0008B4226BFC17000200720704737B5057827
:10DFB000012D04D03BD3022D2BD003B030BD4368DC
:10DFC000244C1978204600F016F990B1224B0190AC
:10DFD0008DF800501B6868469847A168E368A288DE
:10DFE0005B1A9A4211D301221C491D4800F004FF1C
:10DFF000E3E7A268E3689A42EFD002AB164A03F85F
:10E00000080D126818469047E7E7164B01221A7070
:10E01000D3E7C36811491248019301228DF80050DB
:10E0200000F0EAFE0C4B1B6868469847C5E70E49AE
:10E030000E4800F0F2F828B901220B49084800F018
:10E0400085FEBAE702A8032300F8083D024B1B68CF
:10E05000EBE700BF58290020542900207C2900202C
:10E06000C81B0020682900207D2900206C29002081
:10E07000F0B51F46244B89B006461A600C460029AD
:10E0800040D08A882148096800F0A6F8002837D1D6
:10E09000A289A1681E4800F09FF8002830D11D4DCC
:10E0A0000FCD6C460FC495E80F0084E80F0073692C
:10E0B0000693337C184A19488DF81C70003318BF3A
:10E0C00001238DF81430737C002B14BF0E23002322
:10E0D0008DF81530F3680293B368039333680193A6
:10E0E00069467368009300F0C7F848B90C4B187084
:10E0F0003368013304D001220A490B4800F07CFE4A
:10E1000009B0F0BD0720FBE7542900205829002062
:10E110006C29002000580200ADDF0100C41B002064
:10E12000682900207C290020C81B002008B505486C
:10E1300000F084F820B90448BDE8084000F07EB83B
:10E1400008BD00BF582900206C29002070B50A4C7A
:10E1500001460A48267800F060F805464EB10023D3
:10E16000012207490748237000F046FE08B1FEF778
:10E17000D5FA284670BD00BF682900205829002024
:10E180007C290020C81B002010B501460B4800F078
:10E1900032F8044678B90A4800F022FE58B9094915
:10E1A000064800F03AF830B9012206490448BDE8B3
:10E1B000104000F0CBBD204610BD00BF6C290020F0
:10E1C000C81B00207D29002008B5024800F056FD3C
:10E1D000002008BDC81B002049B152B1531E1A408F
:10E1E00007D1826001608380C260104670470E20B4
:10E1F00070470920704710B58468C2688388121B75
:10E20000934208D3C26813400268D154C3680133F3
:10E21000C360002010BD0420FCE78268C3689A42F6
:10E220000AD08268838813400268D35C0B708368CD
:10E23000013383600020704705207047C368836006
:10E24000002070471FB503788DF8003043680193B4
:10E2500083688DF80830C3680393054A054B684608
:10E2600053F8213052F82110984705B05DF804FBAF
:10E270008029002084290020F0B506460F4B16F8AF
:10E28000047B43F827200E4B94460A6943F8272065
:10E290000C460FCC89B06D460FC594E80F00BCF159
:10E2A000000F85E80F00074A049708BF002269465F
:10E2B000304600F023FC09B0F0BD00BF84290020E7
:10E2C0008029002045E2010007B5154B1A687AB194
:10E2D00000221A601B680093009B4FF080430122CC
:10E2E000C3F808230F4B587910B95A711B68984727
:10E2F0000D4B1A6882B100221A601B680193019BC2
:10E300004FF080430222C3F80823064B1B6801200C
:10E3100003B05DF804EB184703B05DF804FB00BFE1
:10E32000000100408829002004010040014B1B68C7
:10E33000184700BF902900200D4B984237B50D4675
:10E3400010D102A8002300F8013DFEF7CBFA094BDB
:10E350001C7914B901221D601A719DF80700FEF79F
:10E36000E5FA14B9002003B030BD1120FBE700BF6F
:10E370000020004090290020034B984201BF034B2E
:10E3800000221A601A717047002000409029002076
:10E3900000F1804000F5E040002382B00360036894
:10E3A0000193019B02B07047F0B5514B514C1B6873
:10E3B00085B0DBB14FF4827094F82E20FFF7E8FFB0
:10E3C00012B194F82F30A3B1636802932389ADF89A
:10E3D0000C30E36800218DF80410002B44D1237425
:10E3E000236801A89847002384F82F3094F82E3032
:10E3F00003B3414B1B68EBB14FF48070FFF7C8FFCC
:10E4000094F82D20638B91B28B4238D95B1A218905
:10E410009BB26383CB1A616801EB4301374BC3F8AE
:10E420002C16C3F830264FF48270FFF7B1FF344B3F
:10E4300001221A60334B1B685BB14FF48870FFF701
:10E44000A7FF002304A82374022300F80C3D2368CF
:10E4500098472D4B1B6813B34FF48A70FFF798FF52
:10E460000023237405B0F0BD208B6083636020819E
:10E47000E160002AB4D1214B01221A60B0E7D2D169
:10E48000E368012184F82F103BB1002161831B490F
:10E49000C1F82C36C1F83026C5E76383C3E7666947
:10E4A0004FF000470125002EDCD0B6FA86F227FA9D
:10E4B00002F34632920026EA030602F1804303F596
:10E4C000E0431B68002BEED01046FFF761FFA2F57A
:10E4D0008C72D30882F00402C2F380028DF80830F7
:10E4E0008DF804508DF80920236801A89847DAE7D1
:10E4F0000471004098290020007100400070004025
:10E5000004700040107100401471004038B5204A7A
:10E5100092F82C300546002B37D111601D49007848
:10E52000C1F8F0056878C1F8F405E878137482F84A
:10E530002D30536182F82F3001246FF0004382F8B0
:10E540002E0082F82C404FF48270C1F80833FFF798
:10E550001FFF4FF48070FFF71BFF4FF48A70FFF727
:10E5600017FFAB780C485B01DBB280F807338023E0
:10E5700003600223C1F8043392F82E300BB1C1F8C6
:10E580000443C1F80045002038BD0820FCE700BF67
:10E59000982900200070004000E100E010B52C4BED
:10E5A0001A7C02F0FF04002A4FD10A79012A9CBF8D
:10E5B000284AC2F8004500F10C0403EB440212792A
:10E5C00022B993F82D20013283F82D2003EB440368
:10E5D000CA791A710A7A5A714B788A781B01120229
:10E5E00002F4E06203F0300313430A7802F00302FE
:10E5F0001343CA78120302F4805213430A791204B7
:10E6000002F4E02213434A79120502F48012134304
:10E610008A79120602F0807213430E4A02EB00144C
:10E62000000100F18040C4F8183500F5E040CB79D6
:10E630000C7AC0F81445C0F810350B79012B02D8BC
:10E640000123C2F80035002000E0112010BD00BFFA
:10E65000982900200070004070B5264A264B0546D8
:10E660001220C2F808031C7C022C03D1C2F8040358
:10E67000112070BD187C01281DD1D86818B1022363
:10E68000C2F80433F4E7DD60198393F82E3063B9E0
:10E690001A4A1368002BFCD04FF48070FFF778FE05
:10E6A000144BC3F82C56C3F83016124B0222C3F891
:10E6B00004230020DDE70220C2F8040393F82E4073
:10E6C0005D60012600201E74D86019813CB1598319
:10E6D00093F82D30C2F82C56C2F83036C9E7C2F88C
:10E6E0002C564FF48070C2F83016FFF751FE2046CA
:10E6F0001660BEE7007000409829002000710040BD
:10E70000084A137CDBB2012B09D192F82E0018B114
:10E71000054A002013607047044A136070470820C0
:10E72000704700BF9829002000700040047000402E
:10E73000F0B51B4F8BB207EB001443EA0243C4F859
:10E740001C35184B40005C6900F1010C4FF000468D
:10E7500011F5006F26FA0CF64FF0800505FA00F56A
:10E760000BBFB44334435C615C610CBFC7F8085312
:10E77000C7F8045340244FF000455969844025FAF6
:10E7800000F040F2FF75AA42054A0BBF81430143E6
:10E79000596159610CBFC2F80843C2F80443F0BD87
:10E7A000007000409829002010B5124B1A7CFAB96D
:10E7B00000F10C0103EB4102127922B193F82D20F4
:10E7C000013A83F82D2003EB410300241C715C7196
:10E7D000030103F1804303F5E04340F2FF72C3F805
:10E7E00014450549C3F81045FFF7A2FF204610BDA8
:10E7F0001120FCE79829002000F8FFFF38B5134BE3
:10E800006FF00042C3F80823114A8021C2F880103B
:10E81000104A01211160104942F21072086808B9CB
:10E82000013AFBD10D4D0024C3F800452C7405EBD3
:10E8300044031B7F13B1E0B2FFF7B6FF0134082C8D
:10E84000F5D1002385F82C3038BD00BF00700040A2
:10E8500000E100E008700040147100409829002099
:10E860000A4A13787BB90121117009490278C1F86D
:10E870000C2542684FF47A70D203B2FBF0F21846CE
:10E88000C1F8042570470820704700BFC92900203F
:10E8900000000140034B01221A60034B02221A7050
:10E8A000704700BF00000140C929002010B5074B88
:10E8B0000748084C19780023DAB2914200D810BDFD
:10E8C00003F5C072013340F82240F5E7C829002063
:10E8D000000001403546526E37B5054602A80024B7
:10E8E00000F8014DFDF7FEFF0B4B1A78072A11D8EF
:10E8F000511C197009492A70D1F808050123934069
:10E900000343C1F808359DF80700FEF70FF82046CD
:10E9100003B030BD0424F6E7C82900200000014000
:10E920000023435082B043580193019B02B07047CB
:10E930000A4610B54FF48E71FFF7F2FF136A916823
:10E94000C95C136A01331362C0F81C1510BD08B509
:10E9500002464FF492710068FFF7E2FF4FF48471B2
:10E960001068FFF7DDFF136801221A6008BD10B5BB
:10E970008B690A464FF4847123B9FFF7D1FFD0F8B1
:10E98000183510BDFFF7CCFF536AD168D0F81805D1
:10E99000C854536A01335362F3E700001FB50123E3
:10E9A0008DF80030044BCDE90110D3E90012684620
:10E9B000904705B05DF804FBCC29002030B54D4AE6
:10E9C000D2F8043313F4007F85B015464FD0D2F847
:10E9D0002431002B4BD04FF492711046FFF7A0FF6B
:10E9E0004FF40173C2F80833434B93F8291009B967
:10E9F000012151603F4902228DF80020D1F8802486
:10EA0000C1F8802403929A690292DA680192002286
:10EA1000C3E906226846D3E9001290473548D0F88A
:10EA20001C315BB134490A6A4B699A420A464CD29E
:10EA300091F82830002B48D1FFF77AFF2D4AD2F801
:10EA4000443193B14FF4A2711046FFF769FF2A4B8E
:10EA500093F8291009B1012111609A692AB10022A5
:10EA60009A61586AD968FFF799FF05B030BDD5F8AB
:10EA700004335B07D2D5D5F80831002BCED01E4C1D
:10EA80001C482146FFF773FF636AA2699A42234636
:10EA9000C4D1E26952B12369E168E3600023606A8E
:10EAA000A261E3616362FFF779FFB7E794F8292079
:10EAB0000AB901226A600F4A4FF40171C2F80813C3
:10EAC00000229A61586AD968EDE74FF48E710948BF
:10EAD000FFF726FF51690029B0D000230291916809
:10EAE0008DF80030019153616846D2E900139847D0
:10EAF000A4E700BF00200040CC2900202DE9F84306
:10EB0000594F067991462C2202FB0672054692F86F
:10EB10002A200C46002A40F0A08054490068FFF7E4
:10EB20000BFC8046002840F09B802268501C0BD0D4
:10EB3000012393404FF0A0420321C2F80835236817
:10EB400003F5E07342F823106368591C1FBF03F5F7
:10EB5000E0734FF0A042002142F823102B68A26915
:10EB6000C3F82425217D637D2A680B43C2F86C35E8
:10EB7000D4E900122B68C3F81425C3F80C15237DC3
:10EB8000012B1FD1A3685A1C1FBF4FF0A04203F5F1
:10EB9000E073002142F82310E268531C0BD00123DC
:10EBA00093404FF0A0420321C2F80835E36803F513
:10EBB000E07342F82310D4E902122B68C3F8082549
:10EBC000C3F810152C237343FA18C2F80490226975
:10EBD000FA50B9F1000F2DD04FF48E712868227FC2
:10EBE000FFF79EFE4FF4A2712868FFF799FE2B688D
:10EBF0001F49C3F804132968090B4BB2002BAEBFA1
:10EC000003F1604301F00F011A4B4FEA4212D2B2F6
:10EC1000AABF03F561435A5483F800232B681B0BEA
:10EC20005AB2012103F01F0301FA03F352091249FA
:10EC300041F822302B680422C3F800252C2303FB63
:10EC400006730022C3E9062283F829205A610122B3
:10EC500083F82A204046BDE8F8834FF00808F9E71A
:10EC60004FF01108F6E700BFCC290020BDE90100F4
:10EC70008000020014ED00E000E100E0F8B5036858
:10EC800004792F4D0022C3F800252C2303FB0453E5
:10EC90005B6883B103682B4AC3F8082303681B0B26
:10ECA0005AB20121520903F01F0301FA03F3203283
:10ECB000254941F8223003684FF0FF3CD3F80C752A
:10ECC000D3F81465D3F80825D3F81015C3F814C584
:10ECD000C3F80CC503686745C3F808C518BF07F536
:10ECE000E077C3F810C51EBF4FF0A0434FF0020CF1
:10ECF00043F827C0771C1FBF4FF0A04306F5E0760E
:10ED0000022743F826704E1C1FBF01F5E0714FF03B
:10ED1000A043022643F82160531C1FBF4FF0A043BD
:10ED200002F5E072022143F822100068FFF724FB8D
:10ED30002C2303FB0454002384F82A306360F8BDBD
:10ED4000CC2900208402020000E100E02DE9F84314
:10ED5000224B07794FF02C0909FB073406466569F9
:10ED60009846002D35D16261A160256284F8285053
:10ED70004FF48E710068FFF7D3FD336801229A606B
:10ED800021463068FFF7D4FD6368A1461BBB356898
:10ED9000226A63699A4211D33368D3F81C21002A8E
:10EDA000FBD00122DA6000202C2303FB078700231D
:10EDB0007B61BDE8F88394F8283043B9D5F81C315D
:10EDC000002BF8D049462846FFF7B2FDE0E70F20B8
:10EDD000EAE71120EDE72846EBE700BFCC29002049
:10EDE0000379044A2C2101FB03235869003018BF22
:10EDF00001207047CC2900202DE9F843384E0579D1
:10EE00002C2303FB056307465C6824B103684FF4B9
:10EE10000170C3F808032C2303FB0563986950B104
:10EE2000D86900283ED024B13B684FF40172C3F882
:10EE30000423112034E09A61D9605862D8612C23F0
:10EE400003FB056393F829301BB910B93846FFF767
:10EE50007EFD4FF02C0909FB05683868D8F80430AE
:10EE6000002B34D14FF4A271FFF75AFDC146386828
:10EE7000D0F82431D0F80821D0F84441B2B90CB907
:10EE8000002BF4D02C2202FB05650022AA611BBBDB
:10EE900024BB95F829103B680122B1B11A6000200B
:10EEA000BDE8F8831961DA610120C8E7002BE9D1D8
:10EEB000002CE7D14946FFF75AFDD8F82430D8F89E
:10EEC00018209A42D3D82346DCE75A60E7E74FF48C
:10EED0000173C0F80433E2E70320E1E70F20DFE726
:10EEE000CC29002033DF70473FDF7047FDF716BCA9
:10EEF00008B5FAF715FD03210520FBF781FA06F0A6
:10EF0000F9FA18B1BDE80840FDF708BC08BD0228B1
:10EF100008B501D1FFF7ECFF012008BD10B504468C
:10EF2000FFF7E6FF54B1FAF7F7FAFBF7D5FCFFF766
:10EF3000D9FF30B1BDE81040FDF7F0BBFAF7D0FAC9
:10EF4000F3E710BD01460420FBF75ABA08B50428C0
:10EF500013D8DFE800F00303080A06000120FFF7DA
:10EF6000F1FF012005E00020F9E70220FFF7EAFFAA
:10EF70000020BDE80840FFF7D1BF08BD08B506F086
:10EF800021FA08B1FDF7CAFBFEF7D2FE08B1FDF782
:10EF9000C5FB0120FFF7A8FFFAF7ACFE0021052012
:10EFA000FBF72EFA00F0C8F9164A14210820FDF7E5
:10EFB000DDFB08B1FDF7B2FB00F0EAF900F004FD5B
:10EFC000114800F0CDFBFBF725FFFAF7C3FBFDF777
:10EFD0006DF901210520FBF713FAFAF795FBFBF712
:10EFE0006BFCFBF709FF094B187800F092F902213E
:10EFF0000520FBF705FAFDF743FCFBF797F9FEF751
:10F00000ADFEF8E7F8290020EDEE0100482B0020C6
:10F010006DDF704774DF704776DF704777DF7047CA
:10F0200078DF70477ADF70477CDF704780DF70479A
:10F030008FDF70471321FFF7EFBFFDF76FBB0000B5
:10F0400013B50388212B2ED010D8112B19D0172BD4
:10F0500033D0102B08D11A4B81881A48198002F03E
:10F06000F9FC08B1FDF75AFB02B010BD562B03D0D6
:10F07000572B20D03B2BF7D113218088FFF7CCFFF3
:10F08000EFE70F4B104C4FF6FF721A8022682AB13F
:10F0900000210846FDF78EFB00232360012108466E
:10F0A000FBF7AEF9E0E702A9002321F8043D8088D0
:10F0B000FFF7BEFFD5E70021F1E700210220EFE7CF
:10F0C000D41B0020182C0020242C00207FB506A97A
:10F0D000082341F8143D4FF6FF72034602A803F0DF
:10F0E0009FFA08B1FDF71AFB019902A803F044FA50
:10F0F00008B1FDF713FB07B05DF804FB00B5B3B032
:10F1000008280AD8DFE800F00E0909050C050C10E4
:10F110002D0003210120FBF773F933B05DF804FBE8
:10F120000421F7E70021F5E732AB0822029243F809
:10F13000BC2D02A912AA04A803F008FA08B1FDF731
:10F14000EDFA0220FFF7C2FF039B0093029A1048DA
:10F1500012AB04A901F0D4F80028DED0FDF7DEFAE6
:10F16000DBE70C4B18884FF6FF739842D5D012A9F5
:10F1700003F006FB0528D0D008B1FDF7CFFA062032
:10F18000FFF7A4FF0DF15901014801F0AAF8E3E7E8
:10F190004C2B0020142C0020032807D14FF0804373
:10F1A000A922C3F820250020FEF7E4BD70477FB5F3
:10F1B00006A9082341F8143D4FF6FF72012302A867
:10F1C00003F02EFA08B1FDF7A9FA019902A803F09D
:10F1D000B3F908B1FDF7A2FA07B05DF804FB00002F
:10F1E00008B5FFF7E4FF0321044800F041FF18B120
:10F1F000BDE80840FDF792BA08BD00BF4C2B0020C7
:10F2000013B5044603F0BFFC204603F0C9FC237885
:10F210000C2B0FD8DFE803F00A0E070E1C0E0E0EA3
:10F22000130E0E0E10000E4BA2881A800221012030
:10F23000FBF7E6F802B010BDFFF7D2FFFAE7237C38
:10F24000DB07F7D5237A072BF4D1FFF7B0FFF1E7FF
:10F2500002A9012301F8043D608803F069F9E9E798
:10F26000142C0020FDF75ABAFDF758BA30B58DB00E
:10F270002C22002101A806F0A1F91A4D282140F600
:10F28000B832CDE905124FF4486044F250620123D0
:10F290000024CDE9070201A928468DF806308DF833
:10F2A00008308DF809308DF804308DF805408DF860
:10F2B0000740CDE9034401F036F821460A4801F041
:10F2C000A5FAAB781BB195F85400FFF7A3FE074BE6
:10F2D0001A884FF6FF739A421EBF054B00221A6030
:10F2E0000DB030BD4C2B002035F00100D41B0020A8
:10F2F000242C002008B9FFF7B9BF704708B5FFF705
:10F30000B5FF03F053FA18B1BDE80840FDF706BA9F
:10F3100008BD08B1FFF7F2BFFFF762BF08B50421CF
:10F32000044800F0A5FE18B1BDE80840FDF7F6B9A5
:10F3300008BD00BF4C2B002013B505F0C7FC08B179
:10F34000FDF7ECF902AC002344F8043D012021460E
:10F3500005F090FD08B1FDF7E1F9204605F0E0FD6C
:10F3600008B1FDF7DBF902B010BD000008B5074B8E
:10F37000024601211888FFF759FE08B1FDF7CEF9C2
:10F3800002210846BDE80840FBF73AB8D41B00202C
:10F390002DE9F041AEB000AF03F06CF808B1FDF715
:10F3A000BDF90522002107F10C0006F007F93B7BAF
:10F3B00043F00103032203F0F10362F306136FF33A
:10F3C000C7133B7307237B731023BB73FB7B134370
:10F3D000FB733B7C07F10C0013433B7403F090F884
:10F3E00008B1FDF79BF9884803F072F808B1FDF702
:10F3F00095F9112385483B7006F0F0F800F10F03F2
:10F4000023F007036E46ADEB030D814B05466C46BA
:10F4100007F10C0C03F1100E18685968624603C21C
:10F42000083373459446F7D17849204606F0CEF864
:10F430005F2304EB050863553D1D2846FFF7E8FDF3
:10F4400041460022AB1807F1B8001B7900EB1310FE
:10F4500003F00F0310F8AC0C487007F1B800034438
:10F46000013213F8AC3C01F8023F032AEAD1002331
:10F4700088F80730204606F0B1F8214682B23846B7
:10F48000FFF7D2FD08B1FDF749F94FF47070B546AA
:10F49000FFF7C6FD08B1FDF741F90822002107F189
:10F4A0000C0006F08BF85B4BFB6007F10C0003F5DA
:10F4B00098133B61FFF7B6FD08B1FDF72FF9002166
:10F4C000554802F01FFA08B1FDF728F9AC220021D7
:10F4D00007F10C0006F072F802233B7306230124A7
:10F4E000FB732C224D4B3B62002107F18400BC735F
:10F4F000BC8306F063F80023282140F6B832C7E940
:10F5000025124FF4486087F8853087F88730C7E9BF
:10F51000233344F2506287F88430414BC7F8B0304F
:10F52000C7E927023F4B404887F8864007F10C01A6
:10F5300087F8884087F88940C7F8B43000F026FD86
:10F5400008B1FDF7EBF8384C0121204600F01BFD17
:10F55000042294F854100120FFF760FD08B1FDF774
:10F56000DDF8324B3248FB6007F10C0102F060FA23
:10F5700008B1FDF7D3F841F20923FB8040F21453A0
:10F5800002243B8140220323002107F10C007B81F0
:10F590003C7106F013F807F10C00264901F0A6F9BA
:10F5A00007F10C007D6487F8484004F05FFA08B169
:10F5B000FDF7B4F8204BFB6007F10C0005F024FACE
:10F5C00008B1FDF7ABF81C22002107F10C0005F093
:10F5D000F5FF00234FF42042C7E903324FF47032A5
:10F5E0007A617B8303223B773B6207F10C00134B6C
:10F5F0003A767B6200F0A6FF08B1FDF78FF8B837C6
:10F60000BD46BDE8F08100BF01F2010030580200A4
:10F610002058020006001800042C0020D01B0020F7
:10F62000FDF0010065F201004C2B00203BF00100D1
:10F63000182C002038580200F5F2010069F2010090
:10F640001FB50B78052B18D0062B1CD0042B17D117
:10F650008B79022B14D1CB7993B90DF10F02019262
:10F660000A4A0B48128800921946012205F0BAF89E
:10F6700030B99DF80F20074B01E0074B01221A70AB
:10F6800005B05DF804FB044B0022F8E7D41B002012
:10F690004C1C002090330020A02C002073B51C4689
:10F6A0000B4B1B7843B181B90A4B1B88214602B032
:10F6B000BDE8704005F053B8064B1B880093134615
:10F6C000224604F0EDFF02B070BD0020FBE700BF52
:10F6D000A02C0020D41B00200328F8B50D461746A7
:10F6E00026D81B4B1C5CFF2C22D01A4E0B463046F2
:10F6F0002146FFF7D3FF13281BD1174B93F83E1079
:10F70000062915D093F83D200C2050430132D2B287
:10F7100003EB000C052ACCE9017601F1010108BFD9
:10F7200000221C548CF8015083F83E1083F83D20D1
:10F73000F8BD112807D8094BC340DB07F8D4BDE852
:10F74000F840FCF7EBBF43F201439842F0D0F6E7F4
:10F75000481C00204C1C0020282C002001810200A5
:10F760002DE9F041394D3A4F92B00646182200215A
:10F77000284605F023FF08220021384605F01EFF29
:10F7800008232B8040F27F136B8040F27F230224FA
:10F790004FF001087B804FF481736B81002140F2B0
:10F7A0000313A7F800807C713C71482268466B8285
:10F7B0006C712C71AC712C816C732C73AC732C82BA
:10F7C0006C752C75AC7505F0F9FE224B22488DF84E
:10F7D0000880CDE9003603238DF80A307223ADF896
:10F7E00024301E4B089300261D4B8DF80960694696
:10F7F00003958DF8108005978DF8186007960C9387
:10F800008DF836600E968DF82C408DF834408DF8CA
:10F8100044408DF842408DF845408DF846408DF8C3
:10F820003C408DF83D408DF83E4004F01DFD08B190
:10F83000FCF774FF0B4B9E8783F83E605E601E6191
:10F84000DE619E625E6312B0BDE8F081682C00202C
:10F85000A22C002041F601004C1C0020D61B0020E9
:10F8600001010003282C0020012870B5CEB21AD166
:10F87000012E17D11E4A92F83E1099B192F83C30F1
:10F880000C2000FB032001330024DBB2013944606B
:10F8900082F83C3082F83E10052B03D1144B002235
:10F8A00083F83C2070BD0028FCD1002EFAD1104C0A
:10F8B00094F83E30002BF5D094F83C100C256943A9
:10F8C0006018615C437842688068FFF7E7FE1328A0
:10F8D000E8D094F83C3094F83E2005FB0345013312
:10F8E000DBB2013A6E6084F83C3084F83E20D3E706
:10F8F000282C0020034B93F83E00B0FA80F040091A
:10F90000704700BF282C002010B5294C294B2178C6
:10F910004A1CD2B2052A23F811002270194646D992
:10F92000002323701A4631F813000133062B0244DA
:10F93000F9D1B2FBF3F2204B2049534341F20300CB
:10F940004FF4B042B3FBF2F39AB282420A8011D96B
:10F9500064238B704FF6FE728978194803F0EFFF2D
:10F96000132820D8174BC340DB0720D4BDE8104034
:10F97000FCF7D4BE40F60650824207D99BB2A3F6EC
:10F980000753092293FBF2F30F33E2E740F65330BB
:10F99000824283BF9BB2A3F654331D22002388BF4B
:10F9A00093FBF2F3D5E743F201439842DED110BD59
:10F9B0009233002098330020E03B02009433002073
:10F9C000AC2C002001810A001FB5102200216846DE
:10F9D00005F0F4FD002300930293642301228DF8C7
:10F9E0000C306946022308488DF804208DF80D304C
:10F9F0008DF80E308DF80F3003F030FF08B1FCF7B2
:10FA00008DFE05B05DF804FBAC2C00202DE9F04123
:10FA1000194D0FCD8AB06C460FC40FCD0FC4174BD4
:10FA200095E803009F7884E8030047B92720FBF797
:10FA3000E8FA27200AB0BDE8F041FBF7B4BB032584
:10FA400064240A26A74210DB97FBF4F292FBF6F33C
:10FA500006FB13230AAA02EB830313F8288C404603
:10FA6000FBF7CFFA4046FBF79EFB94FBF6F4013D13
:10FA7000E8D10AB0BDE8F08140580200943300207C
:10FA80006DDF704779DF70477DDF704764DF704757
:10FA90002DE9F74F0C9CBDF834B02788002580462F
:10FAA0008A4691462E46B8F80020B2420BDC35B1AA
:10FAB0002288013AD21B92B2FF2A39D8DA550020A7
:10FAC00003B0BDE8F08FD8F8042052F8260001906A
:10FAD00000220DF1030101A8FFF7D8FF0028EFD1A4
:10FAE0009DF803204A4521D12288002D14BF002013
:10FAF000022002EB09010144594519DC3DB90132EC
:10FB000092B2228003F802A0228801322280228849
:10FB10000DF103011A4401A8FFF7B8FF0028CFD167
:10FB200021889DF803200A44228001250136BAE786
:10FB30000C20C5E72DE9F341089CBDF82450174679
:10FB4000CDE9004502220646FFF7A2FF48B9102280
:10FB500039463046CDE9084502B0BDE8F041FFF72F
:10FB600097BF02B0BDE8F0812DE9F04F0023168861
:10FB7000138090F82D3085B007460D46144653B3D8
:10FB8000082E01D80C2026E102A8FFF779FF0028F3
:10FB900040F0218113880822CA54238801339BB284
:10FBA0001B222380CA542088013080B22080062284
:10FBB0000DF10901284405F0F6FC23889DF8082082
:10FBC00006339BB212F0FE0218BF01222380EA54D2
:10FBD000238801332380BB78FBB123880433B342ED
:10FBE000D0D802A8FFF74EFF002840F0F480238809
:10FBF0000322EA54238801339BB219222380EA545A
:10FC00002388BDF8082001339BB2E9182380EA5409
:10FC1000120A4A70238802332380FA789AB1238823
:10FC2000D91CB142AED80221E954238801339BB2DA
:10FC300001212380E95423880B449BB22380EA549A
:10FC400023880B4423807A68AAB12388D91CB14247
:10FC500098D8022192F90020E954238801339BB2FD
:10FC60000A212380E954238801339BB22380EA547C
:10FC70002388013323803B89002B40F0A0803B8AFE
:10FC80005BB1CDE900462B460722032107F11000A6
:10FC9000FFF750FF002840F09E803B8B5BB1CDE921
:10FCA00000462B461522142107F11800FFF742FFEA
:10FCB000002840F090803A6A002A40F08F80D7F800
:10FCC0002480B8F1000F30D0B8F804302188981C97
:10FCD0008A1C0244B2423FF655AFFE283FF652AFAF
:10FCE00003336B54238801339BB2FF222380EA54F1
:10FCF000238801339BB22380B8F80020EA54E91826
:10FD0000120A4A702088023080B22080B8F804209D
:10FD10005AB1D8F8081000296AD0284405F043FCED
:10FD20002388B8F804201344238097F82C30002B44
:10FD300040F09980387800284DD03B88012B57D06F
:10FD400021888A1CB2423FF61DAF012805D17B787D
:10FD500002330B449E42FFF415AF023E761A04A90B
:10FD6000B6B221F8086DA818FFF78EFE98BB397857
:10FD7000BDF80820022900F0BB807B78934202D3B3
:10FD8000B24240F2B380012940F0B4809BB29E425F
:10FD9000C0F0B080ADF808300821BDF80830FE2B67
:10FDA0003FF6F0AE22880133AB542288013292B282
:10FDB0002280A95422881344238000200BE0CDE93F
:10FDC00000462B460622022107F10800FFF7B2FE8B
:10FDD00000283FF454AF05B0BDE8F08FB4F800C080
:10FDE0000CF10603B3423FF6CDAE1188052901D8C8
:10FDF0000720F0E76FF4486E01EB0E039BB24FF261
:10FE00007D3E7345F4D95388052BF1D96FF44860D2
:10FE1000181880B27045EBD94FF6FF70814203D0BD
:10FE2000834201D09942E3D8052305F80C3023889A
:10FE300001339BB212212380E954238801339BB202
:10FE400023801188E954E818090A41702388023395
:10FE50009BB223805288EA54E918120A4A70238818
:10FE6000023323802BE7BB6A002BC1D04FF000097F
:10FE70004FF00C0A4FF0160B97F82C305FFA89F20E
:10FE800093427FF657AFB96A0AFB02F201EB020810
:10FE9000B8F80430981CFE283FF674AE208803336F
:10FEA0002B54238801339BB2238005F803B02388A9
:10FEB00001339BB223808A5AEA54E918120A4A7025
:10FEC0002088023080B22080B8F804205AB1D8F8D7
:10FED000081000298CD0284405F065FB2388B8F869
:10FEE00004201344238009F10109C5E7092154E7DF
:10FEF000B242FBD9ADF808604EE770B5C0B14AB167
:10FF000016880024B44203D305196D789D4208D0A9
:10FF1000A14201D800200BE0055D01352C44A4B2BC
:10FF2000F0E7A142F6D9A31C1380005D013880B22E
:10FF300070BD37B502AC002324F8023D13462246BB
:10FF40000546FFF7DAFF10B1BDF80600284403B0FC
:10FF500030BD72DF704773DF704738B50122044649
:10FF60000D46B0F89810D0F89400FFF7E2FF00B10A
:10FF7000057004F13C0204F1940104F15400BDE861
:10FF80003840FFF7E6BF80F830107047F8B50446F8
:10FF90000F46002968D0002866D091F87A301BB14E
:10FFA00091F89830002B61D1D7F8A030042B5DD0A8
:10FFB000D7F89C30042B59D04FF0000C84F802C0C5
:10FFC00007F178060FCE251D0FC50FCE0FC596E899
:10FFD000070085E8070084F830C0D7F8A4306363D1
:10FFE000D7F8A830A3634FF6FF7504F19403C4F863
:10FFF000A430A4F8A8500722614604F1AA0005F035
:020000040002F8
:10000000DDFA23780BB984F85450224604F15501E7
:100010001F25C4F89410384622F8985FFFF7A4FD16
:1000200008BB224604F17401C4F89C1007F13C009F
:1000300022F8A05FFFF798FDA8B9A269A4F84820AC
:1000400001236269206484F850006264014684F8E8
:10005000513084F83C3004F13C0204F15400FFF7C5
:1000600078FF00B92370F8BD0E20FCE70720FAE7FF
:10007000F8B5077804460D46002F00F0FA8000F12D
:10008000AA06A17007220021304605F097FAE388FE
:1000900013B1A378012B04D0E3794BB1A378022BE1
:1000A00006D1636BA3B1012284F8B12008209847E0
:1000B000334604F1B00113F8012F12B99942FAD175
:1000C00017466B1E032B53D8DFE803F0050B0F1206
:1000D00084F8B130ECE7A3791BB194F8243003B96C
:1000E0005FB9E3790BB1002F44D1237A002B43D1C0
:1000F000637A002B0CBF00250425636BA570002BD1
:100100003CD0033D012D39D86279002A36D094F8CD
:10011000B220002A32D184F8B420012284F8B3201E
:100120000720984704F13C0518220021284605F0D5
:1001300045FAE36A0122591E914288BF134684F8AA
:10014000513094F8243084F83C2033B1914296BF6A
:10015000A36A84F8522084F85230A278002384F8ED
:100160005030042A1BD8DFE802F06C0D2232520016
:100170000025C2E70225C0E70325BEE7002384F877
:10018000B330CFE7C4F8A430C4E9106302230122DE
:1001900084F83C30802384F83120A4F84830A378D8
:1001A000002B51D1636B002B5FD100205CE0022358
:1001B00084F83130032384F83C302369A4F84830B4
:1001C0000023C4F8A430E36826646364E7E7636946
:1001D0006364A369A4F848306379B3B194F8B2308A
:1001E0009BB994F8B43083B1022384F850300421D1
:1001F0002046FFF7B2FE0028D1D1052384F8313024
:1002000004F19403C4F8A430C9E70323F6E7E369D3
:100210006364236AA4F84830637983B194F8B230F8
:100220006BB994F8B43053B1022384F850300421F0
:100230002046FFF792FE0028B1D10623DEE7042313
:10024000DCE784F83130AAE72A46D4F8A41004F198
:100250005400FFF77EFE38B994F8301094F854003B
:10026000FFF779FE00289DD0F8BD94F8310098473B
:100270009BE70820F8E710B50388112B0C460AD03D
:10028000262B1FD0102B05D1C37B012B02D18388D5
:10029000A1F8A83010BD002381F8B2308288B1F8EF
:1002A000A8309A42F6D10B79002BF3D101212046D8
:1002B000FFF7DEFE0028EDD0A36B002BEAD0BDE8EF
:1002C00010401847037A013B012BE3D889780523B6
:1002D000013191FBF3F303EB8303C91AC9B2E6E7DB
:1002E000704710B590F8B13043B1002480F8B140A8
:1002F0000722AA3005F057F9204610BD0820FCE778
:1003000090F8B3306BB1002380F8B3303AB9009B5A
:10031000003318BF012380F8B43000207047012358
:10032000F9E70820704730B50D46041D0FCD0FC406
:100330000FCD0FC495E8070084E8070030BD75DFD6
:10034000704776DF70477ADF70477BDF70470000C9
:10035000034B1A8882420CBF18460020704700BF2A
:10036000DC2C0020024B9B6903B11847704700BF8B
:10037000C02C002037B585B22846FFF7E9FF0346B9
:1003800070B1164C017A227B91420BD200F10A0126
:100390002846FFF7D4FFE8B1112801D0FFF7E2FFAC
:1003A00003B030BD237C0022027243B13B212846BA
:1003B000FFF7C7FF30F0080301D0FFF7D3FF6369F1
:1003C000002BEDD000228DF80420ADF8065001A8D6
:1003D0009847E5E71A7A01321A72E1E7C02C00204B
:1003E00013B50B46497A0F4C024669B9D4E901109E
:1003F0001C7A002C18BF0146586805F027F808B190
:10040000FFF7B0FF02B010BD002119726369002B25
:10041000F8D00121ADF806008DF8041001A8984726
:10042000F0E700BFC02C002030B583880588B3F505
:10043000FA7F24BF6FF4F9729C184A8838BF0024F1
:1004400095420CD84088904209D38A88A24206D3AC
:1004500003F2F310904234BF0020012030BD002091
:10046000FCE7000070B50388112B014648D002D884
:10047000102B1ED070BD122B52D0502BFAD12F4B07
:10048000C288DB899A42F5D1038A022BF2D1868891
:100490003046FFF75DFF05460028EBD001F1120062
:1004A00000F016FA30BB686805F014F80028E1D0B7
:1004B00009E0C37B012BDDD14FF6FF70FFF748FF4A
:1004C000054620B90420BDE87040FFF74BBF8E8879
:1004D0001B4A0680002303721368C5F80A300A30ED
:1004E000536843601031FFF79FFF144B6872DB893C
:1004F000002BBFD129463046BDE87040FFF770BFE2
:100500008088FFF725FF04460028B3D0406804F038
:10051000E1FF08B1FFF726FF4FF6FF732380A9E73D
:1005200086883046FFF714FF05460028A2D0083120
:100530000A30FFF779FF6872DCE700BFC02C0020AB
:10054000F02C0020F8B5064650B305460FCD154FE8
:100550003C460FC495E8070084E807003068124B5A
:100560003B60B8B1FFF7EFFEC8B931680A681A609E
:100570004A685A600D480E4A4FF6FF7303800D4BD0
:1005800040F8043F002104F04FFF002814BF03206F
:10059000002004E01846FFF7D8FE0028EAD0F8BD96
:1005A0000E20FCE7C02C0020F02C0020DC2C0020CA
:1005B00075030200F82C0020F7B5174601900E468F
:1005C00091B1019C6CB100252C46294601A8FDF78C
:1005D0003EF918B13946A8B2B04701340135142D9F
:1005E000F3D1204603B0F0BD0C46FAE773B5019194
:1005F000019C06466CB100252C46294601A8FDF752
:1006000026F918B106EB440301349D800135142D01
:10061000F3D13046346002B070BD00002DE9F043E4
:1006200003888488112B8DB0064640D01A2B43D006
:10063000102B16D1294DAB680CA8DB4340F8303D98
:1006400055F8041FFDF759F9009901A8FFF7CEFFEF
:100650000027019B9F4207D3132C18D90420FCF7D5
:100660005DF80DB0BDE8F08301AB03EB47034FF03D
:100670000008B3F8049005EB0800494608F10408A7
:10068000FDF7DBF8B8F1740FF5D10137E1E721464A
:100690001348FDF7BBF821461248FDF7B7F8F37B86
:1006A000012BDED010482146FDF7B0F8D9E70C4801
:1006B0002146FDF7C2F8D4E7057A0C482D09012D33
:1006C000214606D9FDF7A2F8022D21460848F0D0B0
:1006D000EAE7FDF7B2F821460548EAE7182D0020C1
:1006E000202D00201C2D0020242D0020282D00204E
:1006F0002C2D00201328014602D80248FDF7A7B888
:10070000002070471C2D0020FFF7F4BF10B50446F1
:10071000FFF7F0FF38B121460348FDF798F80028AD
:1007200014BF0220012010BD202D002010B504466A
:10073000FFF7E0FF28B121460248BDE81040FDF771
:1007400086B810BD282D002010B50446FFF7D2FF53
:1007500028B121460248BDE81040FDF778B810BD29
:100760002C2D002010B5034B04465968FFF73EFFBF
:10077000204610BD182D002010B50446FFF7BAFF23
:10078000002814BF2046142010BD000008B5182111
:100790000248FDF765F8C0B208BD00BF182D002063
:1007A00070B50A4D064628460C46FDF750F858B17C
:1007B0003046FFF79FFF38B1A01D314605EB8000A2
:1007C000BDE87040FDF743B8002070BD182D002033
:1007D000F8B50D4C054620460E461746FDF737F88E
:1007E00080B12846FFF786FF60B1B01D04EB8000A2
:1007F00029461FB1BDE8F840FDF708B8BDE8F8404C
:10080000FDF71BB8F8BD00BF182D0020034B9B68F7
:100810000A4601461846FFF7CFBE00BF182D00203C
:10082000F8B50A4C05460E46014620461746FDF728
:100830000EF848B1043504EB85043A46A068314609
:10084000BDE8F840FFF7B8BEF8BD00BF182D002086
:1008500070B5054616460AB90E2070BD0023136018
:100860000028F9D00368002BF6D0C38813F00304E6
:100870000FD10846FFF780FFC0B214280BD02B79A8
:1008800083420AD9EB882A6800FB032030602046A7
:10089000E3E70720E1E70520DFE70420DDE7AADF43
:1008A0007047ABDF7047002301380B70042806D86F
:1008B000DFE800F00306080A0C0011230B707047F4
:1008C0002123FBE73123F9E71223F7E72223F5E79A
:1008D000007800F0010070470078C0F340007047D6
:1008E0000B7803704B7843700220704738B504468C
:1008F00008460D4604F072FE6560208038BDF0B5F4
:100900008B7891B005460C46164603B901230322A5
:100910008DF80E3000212388ADF80C30684604F0C5
:100920004DFE6946607CFFF7BEFF0DF10101A07C22
:10093000FFF7B9FF9DF80230E27B62F3C303227C2C
:1009400062F30413227B62F30003227D002A14BFAA
:100950000222012262F3420300211C2209A88DF821
:10096000023004F02BFE637B13F0300F15D002AF82
:1009700003220021384604F021FE0DF10901E07C3C
:10098000FFF791FF11238DF808309DF80A300E977C
:10099000012262F342038DF80A30637B8DF8243024
:1009A0001422A37B8DF82530002104A804F006FE54
:1009B00003AB0493A388ADF81C30A368CDF814D022
:1009C0001BB1E288ADF818200893A369002B32D040
:1009D00001AF03220021384604F0F0FDA3691A8814
:1009E000ADF82C205A88ADF82E205A680D97187B48
:1009F0000A923946FFF757FFA3690DF10501587BAD
:100A0000FFF751FFA2699DF80630917A61F3C303A5
:100A10008DF80630D17A61F304138DF80630117A1F
:100A2000927B002A61F3000314BF0222012262F3C9
:100A300042038DF80630E36903B10C93334604AAF0
:100A400009A92846FFF72BFF11B0F0BD70B50C4681
:100A500088B0054616460021142203A804F0AEFD16
:100A6000A37803B901238DF80A3008AB228823F854
:100A7000182D01AA1146A0790393FFF714FF0DF179
:100A80000501E079FFF70FFF9DF80630E178049249
:100A900061F3C303217961F30413617961F3000306
:100AA000217A002914BF0221012161F342038DF84C
:100AB00006306389ADF81430A389ADF81630E389A8
:100AC000ADF8183032462369079303A92846FFF78B
:100AD000E8FE08B070BDA0DF7047A1DF7047ADDF52
:100AE0007047B3DF704710B50446408800F0E2FC61
:100AF000A0802046BDE8104001F0B6BC30B587B0FC
:100B000005460C4618220021684604F057FD0723CD
:100B100068468DF80030ADF802500294FFF7E3FF0D
:100B200007B030BD30B587B00546182200216846B1
:100B300004F044FD4FF6FF739D42ADF802501AD009
:100B4000284600F062FB0B2804461DD005D8A0B152
:100B500021462846FFF7D2FF05E0112805D043F2D1
:100B600002039842F4D1002200E00122074B2846FC
:100B70001978FFF72DFE07B030BD0E2368468DF8BB
:100B80000030FFF7B0FFEEE70F23F7E7972D0020C7
:100B9000FFF7C8BF024B034918780022FFF740BE99
:100BA000992D0020A90B02002DE9F0433D4F89B09B
:100BB00039780446FFF7F4FD064600286BD120463D
:100BC00000F072FB0828014622D006D888B106281A
:100BD0004BD02046FFF792FF09E043F20203984210
:100BE00005D043F20143984258D01128F1D1012396
:100BF00046E03146182202A804F0E0FC102302A8C7
:100C00008DF80830ADF80A400126FFF76CFFEEE7DB
:100C100001A8FFF766FF012533464FF002080DF1EA
:100C20000609BDF80420AA421FD902AA2946204677
:100C3000CDE90289FFF753FFB8B9BDF806200135A9
:100C400033B942F60523D21A53425341ADB2E8E715
:100C500042F602118A42F9D10DF102020392A9B2C1
:100C600002AA2046FFF73BFF30B1204600F022FCED
:100C700000F034FB002303E0BDF80220002AF4D08A
:100C80001A46094B20461978FFF7A2FD32463978FB
:100C90002046FFF79DFD09B0BDE8F0832046FFF731
:100CA00041FFA4E79A2D0020992D002013B504469A
:100CB00000F000FC00236A46092101F039F80528FC
:100CC00005D1044B012219782046FFF781FD02B0BF
:100CD00010BD00BF952D002008B5084B08491878B5
:100CE0000022FFF79DFD024630B9064B06491878F1
:100CF000BDE80840FFF794BD08BD00BF982D002057
:100D0000550D0200952D00200D0D020013B5042293
:100D100004460021684604F051FC0C4A42F6A62322
:100D20001068ADF800300190012301AA6946204601
:100D30008DF80230FFF7CFFE28B91A46044B204643
:100D40001978FFF745FD02B010BD00BF68580200DA
:100D5000942D002030B5012187B005461C48FCF7D2
:100D6000ACFD0446BFF35F8F00BB284600F008FAD5
:100D7000112801461CD005D860B12846FFF7BEFEF9
:100D8000002405E0862815D043F202039842F4D1EE
:100D9000224601E0012402460E4B28461978FFF74F
:100DA00017FD1CB9BFF35F8F094B1C6007B030BD46
:100DB0000122F1E718222146684604F0FFFB0623D2
:100DC00068468DF80030ADF80250FFF78CFEDFE783
:100DD000902D0020982D002038B503780446A3B943
:100DE0004088FFF79FFE6588284600F04BFA28B13F
:100DF000064B012219782846FFF7EAFC6088FFF7C6
:100E000055FFBDE83840FFF767BF38BD992D00207A
:100E100037B50378082B044630D1427A72BB057A85
:100E2000072D1BD0082D2DD0012D27D16A4629462C
:100E3000808801F0A7F908BB019B1B78F3B1A0885B
:100E400000F066FB4FF6FF73984217D0114B2A460D
:100E50001978FFF7BDFCFFF79DFE0FE0808800F0DA
:100E600057FB4FF6FF739842044607D00A4B012206
:100E70001978FFF7ADFC2046FFF718FFFFF72CFFAE
:100E800003B030BD054B19680129F7D1BFF35F8F5F
:100E90001A60F3E7992D0020982D0020902D002056
:100EA0002DE9F843FFF772FCDFF89090DFF89080AF
:100EB00089F80000FFF76AFC88F80000FFF766FC7D
:100EC000184F194E3870FFF761FC3070FFF75EFC69
:100ED000164D174C2870FFF759FC2070FFF756FC91
:100EE000144B187099F80030182B18D098F800306F
:100EF000182B14D03B78182B11D03378182B0ED028
:100F00002B78182B0BD02378182B08D0182806D054
:100F1000094B00201860BFF35F8FBDE8F883032002
:100F2000FBE700BF992D00209A2D0020952D002071
:100F3000942D0020962D0020902D0020982D00202B
:100F4000972D002073B501230024ADF8003009234C
:100F5000CDF802408DF802300B4BADF8064022462A
:100F60000E4619780546FFF733FC084B084928461A
:100F7000A64208BF1946019100F09CFA2246694634
:100F800000F042FF02B070BD952D00206C580200A9
:100F90007058020070B503888488502B86B00546CF
:100FA00037D00DD8352B47D0362B62D03E4B3F493A
:100FB00018780022FFF734FCFFF7ECFD06B070BD97
:100FC000522B22D0542BF1D118220021684604F074
:100FD000F5FA112320468DF80030ADF8024000F0FC
:100FE00069FAADF8040000F079F9314B2046197820
:100FF0000022FFF7EDFB2F4B204600221978FFF768
:10100000E7FB6846FFF76FFDD0E72046FFF78AFD54
:10101000CCE7037B012BC9D1827A012AC6D1018991
:1010200042F602139942C1D1234B20461978FFF7AB
:10103000CFFBFFF751FEB9E7204E20463178FFF78E
:10104000AFFB0028B2D0002231782046FFF7C0FB6A
:10105000EA883ABBAB89012B24D1E9892046FFF706
:101060003CFDF8B91A46164B20461978FFF7B0FB3D
:101070009CE7134E20463178FFF792FB002895D06D
:10108000317800222046FFF7A3FBE98851B9EB89AC
:10109000012B03D1297C003118BF01212046FFF725
:1010A00051FF83E70021F9E7972D0020910B020003
:1010B0009A2D0020992D0020982D0020942D00209D
:1010C000962D0020AFDF7047B1DF7047B2DF704769
:1010D000B3DF704710B50446808800F019FA6080CD
:1010E0002046BDE8104001F0C1B90000F0B5184B32
:1010F000184C93E8030089B06E4686E803004FF66B
:10110000FF772088B8421CD00022314600F07CFED8
:101110000546C0B11822002102A804F04FFA238826
:10112000ADF80C30112D0CD0862D0CBF06230723F3
:1011300002A80EBF8DF808308DF808300495FFF72F
:10114000C9FF09B0F0BD208800F0B0FE2080D8E7CC
:10115000745802009C2D0020044B1A884FF6FF7330
:101160009A4201D0FFF7C2BF704700BF9C2D0020FC
:10117000024B4FF6FF721A80002070479C2D002012
:101180002DE9F743804600F095F94FF6FF7398423A
:10119000064637D001224FF003096B46082130463E
:1011A000571C00F0F3FFBFB2054630BB01990A4659
:1011B000032342F8049B06314046FFF787FF0446AD
:1011C00048B932460821304601F06BF80446204603
:1011D00003B0BDE8F0830C280DD0052800D12C46C3
:1011E0000821304601F032F8002818BF03243A469F
:1011F000002DD2D1EBE70125F2E7072814BF044602
:101200000C24E4E743F20204E1E72DE9F3418046D0
:1012100000F050F94FF6FF73984217D100240325D0
:10122000264601272B46224631464046FFF74CFF13
:10123000042820D0082823D00B281DD115F0020344
:101240000FD18EB9A4B902B0BDE8F0816A46082179
:1012500000F098FF0028E1D1019B9E1D9C881D682D
:10126000DFE701250027DDE703251C461E46F9E7D9
:1012700003253446F6E71120002F08BF0B20E2E7D4
:101280000020F9E71FB50DF10703039300F012F9F1
:1012900002AA012100F076FF20B9039B187805B05F
:1012A0005DF804FB0020FAE738B504460A48FFF76A
:1012B0000FFF70B9084B43F203054FF6FF72198810
:1012C0002046FFF7FFFEA84204D11A8801321A8097
:1012D000F3E7032038BD00BF9E2D002013B5074A59
:1012E000044692E803006B4683E803000022194697
:1012F000204600F089FD02B010BD00BF7C580200FE
:101300006EDF70476FDF704746DF70472DE9F04FA3
:1013100099B01E46502383468846DDE92257ADF832
:1013200006301446EAB1F6B1002333604FF00109EC
:10133000DDB1E7B100233B604FF0010A0822002134
:101340000DEB020004F03AF9C8EBC80804AB0393B4
:10135000ABF1020BA04444450BD1002019B0BDE80D
:10136000F08F9146E4E7B146E2E7AA46E6E7BA46DF
:10137000E4E75022002104A804F020F90DF106034F
:1013800002AA07213BF8020F00F0D2FC20F0020075
:101390000528E3D09DF82130032B1AD8B9F1000FAE
:1013A00008D007220DF12101204604F0FCF8336833
:1013B00001333360BAF1000F08D010220DF1110192
:1013C000284604F0F0F83B6801333B6010350734E1
:1013D000C1E743F20220C1E7421E00F10F0312F8F9
:1013E000010F10B99A42FAD170470120704708B531
:1013F00070B171B103780A78534013F0FE0F08D131
:1014000006220131013004F0BFF8B0FA80F0400943
:1014100008BD0020FCE72DE9F04700F101084F1C52
:1014200006460D4600F1110901F1110A1022394654
:10143000404604F0A9F80446E0B94046FFF7CCFF67
:1014400018B13846FFF7C8FF044651464846FFF733
:10145000CEFF737C03F0FC03042B04D06B7C03F001
:10146000FC03042B02D1201C18BF012000F0010056
:10147000BDE8F0870024E8E730B585B004460D46A6
:1014800000F08CFC02AA0DF10601072000F08EFC92
:1014900010B94FF6FF700BE0BDF80630AB42F1D04B
:1014A00003992046FFF7B7FF0028EBD0BDF80600F0
:1014B00005B030BD132810B5044602D94FF6FF70B1
:1014C00010BDFFF717F90028F8D00A206043014B40
:1014D000185AF5E7A02D0020132838B504460D460C
:1014E00002D943F2020038BDFFF704F90028F8D012
:1014F00006480A2303FB040050F8023F2B60838850
:10150000AB808379AB710020EDE700BFA02D0020F8
:101510004FF6FF7398422DE9F04106460CD00C4F70
:1015200000244FF00A0808FB04F3A5B2DB5BB342CA
:1015300005D00134142CF6D14FF6FF7504E028468F
:10154000FFF7D8F80028F4D02846BDE8F08100BFA6
:10155000A02D0020038843B9821C00F10A0312F871
:10156000010B10B99A42FAD170470120704710B5AB
:101570000446FFF7EFFF58B122880B889A4208D142
:1015800008220231A01C03F0FFFFB0FA80F04009EE
:1015900010BD0020FCE71FB5044600F0FFFB02AAC7
:1015A0000DF10601072000F001FC10B94FF6FF70A5
:1015B00007E0039920464631FFF7D9FF18B1BDF87F
:1015C000060004B010BD039920462A31FFF7CFFF73
:1015D0000028E4D0F3E7000013289FBF0A235843F4
:1015E000014B1952704700BFA02D002038B50546A9
:1015F000FFF78EFF0446284600F032FE38B9132C60
:1016000005D80A236343024A4FF6FF71D15238BD11
:10161000A02D00202DE9F0410D46CEB0804600B14E
:1016200039B9002211461046FFF76CFE4EB0BDE8F6
:10163000F08120AE50230CAFB82200213046ADF827
:101640000630039703F0BAFF0DF1970305930DF1F0
:10165000AE0306930DF1C503079337AB08930DF165
:10166000F30309930DF585730A930DF22113049684
:101670000B93002450220021384603F09FFF0DF108
:10168000060302AA072138F8140000F051FB20F0ED
:1016900002000528CAD07B7C032B0DD8172202FB41
:1016A00004600DF13101013403F07DFFA542E1D169
:1016B000EAB2002104A8B7E743F20220B6E700002F
:1016C00037B50B4C247811B10D68A5420DD313B179
:1016D0001D68A54209D3CDE900230B4602462146E9
:1016E0000448FFF713FE03B030BD0420FBE700BF42
:1016F000682E00206A2E00202DE9F04110229AB0B9
:1017000007460C462048002103F058FF1F4B07B145
:101710003CB9002119700846FFF7F2FD1AB0BDE888
:10172000F0810025620039460CAE5FFA84F8164855
:1017300083F8008003F037FF3822294630460395AE
:1017400003F03CFFCDE9005503AB32462146384655
:10175000FFF7DCFD0028E1D10DF1370305930DF112
:101760003E0306930DF14503079313AB08930DF168
:10177000530309930DF15A030A930DF16103049683
:101780000B93414604A8C7E76A2E0020682E00206C
:1017900030B58DB014460D4600F110030DF1FF3247
:1017A00013F8011D02F8011F9842F9D10D22002102
:1017B00004A803F003FF2B788DF81F306B788DF8A9
:1017C0001E306846AB788DF81D30FFF79DFD9DF803
:1017D0002F3023709DF82E3063709DF82D30A3704C
:1017E0000DB030BD30B5037803F0FE03042B85B097
:1017F00004460D4618D1411C032201A803F0D3FE74
:101800000322211D03A803F0CEFE02AA03A9284645
:10181000FFF7BEFF032202A901A803F0B5FEB0FA4C
:1018200080F0400905B030BD0020FBE730B50388EB
:10183000102B93B052D1041D0FCC08AD0FC50FCCA7
:101840000FC594E8030012AC85E8030014F8243DAA
:1018500003F0FE03062B4BD000F0A0FA9DF82430D5
:101860005B08012B3CD9022B42D102AA0DF10601E3
:10187000072000F09BFA00283AD003992046013156
:10188000FFF7B0FF0028F0D005E0039920461131A2
:10189000FFF7ADFD20B3BDF80630BDF820101648A7
:1018A0000A224A4385188352AA1C0998C5F80200E7
:1018B000A588A079958090714FF6FF7293420DD064
:1018C00012ACADF80C30002304F8403D2046ADF8D2
:1018D0000A1000F0CDFD2046FFF77EFA13B030BDB0
:1018E00002AA0DF10601072000F060FA0028CCD111
:1018F0004FF6FF73D1E700BFA02D0020A5DF704792
:10190000B5DF704768B14FF0171303601B230371F5
:101910001723C38003810023C1608372C3721846FA
:1019200070470E20704737B583880C467BB9028814
:10193000112A47D00DD8102A2FD0A37A3BB1E188C5
:101940000020FFF7DBFF10B90123A072E37203B0A0
:1019500030BD3A2A3BD0552AEFD1C288C988A3723C
:10196000172A38BF17228A4228BF0A462281184602
:10197000FFF7C6FFE27A002ADFD1E368002BDCD054
:1019800040F67721ADF802202289ADF80010ADF8BD
:101990000420694620469847CFE7C37B012B04BF4C
:1019A0000B88CB80C98823898B42C6D20020FFF7E1
:1019B000A5FF10B90123E372BFE71128BDD10123B0
:1019C000A372BAE71722CA800A818B72F3E74289B1
:1019D000C988E5688A4228BF0A46172A38BF1722F5
:1019E000228165B1E17A51B140F67721ADF800105E
:1019F000ADF80230ADF8042069462046A847002320
:101A0000E372DDE7B0DF704766DF704710B503466D
:101A100000214088FFF7F8FF024608B91A7210BD8E
:101A2000112801D10122F9E75B68BDE81040184791
:101A300060B159B10378DE2B0AD00B684360DE2316
:101A400003704FF6FF734380002070470E207047ED
:101A50000820704728B10378DE2B04D14180002094
:101A600070470E20704708207047F0B5054685B0D6
:101A70000C46F1B1E8B10B78DE2B1AD182884B8885
:101A80009A4204D10B7A13B10846FFF7BFFF2B88A7
:101A9000112B32D0512B0ED0012B0AD12B7A012BD6
:101AA00007D1A9886288914203D123722046FFF7AB
:101AB000ADFF05B0F0BDAE886388B342F9D1AF7910
:101AC000022FF6D1AD7B2B1F022BF2D80021102262
:101AD000684603F073FD052D14BF4FF4C073002357
:101AE000694630468DF80070ADF80430FFF78AFF84
:101AF0000028DED063689847DBE76388AA889A42AB
:101B000004BF4FF6FF736380D3E7012804D0043885
:101B100005288CBF0020012070474FF6FF734380DB
:101B200000F082BA73B504460D461646002108221D
:101B3000684603F043FDA5F58041A4F580406B465F
:101B4000324689B280B2FBF789FD002814BF052018
:101B5000002002B070BD0000F0B5214D8DB0002115
:101B6000082201A8297003F029FD4FF6FF7000F04C
:101B70004BFC4FF6FF770446BC4211D0A4F58046DB
:101B8000B6B201AA03A93046FBF782FD0A2809D0A4
:101B90003046FBF719FD082806460BD101232B70B0
:101BA0000DB0F0BD204600F0D3FB204600F02CFC29
:101BB0000446E1E7002EF3D0182200210DEB0200CD
:101BC00003F0FCFC07238DF8183006A80123ADF8BC
:101BD0001C4008968DF82430FFF79FFFE0E700BF18
:101BE000842E002070B5044686B018220021684675
:101BF00003F0E4FCA0892378334D00F5804080B2E7
:101C00005A1EADF80400042A25D8DFE802F00303C9
:101C100003324B0043F6FE76B042E18904D901F568
:101C2000804292B2B24216D8DA1E534253418DF826
:101C30000930A368039363688DF808108BB90823F3
:101C40008DF800309DF8103043F001038DF810300E
:101C50006846FFF762FF2B780BB1FFF77DFF06B0F8
:101C600070BD0922049301238DF800208DF81430F3
:101C7000EEE743F6FE739842EDD8E389002BEAD1F4
:101C800063683BB90A238DF8003000F061FB012343
:101C90002B70DDE70B22029301238DF800208DF8D5
:101CA0000C30F4E763683BB913238DF800304FF62E
:101CB000FF73ADF80430CBE71422029301238DF8B3
:101CC00000208DF80C30F2E7842E002030B5174844
:101CD00089B0FBF7EBFA20BBFBF7FEFA044610BB1A
:101CE00000F016FB0822214603A803F067FC03AAB4
:101CF00005A94CF20700FBF7BFFC10B1204609B064
:101D000030BD01A905A8FBF7E9FB019B9D8805F5FE
:101D10008045ADB205A8FBF705FC284600F000FBA6
:101D2000E5E70324EAE78624E8E700BFE51B0200B5
:101D3000F0B5FF2887B004460D4617461E462BD83F
:101D40000846FFF7E2FE38B303AA2046FFF7EAFE93
:101D500018B10524204607B0F0BD01A903A8FBF780
:101D6000BDFB04460028F4D1019BBD705D883D8019
:101D7000029926B9796003A8FBF7D4FBEAE7368815
:101D80007868AD00AE4228BF2E46324603F00BFC09
:101D9000B542F0D90C24DDE70724DBE70822002157
:101DA000014803F00BBC00BF7C2E0020F0B587B0CB
:101DB00007460E461546FFF7A8FE0446F8B1A7F5FC
:101DC0008040104A03A980B2FBF756FC18B10024EA
:101DD000204607B0F0BD01A903A8FBF77FFB002850
:101DE000F5D1019BAF705A882A80029A6A609B885D
:101DF00003F58043338003A8FBF794FBE8E7012455
:101E0000E6E700BF7C2E002030B5FF2887B00346F0
:101E10000C46154635D889780846FFF776FE80B31C
:101E2000A3F58042ADF80020A1F58042ADF8022074
:101E30006268019222880292184603AAFFF772FE96
:101E40000528694603A808D1FBF78EFB072804463E
:101E50000CD005D870B1032409E0FBF789FBF5E746
:101E6000082801D00E28F6D1112400E0862420464F
:101E700007B030BD002DFAD0294603A8FBF714FCAB
:101E8000F5E70724F3E74FF6FF7000F049BAFF28A3
:101E900008B505D800F04AFAFFF75EFE002008BD3D
:101EA0000720FCE700F068BA00F070BA00F092BAC0
:101EB00000F0AABA0A68084B70B50C25032A01D9AC
:101EC000002006E005FB02F4E65A864202D10A60D1
:101ED000181970BD0132F1E7DC2F002073B502AC98
:101EE000002344F8043D0E4605462146FFF7E2FF75
:101EF00038B18378B34206D1837A9B0703D1436814
:101F00000BB902B070BD019B0133019321462846F5
:101F1000ECE710B5044600F0FFFC204601F0F4FBAE
:101F20002046FFF719F92046BDE81040FEF770BFC4
:101F300070B50F4E04460025237AAB420FD84FF6FA
:101F4000FF732380A370FF236372A37A03F0FD0362
:101F50006FF30003A37200232372636070BD617A84
:101F60002944C9B2304600F005FF0135E4E700BF5F
:101F7000CC2F002013B50023CDE90033044683782D
:101F8000417A27488DF8023000F0DBFEF0B1237A69
:101F9000A2788DF8022003EB83039B00ADF800309C
:101FA000531E0190072B08D8DFE803F0120707073C
:101FB000071204141423ADF80030221D694620884E
:101FC000FFF722FF07281DD008D8A8B1032019E089
:101FD0000123F0E7838809339B08ECE7112813D02D
:101FE0008628F3D1A37A03F0FD0343F00103A37223
:101FF0000C4B01221A7005E0A37A60F3410360F3F1
:102000000003A37202B010BDA37A43F002036FF382
:102010000003A372034B01221A700020F2E700BFF5
:10202000CC2F0020C82F00202DE9F047374AC16887
:1020300086B0054600230C24174604FB032046689F
:10204000B14203D00133042BF7D100202B78304E5E
:10205000092B10D0132B50D0082B01D0002406E000
:102060006C7A002CFAD10028F8D0FFF761FF2846DF
:10207000FFF74FFF0BE06C7A002CEFD100283ED029
:10208000837A446043F00203837201233370337810
:1020900083B3002535704FF00C084FF0010A08FBA0
:1020A00005739A7AC2F340030BB9D20729D586F893
:1020B00000A003B92CB308FB05794846FFF75AFF87
:1020C000F8B14FF6FF738628ADF80230B9F800304A
:1020D000ADF8043017BF072306238DF800300290B7
:1020E00018BF002368460CBF8DF800308DF80C3007
:1020F000FFF70FFF06B0BDE8F0870124B7E70446FD
:10210000B5E70135042DCAD1F4E700BFDC2F00206C
:10211000C82F0020174BF7B500221E464FF6FF755B
:102120004FF0FF0C0C27144607FB02611D809D70C9
:1021300083F809C0887A013200F0FD006FF30000D7
:10214000042A887203F10C0303F8044C43F8084C8A
:10215000EAD15023CDE900230749084B08484FF442
:10216000A07200F0DAFD002814BF0320002003B0A5
:10217000F0BD00BFDC2F0020882E00200C30002096
:10218000CC2F00200023FFF7D3BD00002DE9F04144
:1021900080460E4614461F46002B4ED0CB1F012B07
:1021A0004ED8531E032B4BD8FFF798FE054610BBA5
:1021B000FF214FF6FF70FFF791FE0546C8B1A0F86A
:1021C000008086706B7AFF2B1AD121461E4800F0E2
:1021D000E9FDFF2868722DD14FF6FF732B80AB7A93
:1021E000A87003F0FD036FF30003AB7200232B72A2
:1021F0006B60112022E0037AA342E3D00F201DE0A0
:102200004FF000082C72697A0F4800F09AFDC8B1AF
:1022100004EB84042401A4B2A408BE7078603C805E
:10222000B8F1000F04D0082E02D1A400063C84802F
:10223000002003E04FF00108E4E70E20BDE8F08144
:102240000720FBE70320F9E7CC2F002008B5FFF7B4
:1022500045FE18B1FFF76CFE002008BD0520FCE725
:1022600037B502AC002344F8043D05462146FFF78C
:1022700021FE30B92846FFF70AFE50B1072808D0E2
:1022800006E081782846FFF7E1FF20B1052802D05B
:10229000032003B030BD019B013301932146284642
:1022A000E5E7CB1F012B70B506460C46154601D954
:1022B000072070BD1046FFF7F5FD0028F8D0214635
:1022C0003046FFF70BFE28B105808470BDE87040F2
:1022D000FFF750BE0520ECE710B54FF6FF7304463C
:1022E0009C4208460AD14FF48071FBF7B9FA84B2D8
:1022F000B4F5807F09D14FF6FF7406E0FF2CFAD8C1
:102300002146FBF78CFA0028F5D1204610BD0000CD
:1023100040220021014803F051B900BF10300020D5
:102320000149FFF7D9BF00BF103000204FF6FF73FF
:10233000984210B5044606D00449FFF7CDFF231A92
:102340005842584110BD0020FCE700BF303000204B
:10235000FF2810B5044609D801460548FBF76DFA79
:1023600021460448BDE81040FBF767BA10BD00BF26
:102370001030002030300020FF28014602D80248EB
:10238000FBF765BA0020704710300020FF28014697
:1023900002D80248FBF75BBA0020704730300020BB
:1023A0004FF6FF73984270B518BF441C0E4614BF19
:1023B000A4B20024A5B2FF2D02D94FF6FF7506E0A6
:1023C00021463046FBF743FA01340028F2D0284674
:1023D00070BD000070B50B490A4EFFF7E1FF4FF6E4
:1023E000FF750446AC4201D1204670BD2046FFF780
:1023F000CDFF0028F8D020463146FFF7D1FF044634
:10240000F0E700BF103000200149FFF7C9BF00BF4F
:1024100030300020F8B5074D074F064600242B78D2
:10242000A34200DCF8BD57F8243030469847013409
:10243000F5E700BF673000205830002010B5074B8B
:102440001B7804464BB1FFF7F1F9204601F09CF9E7
:102450002046BDE81040FEF79DBD10BD663000204F
:1024600008B1FFF7D7BF7047FFF7D4BFFFF7D2BF60
:10247000FFF7D0BF08B5FFF729FC08B1032008BD5E
:10248000FFF748FE0028F9D101F062F90028F5D1E4
:1024900000F098FD0028F1D1FEF702FD0028EDD1F3
:1024A000FEF766FE0028E9D1054B4FF6FF721A8051
:1024B000044B1860044B1870044B01221A70DEE7BD
:1024C000643000206C30002068300020663000202E
:1024D000084B1B7853B1084A1378022B08D80749D8
:1024E00041F8230001331370002070470820704723
:1024F00004207047663000206730002058300020EC
:10250000034B1B780BB101F059B90820704700BF8D
:102510006630002008B5054B1B782BB101F06EF931
:10252000082808BF112008BD0820FCE766300020FD
:1025300009B101F061B97047034B1B780BB1FFF78C
:10254000DBB80820704700BF6630002010B4094C8B
:1025500024785CB110B922B90E2008E00029FBD024
:102560000AB1002BF8D010BCFFF7AAB8082010BCA5
:10257000704700BF66300020034B1B780BB1FFF79C
:1025800049B80820704700BF6630002038B5194BA5
:102590001B7805460C4633B339B3FEF7B7F830B3B2
:1025A000831E58425841237860F300032370284665
:1025B000FEF780FF4FF6FF73C01A237818BF012083
:1025C00060F3C30323702846FEF7B0F8237860F366
:1025D000410323702846FEF7B7F8237860F382039F
:1025E0002370002038BD0820FCE70E20FAE743F2F4
:1025F0000200F7E76630002010B5084B1B78044650
:102600004BB12046FFF752FC0446FFF74DFC002873
:10261000F7D1204610BD4FF6FF74FAE76630002070
:102620002DE9F04F9846464B1E7889B0834689467F
:102630001446002E79D0002979D0002877D00B6875
:102640000193002B75D0B8F1070F72D84FF6FF77C2
:102650000025BA420D6005D11046FFF7CDFFB84204
:10266000044660D00822002104A802F0A7FF082237
:10267000002106A802F0A2FF08F00303029308F06D
:10268000010308F0040A00270393029B002B52D099
:10269000002306AA072120460793FFF749FB0528D8
:1026A00019D038BB0546039B2BB1079B5B7C13F00D
:1026B000FC0F18BF354618F0020F0ED0079B5A1CAE
:1026C000113312F8011B41B99A42FAD1BAF1000F45
:1026D0001FD0354604E03546E5E7BAF1000F10D0CB
:1026E000002304AA092120460593FFF721FB0528B2
:1026F00003D018B109B0BDE8F08F3546059B1B68C3
:102700003BB135B9019A2BF817407B1C9A421F4602
:1027100007D92046FFF770FF4FF6FF739842044633
:10272000B3D1C9F800700020E4E70820E2E70E20EA
:10273000E0E70720DEE7BAF1000FE3D0029DCFE724
:1027400066300020F7B51C460C4B1B7806460F463A
:1027500015467BB182B17CB108220021684602F0A7
:102760002DFF23466A46394630460195FFF7E0FAC9
:1027700003B0F0BD0820FBE70E20F9E7663000202B
:1027800007B502AB502223F8022D0A460721FFF7B6
:10279000D9FF03B05DF804FB034B1B780BB1FEF7C8
:1027A00025BF0820704700BF6630002070B51A4B67
:1027B0001B7886B063B3194E01234FF6FF70337058
:1027C000FFF774FB4FF6FF73984205460CD01E4688
:1027D0002846FFF7E1FF0446E0B92846FFF766FB0D
:1027E000B0420546F4D110E0002418222146684684
:1027F000347002F0E3FE0C2368468DF80030ADF82B
:102800000450ADF80250FFF705FE204606B070BD3B
:102810000824FAE70324F8E766300020543000204B
:102820002DE9F04F87B0CDE900232F4B1B7882466E
:102830008946002B55D04FF6FF70FFF737FB042376
:10284000ADF80A300DF1100B03AB002505935A4685
:102850000DF10A030621044603950495FFF768FA73
:1028600007283AD04FF6FF76B0464FF0FF37F0B169
:10287000052825D04FF6FF739C4230D1A0452AD0C1
:10288000A6420CBF05200020BAF1000F01D0AAF823
:102890000080B9F1000F01D0C9F80050009B03B1CE
:1028A0001E80019B03B11F6007B0BDE8F08F039B42
:1028B000AB4224BFA0461D46BB423CBF26461F4636
:1028C0002046FFF7F3FA0DF10A035A4606210446A3
:1028D000FFF72EFACBE70520D6E70520E4E7032033
:1028E000E2E70820E0E700BF6630002008B50023DB
:1028F0001A4606490648FFF793FF28B1431F58427E
:102900005841044B187008BD0120FAE750300020F0
:102910006430002068300020F0B5044687B080881D
:10292000FEF7F6FD23786080083B032B20D8DFE814
:1029300003F002213166637A5BB9404A116851B1F4
:10294000E068814207D113603D4AA1881180E360AD
:102950000EE0012B0CD13B4B1B784BB1384BA288BE
:102960001B889A4204D1237A062B01D1FFF7BEFFC0
:10297000204660E0637A002BFAD1304A11680029C2
:10298000F6D0E0688142F3D12F4913600A68013A1A
:102990000A60DCE72D4F3B7873B90125294B1B7882
:1029A00033B1274BA2881B889A4201D1FFF79EFFC3
:1029B000002DDDD107B0F0BD4FF6FF70FFF776FABE
:1029C0004FF6FF7398420546E7D1FFF771FAA84228
:1029D0000646E2D100251822294668463D7002F0DD
:1029E000EDFD0C2320468DF80030ADF80460ADF805
:1029F0000260FFF70FFD6846FFF70CFDCEE7134BB3
:102A00001A78002AB4D0002118226846197002F002
:102A1000D5FD0D238DF800304FF6FF73ADF804306F
:102A2000ADF80230A36802932046237B8DF80C306A
:102A3000FFF7F0FC6846FFF7EDFCBBE76C300020C9
:102A400064300020683000205030002054300020D6
:102A50002DE9F041304B1B7888B00646002B56D04C
:102A60002E4B2F4C93E8030022786F4687E8030033
:102A70000AB9FFF73BFF23781BB9112008B0BDE866
:102A8000F081284B1C689846002CF6D1264A274D29
:102A900012882B68B24220D10BB31822214602A81B
:102AA00002F08CFD082330468DF80830FEF730FD2B
:102AB00006238DF810309DF81830ADF80A0064F345
:102AC000000302A8ADF80C608DF8114005948DF854
:102AD0001830FFF79FFC2046D0E75A1C19D001336D
:102AE000104A2B6039463046FFF78EF90028C5D0D2
:102AF0000023C8F800302B68112803F1FF332B6046
:102B0000BBD08628BAD0072818BF0320B6E7082014
:102B1000B4E71320B2E700BF663000208C580200F3
:102B2000683000206C3000206430002050300020DD
:102B300076DF704713B5044669B901A9FFF726FD92
:102B400043F20202904202D008B1F9F7E7FD9DF886
:102B500004309B070CD400212046FFF7DBFC38B182
:102B6000112805D00D2805D113212046FFF7E0FFDD
:102B700002B010BD0B28FBD043F202029042F7D006
:102B8000F9F7CCFDF4E7017811B94088FFF7D2BF1F
:102B9000072903D1806808B1F9F7C0BD704700006C
:102BA0002DE9F041037886B00446142B3CD8DFE8C9
:102BB00003F00B3B2D3B3B3B3E3B653B653B3B3BCF
:102BC0003B3B3B3B3B698F008088FFF741FF8628FA
:102BD00001D0112811D14449444A0B68A08822F839
:102BE000130001335A4202F0070203F0070358BFF3
:102BF00053420B6000F082F816E0132803D83C4BD8
:102C0000C340DB0710D4F9F789FD0DE0037A012BEF
:102C10000AD8848818220021684602F0CFFC684652
:102C2000ADF80440FFF7BCFF06B0BDE8F081314EBF
:102C30003278002AF8D1304D2B78B3B96A4619465C
:102C40001846FFF7EDFD044648B9BDF80000FFF750
:102C5000A3FD044608B1F9F761FD01232B70631F42
:102C6000012BE1D90CB12046CDE7FAF7D3FC10B91E
:102C700001233370D8E70828D6D0C4E71E4B0122C1
:102C80001A70D1E71B4B194D00241C701A4B1C7095
:102C9000154B1F684FF6FF763B195A4202F00702A8
:102CA00003F0070358BF534235F81380B0450BD0EB
:102CB00018220021684625F8136002F07FFC684660
:102CC000ADF80480FFF76CFF0134082CE4D1ABE7CA
:102CD000084B00221A70037B002BA5D083680E2BB3
:102CE00088D0012BA0D185E774300020F61D00208C
:102CF000C100080070300020713000207FB518221C
:102D00000021684602F05AFC062368468DF8003020
:102D1000FFF746FF07B05DF804FB70B5DDE904542A
:102D200068B161B15BB104FB05F6964207D835B1D5
:102D30002CB1C0E90013C0E90254002070BD072087
:102D4000FCE738B50C46054608B9002038BD0368D5
:102D5000002BFAD040680028F7D0FF29F5D0BFF348
:102D60005F8FFAF774FD0028EFD0EB68286803FB4B
:102D70000400EBE738B50D46044690B1036883B113
:102D8000406870B1FF290CD0BFF35F8FFAF75FFD89
:102D900038B16068BFF35F8F2946BDE83840FAF765
:102DA0004CBD38BD2DE9F0418846064618B9FF24D0
:102DB0002046BDE8F0810368002BF8D04368002B63
:102DC000F5D00027FF24B368FDB2AB42EFD9294606
:102DD0007068FAF724FDBFF35F8F40B9FF2C08BF7E
:102DE0002C462D1B01354545E2D00137EBE7FF2C82
:102DF00007D1FF24F9E721463046FFF7BBFF013436
:102E0000E4B2A542F7D8F4E77EDF70477FDF704772
:102E100086DF704710B50378182B044602D1FDF702
:102E2000B5FC207010BD10B504464088FEF742FB8B
:102E3000A0802046BDE8104000F036BC10B586B03A
:102E4000044618220021684602F0B8FB04236846B5
:102E50008DF80030ADF80240FFF7E5FF06B010BD79
:102E600030B587B005460C4618220021684602F0AE
:102E7000A5FB072368468DF80030ADF80250029498
:102E8000FFF7D1FF07B030BDF0B587B004460F465D
:102E900016460021182268461D4602F08FFB0323C8
:102EA0008DF80030094BADF80240002219788DF8FA
:102EB00008702046ADF80A608DF80C50FDF788FCCC
:102EC0006846FFF7B0FF07B0F0BD00BF071E002047
:102ED0007FB502238DF800300388ADF802304379C6
:102EE0008DF8091013F0040F14BF01230223684664
:102EF0008DF80830FFF797FF07B05DF804FB00007E
:102F000030B5114B0A1C87B00C4618BF0122197846
:102F10000546FDF75DFC631E5A425A410B4B28469D
:102F20001978FDF755FC18220021684602F046FB8F
:102F3000012368468DF80030ADF802508DF8084046
:102F4000FFF771FF07B030BD091E0020081E0020EA
:102F50002DE9F041154B0D46197804461646FDF74C
:102F60001FFC0146F0B1124B20461978FDF718FC02
:102F7000002804F580704FF0070180B214BF0127CC
:102F80000227FFF763F9014620B1052802D0204649
:102F9000FFF766FF33462A4639462046BDE8F04132
:102FA000FFF772BF33462A46F7E700BF091E00202D
:102FB000081E0020024B0A781978FDF709BC00BFF3
:102FC000061E0020F8B5104F104E114D114C38461A
:102FD000FFF720FF3046FFF71DFF2846FFF71AFFD7
:102FE0002046FFF717FF3B78182B0BD03378182BB0
:102FF00008D02B78182B05D02378182B0CBF032072
:103000000020F8BD0320FCE7071E0020091E002059
:10301000081E0020061E00202DE9F0418AB00F4650
:1030200090460446FDF770FB20220646002102A8C8
:1030300002F0C4FA012E1FD1364B00221978204627
:10304000FDF7C6FB002F5DD02046FEF733FA4FF6A2
:10305000FF73984215D100253B78DB0725D42E4B12
:10306000CDF814800993012E51D102AB3A4629467E
:103070002046FFF7CBFE26E0002E45D143F20200AA
:1030800021E0012EE7D1234D20462978FDF788FB6A
:103090000028E0D12046FFF7D1FE29782046FDF731
:1030A0007FFB0028D7D18525D6E7852DDBD004F519
:1030B00080706B460122072180B2FFF767F8112864
:1030C00001D018B103200AB0BDE8F08101465022BA
:1030D000019802F073FA019B1E700199CDF81480DB
:1030E00001F13403029301F1180306934B1C07937B
:1030F0001131094B09932046FEF7EEF90028B2D0B2
:103100000820E0E78525B0E7002F9DD1852502AB9B
:103110000022ACE7061E00207830002038B50546B6
:103120000C46FDF7F1FA012808D154B12146284692
:10313000FFF76AFE042808BF112038BD43F20200E1
:10314000FBE72046F9E700002DE9F0470388113B33
:1031500088B00446092B73D8DFE813F00A00720028
:103160001F00470072007200720072009F002A0167
:10317000037A85883D2BA54B2846197841F23D04FA
:1031800018BF4FF48854FDF70BFB002858D00022DD
:1031900021462846FFF7DCFE52E08088FDF7B4FAAE
:1031A000012802460FD1237AA58813F0010F974B0F
:1031B0000CBF0226012619782846FDF709FB314687
:1031C0002846FFF79DFE34F8045F1822002102A86C
:1031D00002F0F4F9043405238DF80830ADF80A50F4
:1031E000049402A8FFF71FFE2AE000F11006304603
:1031F000FEF7D1F94FF6FF7398420546A08822D119
:10320000FEF758F90546814BA78819780122384600
:10321000FDF7DEFA00213846FFF772FE4FF6FF7326
:103220009D4214D10025002329461A46A088FFF7A5
:10323000EFFD0828014603D010B3A088FFF710FE69
:1032400008B0BDE8F0872946FEF7C6F9DBE702AA19
:1032500007212846FEF796FF0028E3D1A37ED90771
:10326000E0D5039D95F84430DA0701D53435DAE727
:10327000314605F14600FEF77AF90028F6D1D1E78C
:10328000A37EDB07DCD5002DDAD1A0882B4641F2E6
:1032900006022946FFF7F8FDD2E75C4B067A19785B
:1032A0008788002E77D100F1040832463846FDF7B2
:1032B0008FFA617A11F0040103D14046FFF708FE4E
:1032C000BEE707F580791FFA89F96B4601220721CD
:1032D0004846FEF75BFF054628B101463846FFF732
:1032E000BFFD3146E9E73846FEF7E4F84FF6FF73D5
:1032F0009842044682462ED101460198FEF7BCF85A
:1033000050450446064676D0DFF808A10146384607
:10331000FEF762F99AF800103846FDF741FA0646C2
:10332000C8B93846FFF78AFD9AF800103846FDF70D
:1033300037FA01460028C0D0072122464846FEF74A
:10334000B0FF014648B90121B7E721463846FEF7EC
:1033500043F90126F0E72E46EEE786280DD1182224
:10336000002102A802F02AF9062302A88DF80830ED
:10337000ADF80A70FFF757FDE5E73846FFF770FD37
:1033800000214046FFF7A4FD002E3FF459AF204630
:10339000FEF72CF954E7447A384604F00304FDF7AD
:1033A000FFF900283FF44CAF224631463846F1E69B
:1033B000174B80881978FDF7F3F9054600287FF44C
:1033C0003FAFA088FDF7B2F90146A08819B90123E3
:1033D00041F206025EE70D4B2A461978FDF7F8F92F
:1033E00002238DF80830A388ADF80A308DF810500C
:1033F0008DF81150F5E6FEF746FDB0420446A4D123
:1034000004213846FFF72CFD294656E7071E002009
:10341000091E0020061E002058B3027802F0820325
:10342000802B25D0C2F30213042B21D802F0F20323
:10343000322B1DD041788378994219D8062917D9A3
:10344000102B15D8C17811F0040311D1007943076E
:103450000ED4084301070BD4D30700F0030003D4B4
:10346000B0FA80F040097047003018BF0120704763
:103470000020704710B50378182B044602D1FDF7E1
:1034800085F9207010BD70B586B006460C4615460D
:1034900000211822684602F091F83046ADF802602B
:1034A000FEF708F80D2CADF8040019D103238DF8B0
:1034B00000309DB12B7813F0010F0CBF02230123C4
:1034C0008DF8083000238DF80C3041F20113ADF86F
:1034D0000A306846FEF7C4FF06B070BD0223EFE76E
:1034E00007238DF80030002302948DF80C30F0E7AC
:1034F00030B587B005230D4614468DF80030ADF881
:103500000200FDF7D7FFADF804006846CDE902548C
:10351000FEF7A6FF07B030BD2DE9F043054687B0A2
:10352000904699460E46D9B92C4BCDE904111B683B
:10353000039306AA12E907006B4683E807001A46C0
:1035400031462846FFF7D4FF254B009F1B7843B92F
:103550009DF809302BB90526304607B0BDE8F08349
:103560000027424639462846FFF7D8FDA0F111034F
:103570005A425A411B4B044619782846FDF728F950
:103580000B2C03D004D80CB1082C17D1264616E01A
:10359000112C05D043F202039C42F7D00D2CF4E726
:1035A000114B324619782846FDF712F90F4B424667
:1035B00019782846FDF70CF90026CDE70326B9F166
:1035C000000FC9D034F00803C6D0112CC4D03A463D
:1035D00021462846FFF757FFBEE700BFC430002052
:1035E000C13000200C1E00200B1E00200A1E0020EF
:1035F00070B5094B19780446FDF7D2F8074B05461C
:1036000019782046FDF7CCF82A46014601232046CA
:10361000BDE87040FFF780BF0A1E00200B1E00208F
:1036200070B51B4B86B00026CDE904661B6803937A
:1036300006AA04460D4612E907006B4683E8070018
:103640001A4629462046FFF753FF124B00991A6885
:103650002046FFF7E1FCA0F111035A425A410E4BFC
:10366000054619782046FDF7B3F80C4B3246197819
:103670002046FDF7ADF835F0080306D0112D04D033
:10368000009A29462046FFF7FEFE06B070BD00BF37
:10369000C4300020B83000200D1E00200C1E002079
:1036A0000021FFF7BDBF000010B50378052B0446CD
:1036B00006D0122B0AD02046BDE81040FEF7D0BE3F
:1036C00081684088BDE81040FFF7AABF0C4B1B681B
:1036D0009BB10C4B017A1B7803F0010291420CD88C
:1036E000417AC3F34003994294BF00210121012391
:1036F00000226088FFF710FFDDE70121F7E700BF38
:10370000C4300020BC30002008B50378083BDBB291
:103710000B2B14D8012202FA03F340F60F021342D6
:103720000DD0074B074918780022FDF779F8064BB2
:10373000064918780022BDE80840FDF771B808BDB9
:103740000D1E0020A13602000C1E0020F1350200E3
:1037500010B50948094CFFF78DFE0948FFF78AFEAE
:103760000848FFF787FE2046FFF784FE2378182BD2
:103770000CBF0320002010BD0C1E00200D1E0020D9
:103780000A1E00200B1E002008B5FFF7DDFC074BCA
:10379000074918780022FDF743F8064B06491878C8
:1037A0000022BDE80840FDF73BB800BF0D1E002019
:1037B000A13602000C1E0020F135020010B50446AF
:1037C00030B90A4B18600A4B01221A70002010BD54
:1037D000FFF722FE38B1074B22681A6022791A716E
:1037E000024A1360EFE70720F1E700BFC430002072
:1037F000C1300020BC300020FFF7DCBB00230A46AC
:103800001946FFF789BEA8DF7047ACDF7047AEDF0F
:10381000704737B505460C46E1B1D8B10388502B47
:1038200018D14B7CB3B1C2884B899A4212D1038A1A
:10383000022B0FD10B686BB11230FDF749F858B16C
:1038400000238DF80430AB88ADF8063001A9236859
:103850002046984703B030BD0123F2E72DE9F0413F
:103860000E4690B00446002867D0002965D00B684A
:1038700003600B79437410A9FF23037441F60F030F
:10388000012021F8383D221D8DF80A00FFF7BBFF0B
:10389000054600284BD12022337B8DF803300146AA
:1038A0000DEB020001F08AFE42F61923ADF820303C
:1038B0004FF0011309930DF10303627C0A939DF805
:1038C0002D30A08862F30413DBB243F002038DF8BD
:1038D0002D30B37B8DF83330A21D737B8DF83130E2
:1038E00008A9FDF70CF8054608BBB16819B30DF13E
:1038F00004084046FCF7F4FF29460746142203A8B3
:1039000001F05CFEB8B242F60813ADF80C30ADF829
:103910001600F37BADF81A0004F10E0203A9E0884B
:103920008DF81230CDF81C80FDF790F8054628463A
:1039300010B0BDE8F081E081F9E70E25F7E72DE949
:10394000F04194B017468DF807100546002858D06E
:10395000027CCBB29A4256D003AE082200213046F8
:1039600001F02CFE4FF001080DF107033246E98803
:10397000CDF80C804FF6FF700493FFF746FF044626
:1039800008BB9DF807302B746B7C002B3DD00146A3
:10399000102205A801F012FEEB88ADF81430BDF836
:1039A0000E30ADF81830049B08934FF6FE739F421B
:1039B0008DF8168007961ED109A8FCF7D3FE254680
:1039C000099BAB4203D8204614B0BDE8F08109AB97
:1039D00003EB45039E883046FCF798FE022805D18C
:1039E00005A9304624B9FFF712FF04460135E7E781
:1039F000FFF70DFFFAE705A93846FFF708FF044671
:103A0000E1E70E24DFE70024DDE70824DBE7A8DF99
:103A100070470000F0B5074689B014461E460D46B3
:103A200011B90846F8F77AFE14B92046F8F776FE81
:103A300020220021684601F0C1FD9DF80D300E9A4C
:103A4000ADF8007043F002038DF80D30064BADF871
:103A5000044069461888ADF8064002958DF811605B
:103A6000FCF74DFF09B0F0BD0031002030B587B044
:103A700006A941F60A03044621F80C3D01205A4AE2
:103A80008DF80E00FFF7C3FF0546002849D12288B4
:103A9000002A49D1228952B15449009194F83C300E
:103AA000E16842F62420FFF7B5FF002847D1228ABB
:103AB00052B14F49009194F83C30616942F625209B
:103AC000FFF7A8FF00283AD1228B52B14949009153
:103AD00094F83C30E16942F62720FFF79BFF00286D
:103AE0002DD1228C4AB14449009194F83C30616A4E
:103AF00042F62620FFF78EFF08BB228D4AB13F49D0
:103B0000009194F83C30E16A42F62820FFF782FFEA
:103B1000A8B9236BABB9616B002938D1A36B002B1B
:103B200042D1284607B030BD3549009194F83C3069
:103B3000616842F62920FFF76DFF0028AAD00546EC
:103B4000EFE71A688DF810201A68120A8DF8112014
:103B50005A888DF81220DA788DF813205A688DF87B
:103B600014209B688DF815301A0A8DF816201B0C4E
:103B7000244A8DF81730009294F83C30082204A9AA
:103B800042F62320FFF746FF0028C4D0D7E71E489F
:103B90000A79009094F83C30096842F62A20FFF731
:103BA00039FF0028BAD0CAE71A788DF810205A8851
:103BB0008DF81120120A8DF812209A888DF81320A2
:103BC000120A8DF81420DB888DF815300F4A009208
:103BD0001B0A8DF81630072294F83C3004A942F6EF
:103BE0005020FFF717FFAAE700310020E030002047
:103BF000F8300020D0300020C830002002310020F2
:103C0000D83000200A310020F0300020E8300020B9
:103C1000A8DF7047A9DF7047ACDF7047AEDF7047A1
:103C2000B0DF704764DF70472DE9F04315468BB075
:103C3000044688466A46A988D0F878011F46FCF7F2
:103C400007FE10B1636803B19847009E8EB3002150
:103C5000102201A8B5F80E9001F0B0FC01238DF8F8
:103C600004300023ADF80830BDF84830A888ADF81E
:103C70000C90A3EB0903ADF80E309DF80A304F44C9
:103C80003E4443F0010301A904968DF80A30FFF782
:103C9000C7FF10B1636803B1984723684BB107228F
:103CA0008DF81420D8F800200692099505A9204621
:103CB00098470BB0BDE8F0832DE9F04186B005468A
:103CC0000C4617468988D0F878016A469846FCF772
:103CD000BFFD10B16B6803B198470098F0B1228A1C
:103CE000E389BDF8301013448B4217DC04F112064F
:103CF0003146404401F057FC2B687BB104228DF81B
:103D000004203A680292E289ADF80C20228AADF8CC
:103D10000E20CDE9046401A92846984706B0BDE805
:103D2000F081F0B513241C80D0F87C41059E4CBB7B
:103D3000D0F88041002C49D1D0F88441002C67D1C3
:103D40000020F0BDD0F87C7137F834401F883C4427
:103D50001C80877CECB2A742EAD90CFB0407013532
:103D6000B7F814E08E454FEAC407EBD142F64D2375
:103D7000138001239370D470D0F87C21D25B328001
:103D80000120DEE700254FF00A0CE2E7D0F8807151
:103D900037F834401F883C441C8090F87870ECB2AF
:103DA000A742C9D90CFB04070135B7F87AE0714581
:103DB0004FEAC407EAD142F64D23138002239370E1
:103DC000D470D0F88031DB5B3380D9E700254FF029
:103DD0000A0CE2E7D0F8847137F834401F883C447D
:103DE0001C8090F8DE70ECB2A742A9D90CFB040746
:103DF0000135B7F8E0E071454FEAC407EAD142F671
:103E00004D23138003239370D470D0F88431DAE704
:103E100000254FF00A0CE4E7F0B5168A022E87B0B1
:103E200004460F4615460FD103686BB102F112002C
:103E3000FCF74EFD50B18DF804603B680293059588
:103E4000236801A92046984707B0F0BD03238DF8E9
:103E50000430F2E72DE9F0438FB0DDE9164507465F
:103E6000884691460021202206A81E4601F0A6FBA6
:103E700042F64D23ADF8183098F800308DF8253013
:103E800023788DF8293063788DF82A30A3788DF85F
:103E90002B302A46012306A93888ADF81C908DF8EE
:103EA00024308DF82730FCF72AFDF8B9142201469A
:103EB00001A801F083FB42F60813ADF80430237823
:103EC0008DF80A30314663788DF80B306846FCF780
:103ED00007FD80B2ADF80E00ADF8120005F1080242
:103EE00001A92888CDF814D0FCF7B0FD0FB0BDE8CB
:103EF000F083F0B5144689B005460F462022002114
:103F000068461E4601F05AFB61789DF80D208DF839
:103F100012100823ADF804300B1C18BF012342F027
:103F2000020263F3C302D2B223788DF8113042F05B
:103F30001002A3788DF80D208DF81330324601233E
:103F400069462888ADF800708DF80F30FCF7D7FC73
:103F500009B0F0BD30B587B004460D4601AA898886
:103F6000D0F87801FCF774FC10B1636803B198478E
:103F7000019BFBB11022002102A801F01FFB0123CD
:103F80008DF80830ADF81230019B05939DF80E3086
:103F9000A8880022ADF80C2043F00103EA89ADF8AF
:103FA000102002A98DF80E30FFF73AFE10B16368B9
:103FB00003B1984707B030BDF0B50388502B8BB0E4
:103FC00005460C4658D0512B00F00481102B40D1EF
:103FD0000AAA0023818842F8183DD4F87801FCF73A
:103FE00037FC10B1636803B19847049888B3D4F8DC
:103FF0007C11002934D0A67C00231322B3422AD39B
:10400000D4F8801121B194F878600023B34229D309
:10401000D4F8841121B194F8DE600023B34226D392
:10402000002101F0CBFA63899BB1049B01261E702D
:104030000822002105A801F0C1FA049B6189A88823
:10404000059605AA0693FFF7E7FD10B1636803B173
:1040500098470BB0F0BD31F8337001333A44CDE7E7
:104060001322CDE731F8337001333A44CEE731F80B
:10407000337001333A44D1E7C188B4F86E010223AA
:1040800000228842ADF80C30ADF80E201ED104AAF3
:10409000A988D4F87801FCF7DBFB10B1636803B1A1
:1040A0009847049A002AD4D02B8A012BD1D1AB7C1B
:1040B0000BB1012BCDD18DF8143053702368002B38
:1040C000C7D0099505A920469847C2E7608988426C
:1040D0001AD104AAA988D4F87801FCF7B9FB10B169
:1040E000636803B19847049A002AB2D02B8A012B47
:1040F000AFD1AB7C1BB1012BABD1062100E0052178
:104100008DF814101370D9E7B4F85201884209D120
:104110000AA942F6222341F8143D2A462046FFF719
:104120007BFE96E7B4F84E01884204D142F6222283
:10413000059208220AE0B4F856318B420FD142F6BC
:10414000322305930A23ADF80C300122ADF80E207E
:104150000092294605AA2046FFF7AEFD79E7B4F89C
:1041600062318B4203D10AA942F63323D3E7B4F874
:104170005E318B4215D0A07C13460A26DAB2824209
:1041800016D30DF10E03009305AA03AB2046FFF7EB
:10419000C8FD00283FF45DAFBDF80C30BDF80E201F
:1041A000D6E742F6332305930B23ADF80C30C0E776
:1041B000013306FB0347FF898F42DFD142F64D23CF
:1041C000ADF8143001238DF817208DF816302A46EB
:1041D00005A9A3E70022ADF8102082790223012A65
:1041E000ADF80E307FF435AF01896089884204D183
:1041F00029462046FFF7AEFE2BE7B4F84E01884271
:1042000004D142F622220592082209E0B4F8563180
:104210008B420ED142F6322305930A23ADF80E30BD
:10422000ADF81020009205A92A462046FFF7FCFCB5
:104230000FE7B4F85E318B4206D142F63323059383
:104240000B23ADF80E30DFE704AB009305AA0DF1A8
:104250000E032046FFF765FD00283FF4FAAEBDF8D7
:104260000E30BDF81020DDE72DE9F04F0C4697B079
:104270000546002800F01282002900F00F828B7A98
:104280000A2B00F28B800B7C0A2B00F287800B7EBE
:104290000A2B00F283800B6803604B6843608B7AC3
:1042A00083740B7C80F878300B7E80F8DE3016A9A2
:1042B00041F6120305F10807012021F8483D3A466E
:1042C0008DF81200FFF7A4FC002873D1034694F880
:1042D0003620D9B28A4263D8238943B301262022EB
:1042E00000210EA894F83C9094F83D808DF824604D
:1042F00001F064F942F64E23ADF838304FF0011367
:104300000F9309AB10939DF8453028898DF849909B
:1043100043F0060305F10A020EA98DF845308DF829
:104320004A808DF84760FCF7EAFA002842D1A37A68
:10433000002B42D1237C002B7DD1237E002B40F02B
:10434000AB80202200210EA801F038F942F64B2361
:10435000ADF83830A38CADF83C30ADF83E30236A70
:1043600010939DF84530288943F002038DF84530BD
:1043700094F82C308DF8493005F5A27201230EA96E
:104380008DF84430FCF7BBFAA0B994F82630002B26
:1043900000F0E380A36A002B40F07081072009E061
:1043A000A06B0EAA30F811102889FFF733FC0133F7
:1043B00000288CD017B0BDE8F08FE368002BB9D08F
:1043C0004FF000084FF00A092FE0012200210EA84B
:1043D000D4F80CB001F0F2F89DF838300BEBC60AB7
:1043E00043F002038DF838309AF805309DF83820F4
:1043F000003318BF012363F3C302D2B242F01002AC
:104400008DF838203BF8362009FB06560AF10403E4
:104410001436009301960AF102030EA93846FFF7FD
:1044200019FD08F101080028C4D1A37A5FFA88F6C3
:10443000B342CAD87EE76369002B3FF47EAF4FF0EA
:1044400000084FF00A0921E0012200210EA8D4F84B
:1044500014B001F0B3F89DF8383043F00E038DF836
:1044600038303BF836200BEBC60A09FB06560AF13A
:1044700004037A36009301960AF102030EA9384626
:10448000FFF7E8FC08F10108002893D1237C5FFACC
:1044900088F6B342D8D850E7E369002B3FF451AF18
:1044A0004FF000084FF00A0922E0012200210EA877
:1044B000D4F81CB001F082F89DF8383043F00A03BC
:1044C0008DF838303BF836200BEBC60A09FB065650
:1044D0000AF10403E036009301960AF102030EA9E3
:1044E0003846FFF7B7FC08F1010800287FF462AFF7
:1044F000237E5FFA88F6B342D7D822E7A06A424605
:104500000DF10F0100EB8600FFF78CFB00287FF414
:1045100051AF0146142209A801F050F842F60713E2
:10452000ADF8243094F82C308DF82A3005F5A672B9
:104530009DF80F30B5F84401ADF82E3009A9ADF85B
:104540003230CDF83480FCF781FA00287FF432AFA6
:10455000013694F826309E42D0DB237A83B305F5EA
:10456000A77304F1420242F622213846FFF7C1FC4C
:1045700000287FF41FAF014620220EA801F01EF88C
:1045800042F63223ADF838309DF84530288943F0A3
:104590000E0301228DF8453094F84530ADF83C20EB
:1045A0008DF849308DF8472094F846308DF84A3020
:1045B00005F5AB720EA9FCF7A2F900287FF4FAAE5C
:1045C000637A002B5ED1238E8DF824301B0A8DF880
:1045D000253094F832308DF82630202294F833308C
:1045E0008DF8273000210EA800F0E8FF42F64A239C
:1045F000ADF838309DF84530288943F002038DF836
:10460000453094F834308DF8493009AE4FF004133A
:1046100005F5B3720EA90F931096FCF770F90028F8
:104620007FF4C8AE01468DF8240020220EA894F82D
:104630003E7000F0C3FF42F64C23ADF838309DF8D1
:10464000453028898DF84A7043F004038DF84530D1
:1046500005F5B7724FF001130EA9CDE90F36FCF73F
:104660004EF900287FF4A6AEE368C5F87C31636993
:10467000C5F88031E369C5F884319BE606460DF143
:10468000140866E705F5AF7304F13F0242F63321E3
:104690003846FFF72EFC002895D08BE60E2089E6E1
:1046A0002DE9F04186B00C4616469846BDF83070AC
:1046B000054600284DD0002B4BD0837C8B424AD935
:1046C0004FF6FF739F4248D0ADF80220394601AA49
:1046D000D0F87801FCF7BCF878BB019BD5F87C21B9
:1046E00013330193C3B29C422AD832F83430B34218
:1046F0002DD332464146019800F055FF002110228B
:1047000002A800F05BFF0A2303FB045402A9A38A5A
:10471000ADF8083001238DF80A300023ADF80C30D5
:1047200038460DF10203CDE90438FFF777FA20B9D6
:10473000049B1B88B34218BF0C2006B0BDE8F08173
:1047400032F83010019B0B4401930130CAE70C2072
:10475000F3E70E20F1E70720EFE70820EDE7F0B5DB
:104760000C4687B016461D460746002836D0AAB329
:104770004FF6FF739D4233D0ADF8021001AA2946CF
:10478000D0F87801FCF764F830BB0198082C00F1F0
:104790000200019003D82246314600F004FF0021B8
:1047A000102202A800F00AFFB7F84E31ADF8083029
:1047B00001238DF80A300023ADF80C3002A90DF169
:1047C00002032846CDE90436FFF728FA20B9049BF6
:1047D0001B88A34218BF0C2007B0F0BD0E20FBE7DA
:1047E0000820F9E72DE9F7430B9F0E4690469946BE
:1047F000054600283CD0002F3AD090F878308B4204
:1048000038D901AABDF82810D0F87801FCF720F8B3
:104810000446C8B9019BA97C133301930246D3B265
:10482000994215D8D5F880110022D3B29E4218D8EB
:1048300031F8363008EB09029A421DDC01994246F4
:104840004944384600F0AFFE204603B0BDE8F0838F
:10485000D5F87C3133F83200019B034401930132D7
:10486000DDE731F83200019B034401930132DCE7BC
:104870000E24E9E70724E7E70924E5E7A8DF704706
:10488000AEDF7047B0DF704762DF70473CDF7047D4
:104890003DDF7047704700007FB5044638B103889C
:1048A000502B5AD005D8102B17D0112B19D004B08B
:1048B00070BD512B1DD0532BF9D12E4DC288EB88E2
:1048C0009A42F4D16B7E002BF1D000F095F90028CC
:1048D000EDD06B6902209847E9E78288254B9A80E2
:1048E000E5E7244B81889A889142E0D14FF6FF7228
:1048F000F5E7204D8288AB889A42D8D18679022E7E
:10490000D5D10289EB889A42D1D1837B043B022B1B
:10491000CDD910220021684600F050FE2B7E8DF884
:104920000060BBB19DF8063043F001038DF80630FE
:104930000023ADF804306946A888FFF7A3FF1128CB
:10494000F9D0BDF80430002BB1D104F1080000F01B
:10495000FFF8ACE740F2FD13EBE7064DC2886B8928
:104960009A42A4D1038A022BA1D11230FBF7B4FFE3
:1049700028769CE71431002030B587B005460C46F8
:104980001022002102A800F019FE0323ADF8023026
:1049900020238DF804300F4B8DF80550DA88ADF8E0
:1049A000082002228DF80A200022ADF80C200DF11B
:1049B0000202049202A901AA98888DF80640059285
:1049C000FFF75EFF20B9BDF80230032B18BF0C20A3
:1049D00007B030BD1431002010B54FF0FF3100207A
:1049E000FFF756FF044658B9B121FFF74FFF0446C1
:1049F00030B9044B01205B6998470220F9F7BAF9F6
:104A0000204610BD14310020F0B51C4B87B002AA1F
:104A1000064603F11007154618685968144603C482
:104A20000833BB422246F7D12EB3154B4FF6FF7227
:104A30009A8032685A610021597619760AB9114A6A
:104A40005A610F4800F050F898B906A94FF659631B
:104A5000012021F8143D0C4A8DF80600FFF70EFFE7
:104A600038B907492846FFF70FFF10B9044800F08E
:104A700045F807B0F0BD0E20FBE700BF94580200D8
:104A800014310020954802001631002070B51449F9
:104A90000B6823B34B6813B30831984708281ED01E
:104AA000104C2368254658B9987601210220FFF75B
:104AB00063FFA0B123685B690320BDE8704018471D
:104AC00000229A7606210220FFF756FF18B12368CC
:104AD00003205B6998472B6802205B69EDE770BD96
:104AE000503100204C31002018B1034B18600020D9
:104AF00070470E20704700BF4C31002010B588B0C1
:104B0000044620220021684600F058FD2246032377
:104B1000ADF8003012F8063B8DF802309DF80D30EC
:104B2000608843F0280317218DF80D30ADF804108C
:104B3000012369468DF810308DF80C308DF8133054
:104B40008DF812308DF81130FBF7D9FE08B010BD8A
:104B500070B50546007B254C012803D0022825D0DE
:104B6000022117E023689E7E56B10621FFF704FF5D
:104B7000002835D023685B690320BDE870401847E2
:104B800058760146FFF7F8FE50B3236811285E7689
:104B900027D00421287BFFF7EFFE18B123680320FC
:104BA0005B699847236802205B69E6E76A7B531ECE
:104BB000132B18D80E4E05F10E01301D00F0F3FC3A
:104BC0006B7BB36123689B7E002BE2D109493046A1
:104BD00051F8083B98470028DBD1236801229A76D8
:104BE00070BD0621D6E70521D4E700BF4C31002077
:104BF000303100205031002008B5044B1B680020E4
:104C00005B699847BDE80840FFF7E6BE4C310020DD
:104C100010DF704711DF704713B504460949684635
:104C2000F9F7FAF8019808B902B010BDD0E90031DF
:104C30002046984718B16846F9F7F7F8F2E71120CF
:104C4000F2E700BFA858020013B5044607496846BA
:104C5000F9F7E2F8019B0BB902B010BD2046D3E989
:104C6000002190476846F9F7E0F8F3E7C0580200E2
:104C7000064B9A6822B11A6822F480021A607047C3
:104C8000034B4FF48002C3F8802070478433002028
:104C900000E100E00B4991F816335A09EC23134167
:104CA000DB0706D5084B9A683AB94FF480030B60CE
:104CB000704742F20200F7F731BD1A6842F48002F1
:104CC0001A60704700E100E084330020F7B5184F08
:104CD0003C785CBB174E012520463570FFF79CFFE2
:104CE000112820D02046FFF7AFFF134B1868019022
:104CF00002A800F8054DF7F7F5FD104901A8FFF7E8
:104D000087FF0446B0FA80F0400938709DF8030030
:104D1000F7F70CFE3CB90A4B34701C70FFF7BAFF72
:104D20002846FFF791FF204603B0F0BD0824FAE7BC
:104D30005D3100205C310020A458020039C7010019
:104D40005E310020F7B5154F3B7813B3144E0120A8
:104D50003070FFF761FF11284FF000051BD00220D3
:104D6000FFF772FF02A800F8015DF7F7BBFDFFF740
:104D700051FF04469DF807003D70F7F7D7FD2CB9A9
:104D80003470FFF775FF0320FFF75EFF204603B086
:104D9000F0BD0824FAE72C46F8E700BF5D3100209B
:104DA0005C310020054B1B7833B1054B1B780BB1F0
:104DB000FFF7C8BFFFF78ABF082070475C310020AB
:104DC0005D310020014B1878704700BF5D31002035
:104DD00007B508496846F9F71FF8019B13B903B0F6
:104DE0005DF804FBD3E9002090476846F9F71DF809
:104DF000F3E700BFB4580200FFF7EABF002108B58F
:104E0000044A0846F7F7D6FC18B1BDE80840F7F7A2
:104E100085BC08BDF94D020060DF704769DF70474F
:104E200061DF704730B5114B1B7891B0E3B1104D85
:104E300034240DF1020103A8ADF80240FFF7F0FFA2
:104E400070B9294601A8F8F7E7FF029B002BF0D0C4
:104E500003A8D3E90021904701A8F8F7E6FFF4E79B
:104E6000052801D0F7F75AFC11B030BD5F310020A2
:104E7000CC58020030B5054685B00C4600294BD011
:104E8000264B0B600C22002101A800F097FB0623A3
:104E90008DF804502268ADF80830012501A92020C2
:104EA0008DF80650FFF7BAFF0C22002101A800F090
:104EB00085FB22688DF8055001A94020FFF7AEFF61
:104EC0000C22002101A800F079FB22688DF8045023
:104ED00001A92846FFF7A2FF0C22002101A800F03B
:104EE0006DFB4FF4B0632268019301A9A120FFF785
:104EF00095FF0C22002101A800F060FB9DF8043012
:104F000022686FF3000301A9A0208DF80430FFF799
:104F100085FF002005B030BD0E20FBE7481B0020B8
:104F200008B5FFF779FF10B9014B01221A7008BDCF
:104F30005F3100204BDF70471FB50D4C01A8FFF714
:104F4000F9FF70B9214602A8F8F766FF039B002B12
:104F5000F4D00198D3E90021904702A8F8F765FF43
:104F6000F4E7052801D0F7F7D9FB04B010BD00BF66
:104F7000D8580200094A537891780133DBB299423C
:104F800008BF0023117899421FBF0370507818237F
:104F900003FB002014BF0430002070476031002064
:104FA000082910B5044602D00020F7F7B7FBD4E972
:104FB0000030BDE81040184773B5054602A800242C
:104FC00000F8014D0E46F7F78DFC0DF10600FFF7D6
:104FD000D1FF90B106700A4B9DF8062045605A70CB
:104FE0009DF80700F7F7A2FC24B9064B4FF4801296
:104FF000C3F80021204602B070BD0424F0E700BFD2
:105000006031002000E100E0024B4FF43C6043F0CF
:1050100001031847F058020038B50C4B0C4C4FF404
:105020000032C3F8802001254FF48033C4F84833A0
:10503000C4F808336560FFF7E7FF064BA56000245E
:105040001C60FFF7E1FF044B1C7038BD00E100E07D
:10505000001001407C3200206D3200202DE9F34128
:105060002549264B0025C1F84051C1F84451C1F8EB
:105070004851C1F84C51C1F80051C1F804511B68A6
:10508000002B34D0D1F804451D49DFF88880096829
:10509000641A24F07F442F461A68A24212D8A41A38
:1050A00015441A7CDE6962B15A691F7400929B69CB
:1050B0000193424608216846F7F77CFB08B1F7F7F1
:1050C0002DFBBEB90F4B104A197813788B4205D1CE
:1050D0000133DBB2022B08BF0023137012780B4B95
:1050E00043F822500A4B4FF48012C3F8002102B05B
:1050F000BDE8F0813346CFE7001001408032002048
:105100007C3200207832002079320020703200207A
:1051100000E100E0A14F02002DE9F74F9E4A9F49B0
:10512000137809789E4D99423CD00133DBB2022BB3
:1051300008BF002313709B4912789B4B0F6853F8EC
:1051400022003B1823F07F4300220B602B68164699
:105150001446944613B942B12B6006E019688142A7
:105160000ED902B12B60091A19604FF001082B68A3
:10517000DFF83CA200930027BEB9DFF83CB260E044
:10518000401A0C44D968C3F800C0D3F81CE031B110
:105190003A1922F07F42C3E90121DE611E46012255
:1051A0007346D7E70026B046E1E73446F6697D4A04
:1051B00063681268DFF804C2A068991A21F07F4181
:1051C000614500F2A58001442160012222742A6811
:1051D0000023C4E90133E361002A40F0A2802C607F
:1051E000CAE75A1C9BF80210D2B291428BF80020F9
:1051F00004BF00228BF80020182202FB03B32A68A8
:1052000019799C68022974D003297ED0012918D10C
:10521000217CB1B9DA6862601A69A2605A69E260F9
:105220009B69A361614B1B78002BC0D06160BEE716
:105230009C4200F093809946DB69002BF8D1002353
:1052400023749BF800309BF801209A42C9D12B6847
:105250002FB9009A934202D1B8F1000F43D0002B2E
:1052600079D0D3F800A0524D4E4BD5F804751C6888
:10527000DFF84C813E1B98F8003026F07F4603365D
:105280009BB94FF48033C5F84433C5F80433494B18
:105290004FF400324FF00109C3F880211A60C5F8BD
:1052A0000090FFF7B1FE88F80090B2452CBF54443F
:1052B000A41924F07F44C5F84045D5F80435DB1B1C
:1052C00023F07F43E41B033324F07F44A3420AD935
:1052D000D5F80435C5F84035FFF796FE354B4FF449
:1052E0000032C3F80021314B00221A7003B0BDE830
:1052F000F08F13469146A0E71174D2690123002A6A
:10530000FAD1002B9DD02A609BE700231946F6E7CF
:10531000D31A23F07F43834234BFC31A0023236090
:1053200053E721681368994213D8591A1160E26152
:1053300055E7091AD8691A4638B1034618688842F1
:10534000F7D3401A1860184613462160E061DC610B
:1053500012E71346F2E7FFF75FFEC4E74C450DD1B5
:10536000D3692B6053B90F4801920121CAF8081084
:1053700003600E4B1970FFF747FE019AE16923683D
:10538000C9F81C1011B1086803440B602B689A42DD
:1053900018BF012753E700BF783200207932002080
:1053A000803200207C320020703200206C320020DD
:1053B0000010014000E100E060310020FEFF7F00AE
:1053C0006D32002010B5FFF727FE114B00200B2295
:1053D00018809A700F4B18600F4B18700F4B187095
:1053E0000F4B4FF48012C021C3F8802183F81413AF
:1053F0001A6002F18042A2F56F220324C2F8084528
:1054000083F81113074BD2F804251A6010BD00BFB2
:105410006031002080320020783200207932002074
:1054200000E100E07C320020074B9B784BB132B1A9
:1054300028B10368187C20B959745A617047072055
:1054400070470820704700BF603100202DE9F74306
:105450001D4FBB7805460E4690469BB390B304297A
:105460002ED9436973B3437C02A80024012B00F8B2
:10547000014D0CBF8946A146F7F734FA0DF106003D
:10548000FFF778FDD0B101230370104B4560D3F8CE
:105490000435C0E90498C0E902369DF806307B70F7
:1054A0009DF80700F7F742FA24B9094B4FF4801230
:1054B000C3F80021204603B0BDE8F0830424EFE7E1
:1054C0000724F7E70824F5E76031002000100140C9
:1054D00000E100E0064A92783AB130B1426922B167
:1054E000002202740221FFF767BD0820704700BF49
:1054F00060310020044B9B781BB103210020FFF793
:105500005BBD0820704700BF60310020014BD3F81D
:10551000040570470010014008B5074B044613B15D
:105520000021AFF30080054B1868836A03B19847E8
:10553000204600F05BF800BF00000000F8580200B1
:1055400070B50D4E0D4CA41BA4100025A54209D129
:105550000B4E0C4C00F04CF8A41BA4100025A542E7
:1055600005D170BD56F8253098470135EEE756F85D
:10557000253098470135F2E7701E0020701E00208C
:10558000701E0020741E002030B50024A24201D1FC
:10559000002007E0035D01340D1915F8015CAB42F2
:1055A000F4D0581B30BD10B5431E0A44914200D1BF
:1055B00010BD11F8014B03F8014FF7E70244034611
:1055C000934200D1704703F8011BF9E7034611F835
:1055D000012B03F8012B002AF9D17047034613F879
:1055E000012B002AFBD1181A01387047FEE700BFD3
:1055F000F8B500BFF8BC08BC9E467047F8B500BFC0
:10560000F8BC08BC9E467047F1A100F001F000F123
:1056100001F701F801F901FA291E1F202122232494
:105620002526272D2E2A2B141A0815171C180C12A4
:10563000132F303139041607090A0B0D0E0F3334BE
:105640000028E1001D1B061905111036373800E54A
:10565000E0E3E200002C00000000C0E765E4353A1A
:105660003B3C3D3E3F4041424344454CC201520118
:10567000C4C5C6C701B4014A4901C150514F010117
:1056800046474801014D000101004CC3B7A8A9AA33
:10569000014B4E4C0001010101000001000000001F
:1056A00001010101000000000000000000000000F6
:1056B0000338FDD87047100F0E0D0C0B1B030405AB
:1056C00006070809191C1D1E1A000000CC1E002028
:1056D000D41E00200400000001000000D0070000DC
:1056E0000C1F00202C1F00204C1F0020140514014B
:1056F0000304372B82C9809806600C0D000000005F
:105700000824002030250020682500200100060123
:105710000338FDD8704700000000000000000000C2
:105720000338FDD8704700000000000000000000B2
:105730000000000000010101010102020202030356
:105740000304040405050606060707080809090AF4
:105750000B0B0C0C0D0E0E0F10111112131414154F
:10576000161718191A1B1C1D1E1F20212223242561
:105770002627292A2B2C2D2F303133343537383A30
:105780003B3C3E3F4143444647494B4C4E505153AE
:105790005557585A5C5E60626466686A6C6E7072D7
:1057A0007476787A7C7F00000C2700202C2700205C
:1057B0004C2700200000FFFFDEC0ADDEFE011EF121
:1057C000DEC0ADDEFF011EF100100000040000008D
:1057D00001000000C9DA0100A9DA010099DA01002C
:1057E000D9DC01008DDC01006DDA010071DA010005
:1057F00075DA0100685902006C59020004000000CB
:10580000FFFFFFFFFFFFFFFFFFFFFFFFFFFFFFFFA8
:1058100000000000000000000000D60106000000AB
:1058200030313233343536373839414243444546D6
:105830004C6F7436302E47004C6F746C6162000000
:10584000270000001E0000001F00000020000000D4
:1058500021000000220000002300000024000000BE
:1058600025000000260000000100FFFF00000000EE
:105870000100000001000100845802000100010045
:10588000885802000100000000000000010006002E
:105890005030002050EADA308883B89F604F15F30B
:1058A0000000C98E010000076C5902007459020003
:1058B000080000008459020094590200080000000A
:1058C00074590200845902000800000018590200AF
:1058D000685902000800000000590200185902002F
:1058E00008000000000000000000000000000000B0
:1058F0000338FDD870470000101E00200000000093
:10590000A5DB010000000000E10202004C2B00209A
:105910008D4A0200000000001D0602000000000089
:10592000770202004C2B002027190200042C0020D3
:1059300065040200000000003D2402000000000099
:105940006B1A0200182C0020B93F02004C1C0020EA
:1059500013380200AC2C00209948020014310020BA
:1059600041F00100000000000FEF010085DA0100A6
:10597000000000004DDC01000000000099F1010072
:1059800000000000254E020000000000394F020018
:1059900000000000AC38FF7F01000000050000009F
:1059A0008D950100BD950100E1950100EB95010089
:1059B0000196010001FF000014059704741F0020E8
:1059C0000400000014059504901F00201000000042
:1059D00014051405E81F00208C00000001000000E1
:1059E00014059604242200204000000091A4010028
:1059F00079A7010059A4010071A4010019A90100AF
:105A000039A90100F5F8010025A9010005010100EF
:105A10007C2600200090D003000000000020004001
:105A20000000000012180100FFFF05010906A10196
:105A3000857F050719E029E71500250175019508FF
:105A40008102950175088101950575010508190107
:105A500029059102950175039101950675081500B8
:105A600025650507190029658100C005010980A188
:105A7000018502150126B700190129B77510950196
:105A80008100C0050C0901A10185031501269C02B6
:105A900019012A9C02751095018100C000FF0102C6
:105AA00000000000000000000000000000000000F6
:105AB00000000000000000000000000000000000E6
:105AC00000000000000000000000000000000000D6
:105AD00000000000000000000000000000000000C6
:105AE00000000000000000000000000000000000B6
:105AF00000000000000000000000000000000000A6
:105B00000000000000000000000000000000000095
:105B10000000000000000000000000000000000085
:105B20000000000000000000000000000000000075
:105B30000000000000000000000000000000000065
:105B40000000000000000000000000000000000055
:105B50000000000000000000000000000000000045
:105B60000000000000000000000000000000000035
:105B70000000000000000000000000000000000025
:105B80000000000000000000000000000000000015
:105B90000000000000000000000000000000000005
:105BA00000000000000000000000000000000000F5
:105BB00000000000000000000000000000000000E5
:105BC00000000000000000000000000000000000D5
:105BD00000000000000000000000000000000000C5
:105BE00000000000000000000000000000000000B5
:105BF00000000000000000000000000000000000A5
:105C00000000000000000000000000000000000094
:105C10000000000000000000D41D00200000000073
:105C20000000000000000000802C00200100200087
:105C3000EC1D00200000000009F90100D007000061
:105C400000000400020000010000FFFFFFFFFFFF53
:105C5000FFFFFFFFFFFFFFFFFFFF181818181818BE
:105C60001818000000000000000000000000000004
:105C70000000000000000000000000000000000024
:105C80000000000000000000000000000000000014
:105C90000000000000000000000000000000000004
:105CA00000000000000000000000000000000000F4
:105CB00000000000000000000000000000000000E4
:105CC0000000000025920100019201000000000088
:105CD000000000009DD10100000000000000000055
:105CE000E1920100C598010031AC0100DC1D0020EB
:105CF00002000000000000000200000000000000A0
:105D0000020000000000000012000000AC1E002095
:105D100011000000A41E0020100000009C1E0020A6
:105D2000981B0020A81B0020100000009C1E0020D3
:10E00000B41495B4010000000100000001000000FC
:10E01000000000000000000028CD0000F274F15262
:10E0200001000000000000000000000000000000EF
:10E0300000000000000000000000000000000000E0
:10E0400000000000000000000000000000000000D0
:10E0500000000000000000000000000000000000C0
:10F00000B41495B4010000000100000001000000EC
:10F01000000000000000000028CD0000F274F15252
:10F0200001000000000000000000000000000000DF
:10F0300000000000000000000000000000000000D0
:10F0400000000000000000000000000000000000C0
:10F0500000000000000000000000000000000000B0
:00000001FF
